:1000000000800020BD01000021A50000D9A400004F
:10001000D9A40000D9A40000D9A40000D9A40000EC
:10002000D9A40000D9A40000D9A4000021A5000093
:1000300021A50000D9A40000A19B0000A59C000000
:1000400021A5000021A5000021A5000021A5000098
:1000500021A5000021A5000021A5000021A5000088
:1000600021A5000021A5000021A5000021A5000078
:1000700021A5000021A5000021A5000021A5000068
:1000800021A5000021A5000021A5000021A5000058
:1000900021A5000021A5000021A5000021A5000048
:1000A000DD800000E980000021A5000021A50000FE
:1000B00021A5000021A5000021A5000021A5000028
:1000C00021A5000021A5000021A5000021A5000018
:1000D00021A5000021A5000021A5000021A5000008
:1000E00021A5000021A5000021A5000021A50000F8
:1000F00021A500008DC5000021A50000B9C60000A3
:1001000021A50000F9AE000021A5000021A50000F6
:1001100021A5000021A5000021A5000021A50000C7
:1001200021A5000021A5000021A5000021A50000B7
:1001300021A5000021A5000021A5000021A50000A7
:1001400021A5000021A5000021A5000021A5000097
:10015000919D0000A59D0000B99D0000CD9D00006F
:1001600021A5000015B2000021A5000021A5000076
:1001700021A5000021A5000021A5000021A5000067
:1001800021A5000021A5000021A5000021A5000057
:1001900021A5000021A5000021A5000021A5000047
:1001A00021A5000021A5000021A5000021A5000037
:1001B00021A5000021A5000021A50000564B4CF20E
:1001C000205210B51A804DF628121A8000BF00BFC9
:1001D0000AF0AAF9514B4FF010621A60504A9A6027
:1001E000504ADA60504A136813F4807304D14F49BF
:1001F0000B604FF4A85313604D4B1A78110703D5C9
:100200001A7842F008021A704A4B4B492A221A7097
:100210004A4A4B4B8B4204D252F8040F43F8040B6A
:10022000F8E7484B484900228B4202D243F8042B9E
:10023000FAE74649464A002352F8230041F82300D2
:1002400001336F2BF8D1434B434A802103F8011B44
:100250009342FBD1414B3D4A1A60414B8A221A70AE
:10026000A3F5805324225A70A0221A709A7992071B
:10027000FCD59A79D406FCD43A4A937903F00C035E
:10028000082B384BF9D103221A7140225A719A79FE
:100290009006FCD5334A9179324B4906FBD5324A58
:1002A000324911600221516020221A709A7902F0BD
:1002B0000C020C2AFAD12E4B2E4A1A602E4B2F4AD2
:1002C0001A6000225A60072243F8042C2C4AC3F813
:1002D0000C2D62B60AF0D8FC144B1B68DA0705D562
:1002E00028480AF0A5FA284B284A1A60284B1B78A0
:1002F0005B0609D5244C254B22689A4204D121483B
:100300000AF096FA002323600DF08EFC0AF012F931
:100310000AF040F8FEE700BF0E20054030800440A0
:10032000823F04000100002B10D0034014D0034092
:1003300002D0074000E00740F49AFF1FEC0A0100DA
:100340004088FF1FF49AFF1FC0A2FF1F0082FF1FFB
:100350000000000000E400E05FE400E008ED00E0E1
:100360000050064000400640448004400000030165
:1003700004800440C010050014E000E0FF76010096
:10038000000020206DD0D75E1CE00340A5C3945A26
:1003900000F00740FFFFFFFFFFFFFFFFFFFFFFFF32
:1003A000FFFFFFFFFFFFFFFFFFFFFFFFFFFFFFFF5D
:1003B000FFFFFFFFFFFFFFFFFFFFFFFFFFFFFFFF4D
:1003C000FFFFFFFFFFFFFFFFFFFFFFFFFFFFFFFF3D
:1003D000FFFFFFFFFFFFFFFFFFFFFFFFFFFFFFFF2D
:1003E000FFFFFFFFFFFFFFFFFFFFFFFFFFFFFFFF1D
:1003F000FFFFFFFFFFFFFFFFFFFFFFFFFFFFFFFF0D
:10040000FFFFFFFFFFFFFFFFFFFFFFFFDEF9FFFF23
:1004100010B5054C237833B9044B13B10448AFF33E
:1004200000800123237010BDF49AFF1F000000001C
:10043000F00A0100084B10B51BB108490848AFF39A
:1004400000800848036803B910BD074B002BFBD0A0
:10045000BDE81040184700BF00000000F89AFF1FD9
:10046000F00A0100F49AFF1F0000000038B50446AE
:10047000104621700A491D460DF0B8F901464FF0AB
:100480007E500DF067FA07490DF0B0F9E560606045
:10049000256165610AF088FBE061204638BD00BF38
:1004A000DB0FC9400024744938B50446104621705A
:1004B00009491D460DF09AF901464FF07E500DF0A6
:1004C00049FA06490DF092F9E560606025616561C1
:1004D0000AF06AFBE06138BDDB0FC94000247449B3
:1004E00038B503780446032B20D8DFE803F01A1848
:1004F0001002C16840690DF06FF80D49054660684B
:100500000DF028FA014628460DF024FA38BD0849B6
:1005100040680DF01FFAE1680DF068F938BDC06859
:1005200038BDC16840690DF057F838BD002038BDAE
:100530000024744970B504460E460AF035FB0546A2
:10054000E069281A0DF0FEF8E3682361E561666151
:10055000A061014660680DF0FDF90146A0601048F9
:100560000DF0F8F90CF0CEFC0CF06EF90CF0E0FF99
:10057000054601464FF07E500DF02EF861690DF0F2
:1005800035F92169064628460DF030F90146304616
:100590000DF024F8E0602046BDE87040FFF7A0BFF2
:1005A000000080BF08B50E2009F0CEFD114B1B885E
:1005B000012B19D0104B1B88984213DB40F6FF71BA
:1005C0008842D4BFC3EB0001C3EB0101C1EB013191
:1005D000C3F57F630F33282091FBF3F1BDE808409A
:1005E0000AF038B90021F3E70146BDE808401420BD
:1005F0000AF030B9CA9CFF1F5A9CFF1F10B5044671
:1006000009F0A4FB204610BD70B44C88A04220D94C
:1006100001230133DBB21CB2660031F8144084427E
:100620001D46F6D3A04211D005F10045013D965B71
:1006300031F8151032F81530401AF21A00FB02F0AA
:10064000641A90FBF4F4E01870BC7047905B70BCC7
:10065000704702260125E5E700280CDA064A4342E6
:1006600082FB0320DA17C2EB600000EB4000A3EB33
:100670008000C0F10C007047ABAAAA2A2DE9F04710
:100680000C2009F02DFD0C200AF0E2F99C49142001
:100690000AF0EEF99B499C4807F026FA0221032054
:1006A0000AF07CFA022104200AF078FA02210520DF
:1006B0000AF074FA022106200AF070FA01210A20D9
:1006C0000AF06CFA012109200AF068FA01210D20D4
:1006D0000AF064FA012128200AF060FA01211420AE
:1006E0000AF05CFA02210B200AF058FA01210C20D2
:1006F0000AF054FA0C2000210AF03CFA04200AF017
:100700003FFA70B305200AF03BFA044680B3002498
:1007100020467E4D287004F07FFD2B78EBB92046F3
:1007200006F0A6F97A4B7B491B887B4C09887B4AEB
:100730002170A3F5AF7140F23A7303FB01F382FB22
:100740000312DB17764D7748A3EB621332335A213D
:100750002B6007F073FD90B9FEE7BDE8F04707F0A6
:10076000D3B806200AF00CFA0028CBD10124D0E738
:1007700003200AF005FAB0FA80F04009C9E76A4A96
:100780006A481268DFF8F8A100230121FFF78CFE08
:100790000B200AF0F5F9011E0CBF012300238AF893
:1007A000003002D111200AF0F9F9DFF89081604E93
:1007B000604F614D0023C8F8003033603B604FF05C
:1007C000040914E009F0C0FC33681844306009F0F3
:1007D000010080F0010003F0F5FB2B88002B14BF13
:1007E0004B20DC200AF002FAB9F1010919D00F20E0
:1007F0000AF0EEFB3B6803440E203B6009F0A4FCCA
:10080000D8F800309AF800200344C8F800301520CA
:10081000002AD7D111200AF0DBFB3368184430607E
:10082000D5E73B68D8F8002044493068DFF854E148
:100830002D88002BB8BF0333002AB8BF03329210B3
:100840000A603F493F4A0988128800284FEAA303FB
:10085000B8BF03303B6080103B4F30605E1A1944D4
:100860003E60CEF80010394F394E3A49C2EB000EC7
:100870000244C7F800E032600B605DB94FF4FA70D3
:1008800003F0B0FB03F09AFB04F0D0FF4FF4AF602D
:100890000AF0ACF9304B012504201D600AF070F914
:1008A00010B92E4B20701D702D4B1B881C2B1CD09B
:1008B0002C4C04F1C805232009F046FC44F8040F31
:1008C00001200AF093F9A542F5D1274A274B107869
:1008D000187005F0D7FF03F06DFB45F6BF522449B1
:1008E0002448BDE8F04709F0E7B9234B18880028F1
:1008F000DED0224BC0B2197805F00CFFD8E700BF5C
:10090000001B3746801A0600FC8FFF1F229DFF1F29
:10091000CC9CFF1F149CFF1F459DFF1FB5814E1BE4
:10092000A089FF1FA09CFF1FA889FF1F609CFF1FBD
:100930002C9CFF1F1C9CFF1F769DFF1FC49CFF1F4C
:100940009C89FF1FA489FF1FE09CFF1F949CFF1F31
:100950000C9DFF1FAC9CFF1F009CFF1F869CFF1F70
:100960005C9CFF1F0C9BFF1FA69CFF1FF49CFF1F9E
:10097000A5050000989CFF1F0A9CFF1F389CFF1FC5
:100980006C9DFF1F409DFF1FF0B40E8886420DD264
:1009900003F10043013B31F81350854202D9F0BC0A
:1009A000FFF732BE32F81300F0BC70471088F0BC7D
:1009B000704700BF094B1B880C2B09D8084A80B22E
:1009C00052F8232028B143F6FE73984203D9108CC5
:1009D0007047108870470349FFF716BECE9CFF1F73
:1009E0001CEF00007CED0000374A38491088384A77
:1009F000F8B5384B12881B68834248DB9342A8BF86
:100A0000134698420B60C8BF002342DD101AB0F5B0
:100A1000804FAABF9B03C3EB8333013093FBF0F0FD
:100A2000FFF7C8FF2C4B2D4F1C883B68C0F3C61541
:100A300005FB04F47F2CA8BF7F249D42064608D006
:100A4000274B1B88002B38D1264B1B88002B30D11D
:100A50003D60254D2B689E4205D0214B1B885A1FB7
:100A6000032A1DD92E60214D2B689C420ED0204BAD
:100A7000188848B11A4B1F4A1B88D35C834203D0A5
:100A8000C0B2E1B205F046FE2C60F8BDF8BD0346E9
:100A900008609A42D4BFC0EB0203C0EB0303B5E782
:100AA000144AD05C2030C0B206F07F0105F032FE5F
:100AB000D8E7284605F0A2FECAE70E4A2946D05CD0
:100AC00005F028FEC0E700BF5A9CFF1F509CFF1F87
:100AD000849DFF1FF09BFF1FFA9BFF1FE09BFF1FE2
:100AE000EC9BFF1FE49CFF1F049DFF1FD89BFF1F73
:100AF000F29CFF1F2089FF1F2DE9F04F172089B0BE
:100B00000AF066FAAF4B186016200AF061FAAE4B95
:100B1000AE4A1B8810600C2B00F03B81AC4BAD4AF9
:100B200019880093AC4B52F8214000221A70AB4B4D
:100B3000AB4D1B88AB4A2E88013B32F91370002E57
:100B40005CD0A94BA94A1B88A9491278013B31F90D
:100B50001380002A40F0DF8011200AF039FAA54BFB
:100B60000193D3F800A00646B24540F3DF80A24BC4
:100B7000DFF8A4921B88A14A012BD9F80030B2F803
:100B800000B09F4A02922046C8EB030800F09A8208
:100B90000CF0D8FD029A52F82B100CF027FE0146FB
:100BA00000200CF019FD0CF0E7FFCAEB0802B0457D
:100BB000B8BFB0469042CAEB080880F2968200FBAC
:100BC0000888013298FBF2F08E4BDFF850820293D6
:100BD000D8F80030034403EBD3735B10C8F800303F
:100BE0002B88012B12D1884BDFF834B20393874B4B
:100BF000DBF8005004934FF0000A47E07D4B01936F
:100C0000DFF814927F4BDFF8148202937E4B03933C
:100C10001D460F200AF0DCF92B689842824641DA23
:100C2000754A1288012A00F01D82744A05931288C1
:100C3000734D049220460CF085FD049ADFF8E0B174
:100C400055F82210DBF800500CF0D0FD01460020D2
:100C50000CF0C2FC0CF090FFEF1B059B5745A7EB77
:100C60000302B8BF5746FF1A9042BABF013200FBD9
:100C70000777474397FBF2F7D8F80020634B0493BC
:100C8000BB1803EBD3735B10C8F80030604B1B88B4
:100C9000013B032B00F2B082DFE813F06301A901EE
:100CA000C4008601594B04931B68984240F3C281EB
:100CB000514A1288012A00F0A682504A07931188EF
:100CC0004F4A0691204605920CF03CFD059A069984
:100CD000DFF84CB152F82110DBF800500CF086FD23
:100CE0000CF04AFF079B2F445745A7EB0302A8BF10
:100CF0005746FF1AD8F800309042BABF00FB07777A
:100D00000132474397FBF2F73B4403EBD3735B108D
:100D1000C8F80030BAE7152009F016FA354B0193F0
:100D2000D3F800A00646B2453FF721AF354B0293FA
:100D3000D3F800A0B24580F289812F4BDFF8D8901C
:100D40001B882E4A012BD9F80030B2F800B02C4A8B
:100D500003922046984400F070820CF0F3FC039A52
:100D600052F82B100CF042FD0CF006FFB045CAEB18
:100D70000802A8BFB046CAEB08089042B6BF00FB05
:100D8000088800FB08F8013298FBF2F0DFF88C804D
:100D90001EE7204B1B78002B3FF4C0AE0C4B0D4AD6
:100DA000198800930C4B52F8210001221A700CF0A4
:100DB000C9FC4FF07C510CF019FD0CF0DDFE04462F
:100DC000B5E600BFE49BFF1F5C9CFF1FB09CFF1FAC
:100DD000F89CFF1F3889FF1F269CFF1F7489FF1F87
:100DE000EA9BFF1F04F000007689FF1F6C9DFF1F28
:100DF0001CF00000949CFF1F809DFF1FA29CFF1F02
:100E000050EF00000C9DFF1FE09CFF1F409DFF1F47
:100E1000AC89FF1F749DFF1F2C9CFF1F049CFF1FAC
:100E20001C9CFF1F28460CF08DFCB2490CF0DEFC28
:100E3000054650460CF086FCAF490CF0D7FC014645
:100E400028460CF0CBFB0CF097FE0546CBF8005083
:100E5000D9F800000CF076FCA6490CF0C7FC074658
:100E600030460CF06FFCA4490CF0C0FC014638463B
:100E70000CF0B4FB0CF080FEC9F800009F4AA04BB8
:100E8000168819889F4AA04B12681B889F4FC6EB93
:100E9000050E3544039EC6F800E0461A084404993E
:100EA0000D6001990E6002993E8808609A4280F2B6
:100EB00089810025C3EB060E954974450F6880F2C1
:100EC0007681611C9F4205FB01F50EF1010E95FB39
:100ED000FEF5C0F2BE81BE42A8BF3E46F61A01FB37
:100EE00006F494FBFEF49A4200F33681BB42C0F252
:100EF0003381884C20680CF025FC87490CF076FC87
:100F000086490CF06BFB0CF037FEA0F5FF531C3B41
:100F1000082B98BF4FF40050D8F800301844002830
:100F20002060C0F24281B0F5804F80F252817C4B4C
:100F30001B781BB1B0F5005F40F05381794D2B78E1
:100F4000002B40F05481784D20682B68714C9842FA
:100F500004D080B205F0BCFC23682B6009B0BDE86A
:100F6000F08F28460CF0EEFB70490CF03FFC054674
:100F700050460CF0E7FB6E490CF038FC0146284661
:100F80000CF02CFB0CF0F8FD0546CBF80050D9F81E
:100F900000000CF0D7FB65490CF028FC07463046F2
:100FA0000CF0D0FB62495FE728460CF0CBFB5A49B6
:100FB0000CF01CFC054650460CF0C4FB5D490CF0DF
:100FC00015FC014628460CF009FB0CF0D5FD054642
:100FD000CBF80050D9F800000CF0B4FB4E490CF0EF
:100FE00005FC074630460CF0ADFB52493CE728466D
:100FF0000CF0A8FB50490CF0F9FB054650460CF0EC
:10100000A1FB4E490CF0F2FB014628460CF0E6FA33
:101010000CF0B2FD0546CBF80050D9F800000CF0FA
:1010200091FB45490CF0E2FB074630460CF08AFB89
:10103000424919E7D8F80030DFF810B103EBD37359
:101040005B10DBF80050C8F800301FE6DFF80081C5
:10105000DFF80091D8F8003003EBD3735B10C8F8C9
:101060000030BDE5364A06931188364A0591204680
:101070000492DFF8D8B00CF065FB049A0599DBF810
:10108000005052F821100CF0B1FB0CF075FDEF1B75
:10109000069B5745A7EB0302B8BF5746FF1AD8F87F
:1010A00000309042BABF013200FB0777474397FBFD
:1010B000F2F73B4403EBD373234A04925B10C8F866
:1010C0000030E3E50CF03EFB029A52F82B100CF0D6
:1010D0008DFB0CF051FDCAEB0802B045B8BFB0461D
:1010E0008242CAEB08083FF76AAD00FB08F898FB9C
:1010F000F2F069E5CDCC4C3FCDCC4C3E9C89FF1F36
:10110000A489FF1FE49BFF1F6A9DFF1FC89CFF1F50
:10111000B09CFF1F7089FF1F9A99193FCDCC4C4599
:101120002F9EFF1F099CFF1F2C89FF1F3333733F26
:10113000CDCC4C3DCDCCCC3E6666663FCDCCCC3DD7
:10114000A29CFF1F50EF0000409DFF1F1C9CFF1F33
:10115000049CFF1F2C9CFF1F009B1B88002B3FF44F
:10116000C8AE2B1B002BB8BF5B42092B47DD05F532
:1011700000500130001B0CF0E5FA3B493B4C0CF0F1
:1011800035FB054620680CF0DDFA39490CF02EFBE2
:10119000014628460CF022FA0CF0EEFCD8F800309C
:1011A000184400282060BFF6BEAE002213E09F4224
:1011B00005FB04F5B8BF002195FBFEF54BDA91FB6A
:1011C000FEF490E6B242D4BFC3EB0205C3EB0605C2
:1011D00070E643F6FF72274B22601B78002B3FF42A
:1011E000ADAE02F0EBFE244B01221A70ABE602F02A
:1011F000E1FE00232B70A6E6D9F800003EE64FF48E
:1012000000501A4C88E61D491D4A069320460D8859
:1012100005920CF097FA059ADFF868B052F825109D
:10122000DBF800500CF0E2FA014600200CF0D4F993
:101230000CF0A2FC2F44069B56E50CF083FA039AAF
:1012400052F82B100CF0D2FA014600200CF0C4F931
:101250008AE51E4642E6B742D4BFC3EB0701C3EBA3
:10126000060104FB01F1AAE7CDCCCC3E7089FF1F3B
:101270009A99193F2F9EFF1F099CFF1FA29CFF1FD9
:1012800050EF00001C9CFF1F08B5244B1B88FBB1CE
:10129000234B1B78FBB1234B1B78E3B1224B1B780C
:1012A000CBB1224B1B78B3B1214B22481A78C2B97B
:1012B000214A22490088128809680244B1EB620F72
:1012C00009DD01221A706420BDE8084002F08ABEE0
:1012D000174A117801B908BD1370BDE8084005F040
:1012E000C1BA154A16490088128809680244B1EB50
:1012F000620FF0DD00221A7005F0B4FA642002F0EB
:1013000071FE642002F06EFE642002F06BFE4FF46A
:101310001670BDE8084009F069BC00BFB49CFF1F0F
:10132000549CFF1F179CFF1F189CFF1F199CFF1F39
:10133000F99BFF1FC89CFF1F6A9DFF1FE49BFF1FB7
:10134000B09CFF1F38B5114C2320257808F0FCFE17
:101350000F4A42F82500131F02F1C400002253F87F
:10136000041F83420A44FAD123780A4907480A4CE9
:101370000133DBB2322B81FB025108BF0023D217AD
:10138000C2EB21120370226038BD00BFF09CFF1F2A
:10139000109BFF1F1F85EB51FC9CFF1F2DE9F04F99
:1013A000B84CB94D2068B94F83B00CF0CBF9B849AF
:1013B0000CF01CFA0646102009F00AFE0CF0C2F9E7
:1013C000B4490CF013FA31460CF008F90CF0D4FBD8
:1013D0002988206088423B8843DA9E465B1A7F2B2F
:1013E0004FF0000247DDD2015E1C92FBF6F2AA4EDE
:1013F000DFF8C882B6F800C0C8F80020BCF1190FA9
:1014000000F0DF80BCF11A0F00F01781BCF11E0F55
:1014100000F020810126B146A04A1288002A00F07F
:101420009D808842C0F207817045D4BFC1EB0000A7
:10143000C1EB0E009A42BABF02FB000001335043D9
:1014400090FBF3F3964A1360964B1888C0B9964AFE
:101450001288AAB9954B197801B11A7003B0BDE88A
:10146000F08F9842D4BFC1EB0002C1EB03029E464D
:101470005B1A7F2BB7DCC2EBC21292FBF3F2B6E72A
:101480002988D4F800E0DFF80082DFF8F8A1714580
:101490006CDCDFF818C29CF80020002A2ED14FF037
:1014A000010B04288CF800B028D1002E40F0948164
:1014B0007D4B18880028D1D0B9F1000FCED0236819
:1014C0002C883A88A34280F265810023141B7E2C6D
:1014D000774DD5BFC3EB8313C3EBC3135B0001345C
:1014E00093FBF4F42B680134A34203D0C0B2E1B201
:1014F00005F010F92C6003B0BDE8F08F012800F072
:10150000F680022800F0EB800328D1D1694B1B88BC
:10151000092BCDD0002ECBD023682E883A88B34239
:1015200080F27B810023961B7E2EDFF88CA1D5BF35
:10153000C3EB8313C3EBC3135B00013693FBF6F6D7
:10154000DAF800300136B34203D0F1B24A2005F098
:10155000E1F8CAF80060ABE716469146BCF11E0FF1
:101560007FF472AF0022DFF858817EE04F4B1A788B
:10157000002A3FF473AF002401281C7000F0A480FF
:10158000022840F00E81002E00F0A3804A4D2B6807
:10159000002B00F09E800420214605F0BBF8424B52
:1015A0002C60188800283FF459AFB9F1000F3FF4C0
:1015B00055AFC0B2002105F0ADF83D4B00221A60D6
:1015C0004CE7DFF8FC8098F80020C2B1DFF8D89033
:1015D000B9F800A0BAF1000F11D0DFF8E89099F83F
:1015E00000B0934578D05FFA8AF07F2105F092F839
:1015F00098F80030B6F800C089F8003010E0DFF845
:10160000C49099F800A0924566D0274B0021187825
:1016100005F080F898F80030B6F800C089F800307E
:101620001E4B1A88002A97D0BCF11E0F40F006818D
:101630000026B14619E00020FCE6DFF8848098F827
:101640000020002A0BBF012600264FF000094FF0B2
:101650000109E1E6DFF86880104B98F800601A880D
:10166000B6FA86F676094FF0000998F80030002B9C
:101670003FF4E8AE2988B7F800E02068C1EB0E031C
:10168000CFE600BF489DFF1F2A9DFF1F929CFF1FB2
:101690009A99193FCDCCCC3E5C9CFF1F6E9DFF1FDD
:1016A0000C9CFF1F249DFF1FDC9BFF1F169CFF1F30
:1016B0004C9CFF1FEC9BFF1F289CFF1F109CFF1FD3
:1016C000749DFF1F829CFF1F1EB1614D2B68002B74
:1016D0007BD1604B188865E70026B1469CE6002E5A
:1016E0003FF4E6AEDFF868A1DAF800202EE0002E25
:1016F0003FF4DEAEB7F80080F045D4BFC1EB08027E
:10170000C1EB0E02C1EB0808B8F17E0FDFF840A173
:10171000D5BFC2EB8212C2EBC212520008F101081F
:1017200092FBF8F8DAF8002008F10108424506D0EB
:101730005FFA88F10120009304F0ECFF009B188809
:10174000CAF8008002287FF4DFAE42462168B5F86F
:1017500000803888414559DA0021C8EB0008B8F10B
:101760007E0FD3BFC1EB8111C1EBC11108F101089C
:10177000490091FBF8F808F10108904506D05FFA9E
:1017800088F10420009304F0C5FF009B1888CAF874
:101790000080B9E69342D4BFC4EB0303C4EB020359
:1017A00094E6032827D12C4B1B88092B91D0002EBF
:1017B0008FD0274D2B68002B8BD04A20214604F078
:1017C000A9FF244B2C601888ECE6214604F0A2FF08
:1017D000204B2C601888E5E640207F218DE80C0026
:1017E00004F098FF019B009A188858451CD00228E5
:1017F0007FF48AAE76E704287FF46BAF002E3FF4C7
:1018000068AF2146402004F085FF62E78142D4BFE3
:10181000C8EB0101C8EB00019FE79342D4BFC6EBC0
:101820000303C6EB02037EE6B8F80010DAF800E026
:10183000B7F800808E45FFF665AF5DE72988B7F8F9
:1018400000E020680026C1EB0E03B146E9E500BFC9
:10185000289CFF1FDC9BFF1FEC9BFF1F08B50F4B55
:101860001B88022B0FD0032B12D0042B03D00C4B60
:1018700001221A7008BD7F21092004F04BFF084B9C
:1018800001221A7008BD7F21412004F043FFEEE7DA
:101890004021092004F03EFFE9E700BF909CFF1FB4
:1018A000309DFF1F38B51C4B1B881D2B26D01B4BB2
:1018B0001B88012B25D01A4A1A4B14881B681A4A18
:1018C000A342128818DB9342D4BFC4EB0303C4EBDA
:1018D0000203141B7F2CC6BFDB010134C3EBC3130F
:1018E00093FBF4F4114D2B689C4203D0E1B2052028
:1018F00004F010FF2C6038BD0023EAE70C4B1C8875
:10190000F0E70C4B0C4A0D491B6812680C689B1AD7
:101910001C1B84F30704E5E75C9CFF1FEA9BFF1F89
:10192000109DFF1F3C9DFF1F569CFF1F009DFF1F2A
:10193000389CFF1FAC9CFF1F3089FF1F349DFF1F89
:1019400010B50F4C23685BB90E4B1B88022B11D0CE
:10195000033B012B09D90C4A00231370236010BDEF
:101960000021052004F0D6FEEEE70021092004F056
:10197000D1FEF0E70021412004F0CCFEEBE700BFF0
:10198000009DFF1F909CFF1F309DFF1F08B5274B38
:101990001B78ABB1152008F0D7FB254A254B1288E0
:1019A00018601D2A15D0244A1288EAB1012A25D0D0
:1019B000224B1B78002B34D0BDE80840FFF7C0BF96
:1019C000112009F005FB1A4A1A4B128818601D2ACB
:1019D000E9D11B4B1B78002BEAD0184B1B780BB3BB
:1019E000BDE80840FFF75EBF164A1288002ADFD024
:1019F000154A1B6812889A42DADCEEE70F2009F0DC
:101A0000E7FA104B114A1B88106033B1104B114A92
:101A10001B6812689B1A9842DFDD084B1B78002B6D
:101A2000CAD108BDFFF71AFFDAE700BF6C9DFF1FA0
:101A30005C9CFF1F3C9DFF1FEA9BFF1F309DFF1F0B
:101A4000749DFF1F909CFF1F109DFF1F349DFF1F63
:101A5000AC9CFF1F3089FF1F2DE9F04F8BB007AD05
:101A6000B54F2C460AAE611BC9B2B44806F0AAFBBA
:101A70003B88834294BF0020012004F8010BA6425A
:101A8000F1D1AF48AF4A9DF81C50AF4905709DF8A1
:101A90001E00AE4E10709DF820209DF82430AC4FF3
:101AA000AC4C0A709DF82210317000263B702670F5
:101AB00063B9002940F00581002A40F0C581A64A9B
:101AC000002800F0C9810223237005E0002A40F0BD
:101AD000A9800523A04A2370DFF8D4B2DFF8D4929E
:101AE0009DF81DE09DF81F00DFF8CC82DFF8CCA246
:101AF0009A4D9B4F9B4E9DF8211013708BF800E080
:101B00009DF826209DF823309DF825E089F80000F7
:101B10009DF827C088F8001001208AF800202B705B
:101B200087F800E086F800C009F052FA8E4A8F4B21
:101B300011688842CCBF012200221A7076DD8C4BDE
:101B40001B88182B72D88B4AB2F800E00C3B00932C
:101B5000BEF1000F72D1884A9BF800C092F800B025
:101B600098F8008099F800209AF8009094F800A066
:101B70002C78ABEB4C0BC2EB0B0BA8EB880EDE44C6
:101B8000C9EB897BC9EB8B09DFF8F4B1F14497F815
:101B900000E0BBF800B009EB44093478CE4404FB04
:101BA0000BEE4FF00C09754C19FB0AEEC4F800E07F
:101BB000B8F1000F0BD036784EB1714E3688042E36
:101BC0000CBF0EF1020E0EF1040EC4F800E06D4CD5
:101BD000DFF8EC912488B9F800A06B4EDFF8E491AF
:101BE0003688D9F80090009B033C04EB4404CAEB10
:101BF000CA0A0EEB84043444D144644E0C3C56F8BB
:101C000029601C44A319BCF1000F28D02C7834B3F0
:101C1000002A5AD1B8FA88F85D4C4FEA581884F86F
:101C2000008023E0062323704B4A55E7514AB2F85F
:101C300000E000230093BEF1000F8CD0BEF1010F35
:101C400047D0BEF1020F00F0C1804C4C9BF800C0A1
:101C500099F8002098F80080D4F800E0A8E74C4CF0
:101C6000002525700AB13A781ABB0022494C8842F7
:101C700022704949C4BF494AC2F800E00A68934249
:101C800013D0474A474C10680590059820601268A9
:101C90000692454C069A24880B60121AA24284BF11
:101CA000424A13600BB0BDE8F08F3E483C4A0068E2
:101CB000EDE7BCF1000FD8D1B8F1000FD5D101226A
:101CC000D4E704232370244A06E7314A0024147021
:101CD000CBE7294A9BF800C092F800E098F8008012
:101CE00099F8002094F800B09AF800902C780194AC
:101CF000AEEB4C0EC2EB0E0EA8EB88047444C9EB9D
:101D0000C909D944A31EDFF878A0DFF8BCE0019C24
:101D100097F800B05EF829E0BAF800A096F80090B5
:101D200003EB44045C4409FB0A4909F11809134C0C
:101D3000CE44C4F800E03BE7CC9CFF1FA09CFF1FF3
:101D4000179CFF1F189CFF1F199CFF1F1A9CFF1F49
:101D50001B9CFF1F2C9DFF1FBE9CFF1FF89BFF1F9E
:101D6000589CFF1F7C9DFF1FA089FF1F749DFF1FB4
:101D70005C9CFF1FF69CFF1F6C89FF1F649DFF1F6B
:101D8000C09CFF1F849CFF1F3A9DFF1F78EF00003F
:101D9000A49CFF1FA59CFF1FF49BFF1F789DFF1FA6
:101DA0006C9EFF1F209CFF1F829DFF1F309CFF1F0A
:101DB000709DFF1F719DFF1F739DFF1F549CFF1F90
:101DC000BC9CFF1F0C9CFF1F20ED0000274A9BF8C6
:101DD00000C092F800B0247899F8002098F80080AC
:101DE0000394ABEB4C049AF80090214B95F800A0BB
:101DF000CDF804A0A8EB880BA41A5C444FF0050BA7
:101E00001BFB094B039C97F800A0CDF808A0C9EB79
:101E1000C909B3F800A009EB0403BDF80490029CC3
:101E20000BF1050B1EFB09BE96F800B0DFF84C90D5
:101E3000A6440BFB0AEE59F823900E4C0EF10C0E43
:101E4000CE44C4F800E0B3E60B4A1378002B3FF40D
:101E500037AE032323703FE615B1012323703BE621
:101E60001378012B8CBF23702B4635E66C89FF1F3E
:101E7000C09CFF1F649DFF1FBE9CFF1F54EE00000F
:101E80002DE9F04F3B4B1B788BB0002B6DD10E2012
:101E900008F05AF90BF056FC01463748374C384DDC
:101EA000FEF748FB3448FEF71BFB0BF065FE80F3A2
:101EB0000C002060FFF7D0FD2E68012E7CD0022E92
:101EC00000F0AA82032E00F0B9832E4C23682E4A1C
:101ED0002E4E0993099B177830682D4C072101225B
:101EE000181A11FB07229042236000F29082294EBB
:101EF00032689A1A0D2A00F28382274E32689A1AA3
:101F0000132A00F27882254E32689A1A252A1AD9A5
:101F1000234B1B88002B40F06781224B1B78002B42
:101F200040F06281FFF70EFA1F4B1B881B3B9BB2F0
:101F3000022B04D81D4B1B78002B40F0588102F077
:101F400063F8236833601A4D2A689B1A502B00F2FD
:101F50001182184B1B88012B00F0298204F06EFCC3
:101F600004F09CFA0BB0BDE8F08F05F055FB0BB008
:101F7000BDE8F08F229DFF1F609CFF1FF09BFF1F9D
:101F8000009CFF1F6C9EFF1F449DFF1F189DFF1F9D
:101F90003C9CFF1FEC9CFF1FB89CFF1F5C9DFF1F1C
:101FA000B49CFF1FF99BFF1F5C9CFF1F749DFF1FCC
:101FB0008C9CFF1FCA9CFF1FDFF82883A34AB8F838
:101FC00000001378834204D0C3B21846137004F0A3
:101FD00071FBDFF80C939E4AB9F8003011789942F2
:101FE00004D09C4F3978002940F07E879A4A2368B4
:101FF00012889A4C9A42C0F2FF80994A1278002ABD
:1020000040F0FA80DFF8E0A2BAF8003023B9954B2F
:102010001B88002B00F01F85934A944B11881B8866
:10202000934A0B4412685B109342924A126880F202
:10203000C28400219342B4BF01230B460491009354
:10204000ACBF4FF0010B8B4605910E2008F07CF8D9
:10205000894B8A4A1B68176803930133A7F25232EF
:10206000002B8446029240F35087802BA8BF802328
:10207000834A844912780191002A00F0C7800978C8
:10208000914200F0C380B9F80010DFF854E29942A1
:1020900001F047816F49AEF800307B4B4FF0010EE5
:1020A00081F800E01978DFF844E2019B8EF8001017
:1020B0001A70009B002B00F01B81BAF80030002B37
:1020C00000F01681714B1B685A1C002A40F32187CF
:1020D000802A00F31D876E4E6E496F483688098846
:1020E00000683144B0EB610FC1F2EF81A3F1480207
:1020F0000F2A02D8473BA8F800300E2008F024F839
:102100006FF454731F44874202DC644B00221A7040
:10211000002008F05DFF624A624B1168624E1B8826
:102120008842D4BF002201223270002B00F03A8492
:102130005E4B1E78964240D088423EDD5C490E7868
:10214000002E00F0CB875B4991F800C0BCF1000F76
:1021500040F0C287584F0097584F59480297564F42
:10216000007887F800C0554F4FF0010E87F800C087
:1021700081F800E0002841F0668152490978002981
:1021800001F02780504903910E460978002941F05B
:102190001D804E48494F00783970012102973170F7
:1021A00058B1454843490090002008700099029FAB
:1021B0000870039901263E7008701A70444B1B8802
:1021C000A3F11B02012A40F26A861D2B7FF47EAE2A
:1021D0003E4F3B78002B41F0E9803E4E3378002B98
:1021E00040F06984337071E6FFF74EF89AE62B6889
:1021F000012B7FF4A4AEA4E62168374A0691069825
:102200003649106002220B602A60FBE61E49DFF8A7
:10221000DCE0097800293FF448AF9EF800008142D5
:102220003FF443AF03984B2841F327801833802BAA
:10223000B9F80000A8BF802398423FF436AF284881
:1022400003800448012303702FE700BFF49CFF1FA5
:10225000459DFF1F869CFF1F5A9CFF1F6C9EFF1F02
:10226000F99BFF1F809CFF1FC89CFF1F6A9DFF1FDB
:10227000E49BFF1FB09CFF1F789DFF1FC49CFF1FA6
:10228000A49CFF1F729DFF1FA59CFF1F649DFF1F45
:102290002A9DFF1F929CFF1F489DFF1F609DFF1FEF
:1022A000A089FF1F209DFF1F359CFF1F489CFF1F1B
:1022B000549CFF1F349CFF1FA89CFF1F089CFF1FFE
:1022C000F89BFF1F709DFF1F369CFF1F749DFF1F13
:1022D0005C9CFF1F829CFF1FFC9BFF1F509DFF1FEC
:1022E000149CFF1FA69CFF1F269DFF1F4C9DFF1FD8
:1022F000029B9C45BFF601AFAC4B1B88002B3FF403
:10230000FCAEBBF1000F7FF4DDAEA94B1B881BB107
:10231000059B002B7FF4D6AE049B002B3FF4EDAE63
:10232000A44B1A78002A7FF4E8AEDFF8048398F80B
:10233000006001221A70002E40F05A839E4B1B78D9
:10234000002B01F004819D4B1B78002B01F01581BF
:102350009B4B1B78002B7FF4D0AE9A4B1B78002B45
:102360003FF4CBAEB9F8003097490A3BA9F80030EA
:102370000A70C2E602F098FF944B1B7873B9944B35
:102380001B785BB9934B1B7843B9934B1B782BB9E4
:10239000924B1B7813B901F00DFE01E001F016FE1F
:1023A00023682B608E4B1B88012B7FF4D7AD8D4AA1
:1023B0008D4B11688D481A78A1F118032A2101FB71
:1023C00003F10160002A00F0D782894A136899421C
:1023D00000F3458380F24F8386480068D0F17F0088
:1023E00048BF0330801001301B1A994200F3438329
:1023F00013601946C2E2FFF7C9FA2368336082E529
:10240000FEF77AFBFEF7CAFF2368336075E5FEF737
:10241000EBFA236833606AE5774A26681288B2428D
:1024200004DB6E4B1B78002B00F04083734C744828
:1024300023680793734B079900681B88091A994210
:1024400063D8002B61D0704B198800293FF43EAD52
:102450006E4B6F481B680088B342B8BF33469A4240
:1024600041F32C806B4B1A60DFF8C88188F80010AC
:102470005C4FFEF7B9FA38687F2840F32986664B2F
:102480007F3883FB0032C317C3EB620303EB4303C4
:10249000A0EB83007330614B01931B883860002BE5
:1024A00040F031874B4B00931B78002B00F05A848F
:1024B0005B4E3378002B00F05584DFF87C91DFF819
:1024C00058A14FF0000B0CE003F17300C0B298F874
:1024D000001004F047F933780BF1010B5B4540F332
:1024E00041843B6859F8040F1844A0F17F038AFB2C
:1024F0000321DA17C2EB610202EB42027F28A3EB51
:102500008203E1DCFEF7A8F8E0E7404B40491B6896
:1025100008883D49B342B8BF33469A4200F3AD82C2
:102520003C4E09888342A8BF0346336000299BD1F3
:102530009A42C8BF0B4640F3A782801AB0F5804F7D
:10254000AABF9B03C3EB8333013093FBF0F0FEF78C
:1025500031FAC0F3C6100BF0F5F8324B0646188876
:102560000BF0F0F83049074630460BF03FF90146D2
:1025700038460BF03BF931460BF030F84FF07E5106
:1025800006460BF0D1FA002840F08D8727493046E7
:102590000BF0E8FA002840F04A8730460BF012FBB7
:1025A000C0B2DFF8908088F8000061E7809CFF1FD0
:1025B000289DFF1F609DFF1F709DFF1F719DFF1FC6
:1025C000739DFF1F549CFF1F869CFF1F089CFF1FCD
:1025D000349CFF1FA89CFF1F369CFF1FF99BFF1F09
:1025E000CA9CFF1F309CFF1F309DFF1F149DFF1FC3
:1025F000449CFF1F009DFF1F5A9CFF1F6C9EFF1FE6
:10260000FC9BFF1FE89CFF1F7E9DFF1F509DFF1F2F
:10261000849DFF1F509CFF1FABAAAA2A889CFF1F06
:102620003489FF1FE89BFF1FCDCCCC3D0000FE424C
:102630002C9DFF1F409CFF1F7489FF1FB94B26680C
:102640001988B14253DDB84B1B78002B4FD1DFF80E
:10265000209399F800007F2840F3A486A3F1553316
:102660007F3803F1004383FB0032C317C3EB6203DF
:1026700003EB4303A0EB83007330AC4B01931B8847
:10268000C0B289F80000002B40F0ED86A84B009303
:102690001B78002B00F04D85A64E3378002B00F000
:1026A0004885A54FDFF898824FF0000A0AE003F151
:1026B0007300C0B204F07EF833780AF1010A534582
:1026C00040F3378557F8043F99F800001844A0F10B
:1026D0007F0388FB0321DA17C2EB610202EB42029F
:1026E0007F28A3EB8203E2DCFDF7B6FFE1E7934F1F
:1026F00038687F2840F3CF81914B7F3883FB0032CD
:10270000C317C3EB620303EB4303A0EB83007330F7
:10271000DFF85C9299F800A0824500F02682894B90
:102720001B88002B43D1884A884812680088914250
:1027300005DC8242D4BFC1EB0203C1EB0003411AA6
:10274000B1F5804FA6BF9B030131C3EB833393FBED
:10275000F1F0FEF72FF9C0F3C6100AF0F3FF7C4B3F
:10276000064618880AF0EEFF7A49804630460BF09C
:102770003DF8014640460BF039F831460AF02EFF8D
:102780004FF07E5106460BF0CFF9002840F06886E6
:10279000714930460BF0E6F9002840F037863046A4
:1027A0000BF010FAC0B2DFF8CC8188F80000BAF163
:1027B0007F0F40F388846248AAF17F0A80FB0A30C9
:1027C0004FEAEA73C3EB600000EB4000AAEB800025
:1027D0007330574B00931B78C0B289F80000002B70
:1027E00040F0E8835D4B03931B78002B40F0B585E8
:1027F0005B4B02931B78002B40F058864B4B0193A8
:10280000029B1B78002B3AD0564B1B88182B17D0F5
:1028100099F800201344A3F118007F2840F3F985AC
:10282000474A973B82FB0321DA17C2EB610202EBB6
:102830004202A3EB820303F17300C0B203F0BAFFBC
:10284000494A4A4B127833F81230182B17D099F8AE
:1028500000201344A3F118007F2840F3E485384A90
:10286000973B82FB0321DA17C2EB610202EB4202C3
:10287000A3EB820303F17300C0B203F09BFF009B44
:102880001B78002B00F0B584019B284E1988002985
:1028900000F05C8538687F2840F35783284B7F38E9
:1028A00083FB0032C317C3EB620303EB4303A0EBCC
:1028B000830073303860002940F0F084009B1B785F
:1028C000002B00F05D811B4E3378002B00F0588107
:1028D000DFF864A0DFF89C804FF0000B0CE003F100
:1028E0007300C0B298F8001003F03CFF33780BF18E
:1028F000010B5B4540F344813B685AF8040F104AD2
:102900001844A0F17F0382FB0321DA17C2EB6102B6
:1029100002EB42027F28A3EB8203E0DCFDF79CFE82
:10292000DFE700BF5A9CFF1FF99BFF1F889CFF1F1A
:10293000A89CFF1F3489FF1F7489FF1F309CFF1F55
:10294000ABAAAA2A7E9DFF1F509CFF1F849DFF1FDC
:10295000E89BFF1FCDCCCC3D0000FE42369CFF1F04
:10296000089CFF1F2E9DFF1F389DFF1F549DFF1FBA
:10297000E69CFF1F409CFF1FA84B1960A84B1B68DB
:10298000A92202FB03F3002BBCBF03F57F533F33A7
:102990009B13543B194481F30C01282007F05AFF84
:1029A000FFF7DCBA9F4EA048A049A14A33700370DC
:1029B0000B70137002E493424FF0000B6EDA0123A8
:1029C000CDF800B0CDF814B00493FFF73EBB994B9F
:1029D0001B78002B7FF491AB039B974A243B83F336
:1029E0004703D9B25B20136003F094FE98F80060AF
:1029F000032E30D1DFF8908298F80030002B40F0A1
:102A00003F868E4F3B78002B40F02D86894E3378E1
:102A1000002B40F01B868A4B1B78002B40F0098668
:102A2000884A1380884B1B78002B40F0F585874B34
:102A30007F221A8098F800306BB93B785BB9337805
:102A40004BB9834A7F210720138003F063FE7F2167
:102A50000B2003F05FFE7F4B1F68FFF74EBB7E48E5
:102A60000068D0F17F0048BF033003EBA0030133BF
:102A70009942BFF6BDAC116080E7784B09881A60B7
:102A800000297FF4F1AC13469842D4BFC2EB000397
:102A9000C2EB030351E5FDF7DFFD39E60123CDF875
:102AA00010B0CDF800B00593FFF7CFBA01232B602B
:102AB0006B4CFFF70BBA6B4B6A20198803F0AEFF23
:102AC0003B783370FFF702BA564B1B78002B3AD095
:102AD000654B1B88182B17D099F800201344A3F1DD
:102AE00018007F2840F3F684604A973B82FB03215D
:102AF000DA17C2EB610202EB4202A3EB820303F19D
:102B00007300C0B203F056FE594A5A4B127833F89C
:102B10001230182B17D099F800201344A3F1180095
:102B20007F2840F3DB84514A973B82FB0321DA176D
:102B3000C2EB610202EB4202A3EB820303F17300DA
:102B4000C0B203F037FE019B1B88002B00F0958478
:102B5000354B1B78002B40F08A84474B3F4A19883D
:102B600026680020012310602B60B1423C4CBFF668
:102B7000ADA92268414B0892089A1A60FFF7A6B9DE
:102B8000039B1B78002B00F083803B68A3F10C00B3
:102B90007F2840F3FA8335488B3B80FB0320DA170C
:102BA000C2EB600000EB4000A3EB800303F1730075
:102BB000DFF8D080C0B298F8001003F0D3FD009B7E
:102BC0001B78002B64D02E4E3378002B60D0DFF8BA
:102BD000BCA04FF0000B0BE003F17300C0B298F8FB
:102BE000001003F0BFFD33780BF1010B5B454FDDA7
:102BF0003B685AF8040F1D4A1844A0F18B0382FB6E
:102C00000321DA17C2EB61020C3802EB42027F2883
:102C1000A3EB8203E0DCFDF71FFDDFE7449CFF1F11
:102C20007089FF1F089CFF1F349CFF1FA89CFF1F7B
:102C3000369CFF1F549CFF1F089DFF1F739DFF1FA5
:102C4000719DFF1FE49CFF1FF89BFF1F7E9DFF1FD0
:102C5000EC9BFF1FC49CFF1F009DFF1F509CFF1F8C
:102C60006C9EFF1F389CFF1F2E9DFF1FABAAAA2A38
:102C7000389DFF1F549DFF1F5A9CFF1F0C9EFF1F76
:102C80003489FF1F409CFF1F709DFF1F7489FF1F29
:102C9000029B1B78002B3AD0AD4B1A88182A18D00B
:102CA0003B681344A3F118007F2840F3B683A94A78
:102CB000973B82FB0321DA17C2EB610202EB42026F
:102CC000A3EB820303F17300A34BC0B2197803F0A6
:102CD00049FDA2490B78022B00F253830133DBB28A
:102CE0000B701A469E4830F81260182E40F0908201
:102CF0000422032B03F10106F3B208BF002330F8CE
:102D00001360182E40F08382013AF2D10B70019BC0
:102D10001B88002B00F0CB82009B1B783BB9039BE8
:102D20001B7823B9029B1B78002B00F0E0838D4BAE
:102D30001B78002B00F0D6808B490B78082B00F213
:102D4000D1808A483A680068894E0133DBB25F1E41
:102D5000101A46F827000B70864B2668198889F8E8
:102D6000002002E77F4B1B78002B40F0C1823B68BC
:102D7000814A1278002A45D0A3F10C007F2840F345
:102D80000A83744A8B3B82FB0321DA17C2EB610290
:102D900002EB4202A3EB820303F17300C0B298F886
:102DA000001003F0DFFC009B1B7853B36E4E3378AA
:102DB0003BB3DFF8FC91DFF89CA14FF0000B0BE078
:102DC00003F17300C0B298F8001003F0CBFC337825
:102DD0000BF1010B5B4514DD3B6859F8040F1844F7
:102DE000A0F18B038AFB0321DA17C2EB61020C38D6
:102DF00002EB42027F28A3EB8203E1DCFDF72CFC0F
:102E0000E0E73B685D4A1278002A3DD0504A1288BC
:102E1000182A18D01344A3F118007F2840F30D831B
:102E20004C4A973B82FB0321DA17C2EB610202EBAB
:102E30004202A3EB820303F17300C0B298F80010C2
:102E400003F090FC3B6845490A78022A00F2A6820A
:102E50000132D2B20A701646414830F816E0BEF18F
:102E6000180F40F0F0810426032A02F1010E5FFAE8
:102E70008EF208BF002230F812E0BEF1180F40F0C9
:102E8000E181013EF0D10A70019A1288002A00F017
:102E900041823B4903220B702A60FFF717B8394F74
:102EA0003B78002B3FF499A9374E307801F0FCF8BD
:102EB000364B1B78002B00F0918233887E2B00F27A
:102EC0008D82334A0133108899B23180002800F096
:102ED0009582C9B2C0B22F4E03F01CFC3B78337010
:102EE000FEF7F4BF3A6837E7DBB21846137003F019
:102EF000EFFB294B1B491A461F4B184600230B704A
:102F00003B7013700370FFF771B80123FFF7B0B87F
:102F100080262249224B234A09881B8812680B44C9
:102F2000B2EB630FBFF6E9A8164B1B78002B40F0FD
:102F3000FE81B9F800301C4AB3423FF4DEA81B4BB7
:102F4000168001221A70FFF7D8B8FDF785FBB1E4AF
:102F50002E9DFF1FABAAAA2A409CFF1F389DFF1F72
:102F6000549DFF1F349CFF1F3489FF1F1C9DFF1FB2
:102F70007889FF1F5A9CFF1F369CFF1F089CFF1F6C
:102F8000E69CFF1F749DFF1F389CFF1F589CFF1F6E
:102F90000A9CFF1F829CFF1FA89CFF1F929CFF1F83
:102FA0002A9DFF1F489DFF1F149CFF1F869CFF1F2B
:102FB0007489FF1FC14B01931B88002B40F06C8369
:102FC000BF4B0393BF4B0293BF4E33786BB3DFF815
:102FD0001483DFF8F8A24FF0000B09E003F173004F
:102FE000C0B203F0E7FB33780BF1010B5B451CDD4E
:102FF00058F8043F99F800001844A0F17F038AFBB9
:103000000321DA17C2EB610202EB42027F28A3EB35
:103010008203E3DCFDF720FBE2E7AA4B029303F017
:10302000C9FB009B1B78002BCED1039B1B78002B88
:103030003FF4E6AB99F80030A3F10C007F2840F391
:10304000A781A2488B3B80FB0320DA17C2EB60000C
:1030500000EB4000A3EB800303F17300C0B203F068
:10306000A9FB009B1B78002B00F08081964E3378E3
:10307000002B00F06582DFF86C82DFF850A24FF081
:10308000000B0AE003F17300C0B203F093FB337846
:103090000BF1010B5B457FF7B3AB58F8043F99F890
:1030A00000001844A0F18B038AFB0321DA17C2EB5E
:1030B00061020C3802EB42027F28A3EB8203E1DCC1
:1030C000FDF7CAFAE0E75046FDF7C6FAFFF781BB05
:1030D000FDF7C2FAFFF7DFB9002008707C490878D5
:1030E00040B17C4900910978002900F0A981009F36
:1030F000002139707849097800297FF443A8002E0F
:1031000067D1002865D1754E724F96F800E06C4E7D
:1031100003966C4E02966A4E71493070694E009764
:10312000087038703070BEF1000F7FF43DA8FFF7D3
:1031300044B8634B1B78002B3FF4C6AC99F80030C1
:10314000A3F10C007F2840F3C281604A8B3B82FBD5
:103150000321DA17C2EB610202EB4202A3EB820306
:1031600003F17300C0B203F025FB009B1B78002B1A
:103170003FF4AAAC544E3378002B3FF4A5AC594F22
:10318000DFF848814FF0000A0AE003F17300C0B293
:1031900003F010FB33780AF1010A53457FF794AC32
:1031A00057F8043F99F800001844A0F18B0388FBFE
:1031B0000321DA17C2EB61020C3802EB42027F28CE
:1031C000A3EB8203E1DCFDF747FAE0E70398002177
:1031D00001704249097800293EF4EFAF3949029164
:1031E0000978002900F08881029800210170FEF71B
:1031F000E4BF039B1B78002B7FF446AB029B1B783C
:10320000002B7FF441AB019B1988FFF743BB0B7088
:103210003B681E44A6F118007F2840F301812B4B28
:10322000973E83FB0632F317C3EB620303EB4303C2
:10323000A6EB830606F173002B4BC0B2197803F09E
:1032400091FA64E50A707344A3F118007F2840F3F3
:10325000F1801E4A973B82FB0321DA17C2EB610221
:1032600002EB4202A3EB820303F17300C0B298F8B1
:10327000001003F077FA3B6806E6243B002BB9F810
:10328000000040F32F8198423EF40FAF9BB21748E5
:10329000A9F8003001230370FEF707BFDFF848806C
:1032A000C0B298F8001003F05DFAFFF707BB0E4BB1
:1032B0003878197803F056FA2EE500BF889CFF1F76
:1032C000369CFF1F089CFF1F3489FF1FABAAAA2A48
:1032D000F89BFF1FA89CFF1F709DFF1F749DFF1F81
:1032E000349CFF1F7489FF1F409CFF1F869CFF1F9B
:1032F0007F21402003F00EFAB349B44A3B680B60CB
:103300000021117034E5C0B298F8001003F02AFAD9
:10331000FFF7C8B8D8B298F8001003F023FA3B685A
:10332000B7E5AB4BDFF8ECE21978FEF7BEBE4B2EEB
:1033300040F3A9801836802EB9F80030A54AA8BFFE
:103340008026B3427FF4FBADFEF7D7BE99F80000AC
:1033500003F030FA3188FFF79DBA9F4B01931B8829
:10336000002B7FF45AAE9D4B029363E6029B1B78C1
:10337000002B7FF449AA039B1B78002B7FF484AABF
:1033800041E7002213460A70ACE4FDF765F90FE44B
:10339000FDF762F962E6FDF75FF9FFE400221646E9
:1033A0000A7059E5FDF758F9FFF767B98C4E307888
:1033B00000F07AFE8B4B1B781BB133887E2B40F2DA
:1033C000A780894B1B7823B13388854A002B40F0B6
:1033D000AB80864E3B783370FEF778BD824B1B780E
:1033E000002BF6D033887E4A002BF2D08049013B77
:1033F000088899B2118000287FF46BADC8B27B4E6B
:1034000003F0FCF93B783370FEF760BD7F20FFF7D7
:10341000CAB9FDF721F9FFF710BAFDF71DF953E41A
:10342000FDF71AF908E7FDF717F9FFF725BA7F202E
:10343000FFF7B7B8FDF710F918E7FDF70DF9FCE451
:10344000664F6C4902974FF0000C81F800C0009F56
:1034500002994FF0010E87F800E081F800C049E6BC
:103460000120FFF7A0B903F0A5F9FFF70FB900217C
:10347000402003F04FF9FFF770BB99F8000003F00C
:1034800099F9FFF765BB243E002EB9F800303ADD0C
:10349000B3423EF432AEB6B2574BA9F800600122F7
:1034A0001A70FEF72ABE0120FFF77BB84A4B019342
:1034B0001B88002B7FF4B3ADFFF7A2B94F4A8342BC
:1034C000A8BF03461360FEF7CFBF16462CE5FDF7F5
:1034D000C3F847E6FDF7C0F8FFF713BBFDF7BCF8EC
:1034E000FFF72EBB01283EF4E0AD0123CFE699F8AB
:1034F000000003F05FF91AE44148009041483D495B
:103500000390FEF751BE012B3EF4F7AD0126C3E751
:1035100001339BB23380D9B20520344E03F0FAF860
:103520003B783370FEF7D2BC013B9BB2D9B2052089
:103530002E4E138003F0EEF83B783370FEF7C6BCD6
:10354000029B1B78002B7FF45FA9FFF79DB92E4BE0
:103550001B782BB32D4B1B78002B7EF4CEAD2C4B60
:103560001B78002B3EF4C9ADB9F8003022490A336C
:10357000A9F800300A70FEF7C0BD244B1B78002B61
:103580007EF4BBAD224B1B78002B3EF4B6ADB9F8F0
:1035900000301949013BA9F800300A70FEF7ADBDB3
:1035A0001A4B1B78002B7FF412AA194B1B78002BA7
:1035B0003EF4A3ADB9F800300F490133A9F800304B
:1035C0000A70FEF79ABD00BF1C9DFF1F3489FF1FC4
:1035D000A59CFF1F149CFF1F889CFF1F089CFF1FBA
:1035E000389CFF1F589CFF1FF89BFF1F829CFF1FEA
:1035F0000A9CFF1F349CFF1F869CFF1F509CFF1FCF
:10360000A89CFF1F369CFF1F719DFF1F739DFF1F0E
:10361000549CFF1F4C9DFF1F224B00227F2107203F
:103620001A8003F077F87F210B2003F073F8FFF77F
:1036300001BA1D4B01227F2107201A8003F06AF88E
:103640007F210B2003F066F8FFF7ECB9174B04223B
:103650007F2107201A8003F05DF800210B2003F082
:1036600059F8FFF7D8B9114B02227F2107201A80A1
:1036700003F050F87F210B2003F04CF8FFF7C6B998
:103680000A4B002107201E8003F044F87F210B2005
:1036900003F040F8FFF7B5B9054B0393054B0293D0
:1036A000BDE400BF7E9DFF1FE49CFF1FEC9BFF1F3E
:1036B000369CFF1F089CFF1F38B506F0E1FD0B4844
:1036C00004F018FD00234FF07E5201210848FCF75A
:1036D000CDFE084B084A0949802400251C71184674
:1036E0001D60BDE838400AF08DBA00BFA09CFF1FE6
:1036F000609CFF1F989CFF1F1C89FF1FFD05000099
:1037000043682A20198803F089B900BF10B5044620
:1037100022206368198803F081F9E368242019885E
:10372000BDE8104003F07AB910B504460A2063687A
:10373000198803F073F9E3680C201988BDE810407C
:1037400003F06CB910B5044606206368198803F0CD
:1037500065F9E36808201988BDE8104003F05EB9F8
:1037600010B5044602206368198803F057F9E3682E
:1037700004201988BDE8104003F050B970B50E4C14
:1037800084B01225042201230646039002932046AA
:103790008DE824001423102105F0B0FE0622092331
:1037A000029303960195204600921423102105F000
:1037B000A5FE04B070BD00BFA89DFF1F2DE9F0411C
:1037C000224D82B0012602B284B2009228460196B0
:1037D0007823192105F0D8FD04F10C0212B28DE80E
:1037E00044002846A7197823192104F1020805F09E
:1037F000CBFD3FB20FFA88F819233A4628461946FE
:103800000196CDF8008005F0BFFD78233A462846A2
:103810001946CDF80080019604F10A070B3405F033
:10382000B3FD3FB224B278233A46284619468DE8C4
:10383000500005F0A9FD192300943A460196284648
:10384000194605F0A1FD02B0BDE8F081A89DFF1F5B
:103850002DE9F0411E4682B01446002A6AD0099B29
:103860004D4A00EBC305012C6F8929896868A7EBD5
:10387000010382FB03E21A444FEAE373C3EBA21392
:1038800002887BD0042C38D112FA83F3994203DCEE
:103890009F423946A8BF1946089A0180B6F9003000
:1038A000BDF920803D48971D4FF0000E3FB21946EC
:1038B00042460097CDF804E005F066FD29896A8943
:1038C0006B68521A1B885C2AA3EB010359DD03EBDA
:1038D00043030132C3EB431393FBF2F303F11B02E7
:1038E00013B20120328019464246019000972B48BE
:1038F00005F04AFD2A4B00221A702A4B022CB3F91C
:10390000001045D0082C31D100221A8091422DD0D0
:10391000089AB6F9003021480632012412B200920A
:1039200019460194BDF9202005F02EFD204602B075
:10393000BDE8F0811C4D1D4A2B681268CB1A9342DA
:103940000F4617D9164A338811781448012918BF31
:1039500001241470089A06321BB212B28DE81400CA
:103960001946BDF9202005F00FFD2F60012002B09F
:10397000BDE8F081204602B0BDE8F0819BB2D31AC9
:1039800084E75C2101FB03F393FBF2F21B32A7E710
:103990004A1C12B21A80B9E7C94216B2A89DFF1F8D
:1039A0002E9EFF1F909DFF1F0C9EFF1FF8FB000027
:1039B00030B583B000230C4605B2009326225B236A
:1039C0001C210C4805F030FA29460123262209481B
:1039D00004F03AFD002C24B205DB21460123262207
:1039E000044804F031FD044A044B15801C8003B0E8
:1039F00030BD00BFA89DFF1FAE89FF1FB089FF1F0C
:103A000070B5944C237882B01BB1934B4FF6FF7284
:103A10001A80924BB3F90030C3B9914A8E4B1068AB
:103A2000B3F9002080F30C005B2303FB00F00013CC
:103A30001C3082425AD04FF0FF31FFF7B9FF89485E
:103A400005F056FA0023237002B070BD012B32D06E
:103A5000022B6AD0032B4FD0042BF3D12722002551
:103A60008DE8240076231C217E487F4E05F08CFCD7
:103A700017E0B0F5AF7FA8BF4FF4AF70323803FB4B
:103A800000F386FB0321DB17C3EB61111C3109B284
:103A900001231D442722734804F0D6FC0C2D00F0AE
:103AA0008180E9B2714804F08DFB31284FF05B034F
:103AB000DFDC1C21ECE76E4B1A68B2F52F7F32DB9E
:103AC00041F25C239342A8BF1346A3F52F735B22F8
:103AD000684802FB03F380FB0320DB17C3EBA02045
:103AE0001C305D4BB3F900308342A4D1624BB3F973
:103AF000003001339FD1A5E7604B1B68B3F5FA7F17
:103B000011DBB3F57A6FA8BF4FF47A63A3F5FA72AD
:103B10005B485B2303FB02F380FB0320DB17C3EB53
:103B200020201C30DDE71C20DBE7564B1B68B3F57B
:103B3000FA7F33DBB3F57A6FA8BF4FF47A63A3F54E
:103B4000FA724F485B2303FB02F380FB0320DB1771
:103B5000C3EB20201C304C4B1B68B3F5FA7F1FDBF6
:103B6000B3F57A6FA8BF4FF47A63A3F5FA724449AC
:103B70005B2303FB02F381FB0321DB17C3EB212152
:103B80001C31354BB3F9003083427FF456AF3A4BCA
:103B9000B3F900308B427FF450AF53E71C20DAE7D3
:103BA0001C21EEE7012007F013FA6FF49573323809
:103BB000364A03FB00F082FB0023C017C0EB6323EF
:103BC00003F5AF73312B3ADDB3F5AF7FA8BF4FF4E8
:103BD000AF735B22323B244D02FB03F385FB0325CD
:103BE000DB17C3EB65151C35002007F0F1F96FF406
:103BF00095733238254A03FB00F082FB0023C0177F
:103C0000C0EB632303F5AF73312B1ADDB3F5AF7F40
:103C1000A8BF4FF4AF735B22323B134902FB03F39F
:103C200081FB0321DB17C3EB61111C310A4BB3F994
:103C30000030AB4207D02846FFF7BAFEFFE61C254E
:103C4000D2E71C21F2E70C4BB3F900308B42F2D1E2
:103C5000F5E600BF869DFF1FAE89FF1F8C9DFF1FED
:103C6000F09BFF1FA89DFF1F4B48371BA09CFF1F09
:103C70003C9DFF1FD3058541B089FF1F489DFF1F55
:103C8000011FB812E49BFF1FB09CFF1F67BBCF460C
:103C90002DE9F04FDFF8EC82B74CB8F900604D78B1
:103CA00054F8264087B08246039305B10D78DFF8BB
:103CB000FCB2002A34D19BF800308BBBAF4EB6F972
:103CC0000000002800F0CE80012800F024810120AF
:103CD00032232A46019000935146A94B2046FFF714
:103CE000B7FD00250746B6F90030022B40F3F480FB
:103CF00000233380B8F90030A24A002BC0F2F880CC
:103D0000042BC4BF00231380039B002B40F0F680DC
:103D1000002D0CBF38464FF0FF3007B0BDE8F08FE4
:103D2000964EE368226898480493002705923780EE
:103D30008BF8007004F0D0FF1120FFF73FFD4FF02B
:103D4000010919232821CDF8049000912422194655
:103D50008D4805F019FB782328212422CDF8049002
:103D600000918948194605F00FFB4946864805F041
:103D7000A1FE02221921844805F098FEDDF8149076
:103D800048460AF01DFD494602467F4806F028F8DD
:103D90007D4806F03BF8394614227B4805F086FE44
:103DA00003227A49784806F01BF8774806F02EF887
:103DB00039462322744805F079FE0322744972487B
:103DC00006F00EF8704806F021F8049B002B72D123
:103DD0000123704A18461370FFF7D0FC20896389CD
:103DE0006768191A5C293A885BDC131A5C2202FBAB
:103DF00003F292FBF1F31B33674A634813800127F8
:103E00001BB21A2219468DE88400142205F0BCFA70
:103E1000049BDBB1218A638AE768581A5C283A88D8
:103E20006FDD521A02EB4202C2EB4212431C92FBBC
:103E3000F3F31B33524A54481380012738221BB234
:103E40008DE884001946322205F09EFA534A544BFD
:103E5000B6F90000012111704FF6FF721A80002898
:103E60007FF432AFDFF848914E4AD9F8003012683B
:103E7000C3EB0A0393424CD9464B1A78012A18BF68
:103E8000012018700127FFF779FCC9F800A0012D67
:103E90004ED0042D59D0022D60D0082D64D00025BD
:103EA00021E7121A02EB4202C2EB42124B1C92FBB8
:103EB000F3F31B33A0E72F20FFF780FC39463222B3
:103EC000314805F0F3FD032237492F4805F088FFFC
:103ED0002D4805F09BFF7BE77FF40CAFE368002BD8
:103EE0003FF406AFB8F90030264A002BBFF608AF02
:103EF00004231380039B002B3FF40AAFFFF780FDE0
:103F000006E7511A5C2202FB01F292FBF0F31B332D
:103F100090E70746BBE7002714238DE888002A4670
:103F200051461D4B2046FFF793FC3D460746DAE617
:103F3000B8F800308BF800500133A8F800306369FE
:103F400083B1002520469847CDE6B8F8003001221D
:103F5000013BA8F800308BF80020F0E70123338004
:103F60000025C7E61D46BEE66369002232804FF099
:103F7000FF35002BE6D1BDE6B489FF1F909DFF1FE2
:103F80008A9DFF1F8C9DFF1FA89DFF1F94F00000BE
:103F900098F000002E9EFF1F889DFF1F869DFF1F2B
:103FA000AE89FF1FF8FB00009CF000008E9DFF1FF4
:103FB0000C9EFF1F01210D2006F0DCBD00210D200D
:103FC00006F0D8BD01460D2006F0D4BD08B50D2081
:103FD00006F0D6FDB0FA80F149090D20BDE8084091
:103FE00006F0C8BD10B5002144080D2006F0C2FD42
:103FF000204606F0FBFD0D20012106F0BBFD20460A
:10400000BDE8104006F0F2BD214A224B10881B6823
:10401000984210B535DA204A1288141A9A42A8BF7D
:104020001A46B4F5157F22DA121A40F2532303FB25
:1040300002F393FBF4F105310A2006F00BFC174B59
:10404000197801B3164B17491B6840F2271283F306
:10405000070302FB03F381FB03211944DB17C3EBC6
:10406000A11105310920BDE8104006F0F3BB131A79
:104070004FF41572611C02FB03F393FBF1F1053160
:10408000DAE70021D8E70920BDE8104006F0E2BBDE
:104090005A9CFF1F509CFF1F849DFF1F309DFF1FD8
:1040A000009DFF1F090402817F2838B5A8BF7F202B
:1040B0000F4C4FF4167202FB00F284FB02311144E4
:1040C000D2170546C2EBA1110A2006F0C3FB7F3DC3
:1040D0004FF4967303FB05F384FB03211944DB17AC
:1040E000A3EBA1110920BDE8384006F0B3BB00BF27
:1040F00009040281024B4E20198802F08FBC00BFD8
:10410000889CFF1F024B4420198802F087BC00BF27
:104110002E9DFF1F024B1020198802F07FBC00BFAC
:10412000A69CFF1F024B2C20198802F077BC00BF11
:10413000CE9CFF1F024B1E20198802F06FBC00BFEF
:10414000A29CFF1FC3680E20198802F067BC00BF45
:10415000024B2820198802F061BC00BF849CFF1F1D
:10416000024B6220198802F059BC00BFC09CFF1F9F
:10417000024B6420198802F051BC00BFCA9CFF1F8B
:10418000024B5A20198802F049BC00BFFA9BFF1F5E
:10419000024B1620198802F041BC00BF7E9DFF1F14
:1041A000024B2E20198802F039BC00BFE89CFF1F8B
:1041B000024B3020198802F031BC00BFE89BFF1F82
:1041C000024B1820198802F029BC00BF909CFF1FE9
:1041D000024B1A20198802F021BC00BFF89CFF1F77
:1041E000024B1C20198802F019BC00BF249DFF1F40
:1041F000024B6620198802F011BC00BFDC9BFF1F38
:10420000024B7220198802F009BC00BF6E9DFF1F8F
:10421000024B2020198802F001BC00BF829DFF1FC5
:10422000024B3220198802F0F9BB00BF5C9CFF1FD3
:10423000024B6820198802F0F1BB00BF0A9CFF1FE7
:10424000024B6C20198802F0E9BB00BFF69CFF1FEF
:10425000024B5220198802F0E1BB00BFAC89FF1F5E
:10426000024B5020198802F0D9BB00BF7489FF1F90
:10427000024B5420198802F0D1BB00BF9C89FF1F5C
:10428000024B5C20198802F0C9BB00BF7689FF1F72
:10429000024B5E20198802F0C1BB00BFA489FF1F3A
:1042A000024B6020198802F0B9BB00BFEA9BFF1FD8
:1042B000024B5620198802F0B1BB00BF809DFF1F42
:1042C00038B5094D4624204602F0C2FB35F8021BE2
:1042D00000B28842204601D002F0A0FB0234A4B212
:1042E0004E2CF0D138BD00BF549DFF1F064B074A2E
:1042F00010B41C88064B0846002C14BF1146194602
:10430000042210BC0AF01ABB269DFF1F90F7000084
:1043100094F70000064B074A10B41C88064B084669
:10432000002C14BF11461946042210BC0AF006BB2B
:10433000809CFF1F90F7000094F70000064B074A8F
:1043400010B41C88064B0846002C14BF11461946B1
:10435000042210BC0AF0F2BAB49CFF1F90F70000D0
:1043600094F70000064B074A10B41C88064B084619
:10437000002C14BF11461946042210BC0AF0DEBA04
:10438000209DFF1F90F7000094F70000064B074A9E
:1043900010B41C88064B0846002C14BF1146194661
:1043A000042210BC0AF0CABA289DFF1F90F7000033
:1043B00094F70000064B074A10B41C88064B0846C9
:1043C000002C14BF11461946042210BC0AF0B6BADC
:1043D000769DFF1F90F7000094F70000064B074AF8
:1043E00010B41C88064B0846002C14BF1146194611
:1043F000042210BC0AF0A2BAE49CFF1F90F7000050
:1044000094F70000F0B52B4E2B4FDFF8C4E00546C3
:104410000FCE87B06C460FC496E803003B68274A6E
:10442000274F44F8040B40F6CC308342C8BF3A46CD
:10443000BEF800602180012E11889278ADF80D1031
:104440008DF80F202AD032D340F6CA02022E18BFB0
:1044500000229A4226DCA3F698031A491A4AC3EBB3
:10446000031381FB03011944DB17C3EB61232433DE
:1044700082FB0321DA17C2EBA10202EB8201A3EB5C
:104480004103303330328DF813308DF811206946F6
:10449000284616220AF052FA07B0F0BD40F69802FC
:1044A0009A42D8DD094B1868CDF81100EFE740F6C5
:1044B000FC02CEE7A8F70000FC9CFF1F9CF7000061
:1044C00098F700003B773B9867666666A0F70000A8
:1044D000689DFF1FF8B5174C174E2278174D33789B
:1044E0002F888E46003218BF012201467046FFF722
:1044F000CFFB002398423370237015DB14BF0120DB
:1045000000202B889F420ED040F23A72A3F5AF7381
:104510000B490C4C02FB03F381FB0312DB17A3EBEB
:10452000621332332360F8BD0749012218460A702E
:104530002270E6E7588AFF1FA19DFF1FCC9CFF1F3A
:10454000B5814E1BA089FF1F249EFF1F014B1878C9
:1045500002F0FCB9089EFF1F014B187802F010BA58
:10456000BC8FFF1F134BB3F9003030B583EAE374FF
:10457000A4EBE374002BA0B218DB012300E0134688
:1045800003EB830252009442F9DA0B4D90FBF3F2F5
:1045900085FB03E403FB1200DB173032D3EBA403EB
:1045A00080B201F8012BF1D10B7030BD2D230B70BF
:1045B0000131E2E7BC8FFF1F67666666144BB3F9F3
:1045C000003070B583EAE375A5EBE375002BACB260
:1045D0001ADB012300E0034603EB83004000854221
:1045E000F9DA0C4E94FBF3F086FB03E503FB104471
:1045F000DB173030D3EBA503A4B201F8010BF1D1E6
:1046000005480B70106070BD2D230B700131E0E781
:10461000FA9BFF1F67666666C0F70000134BB3F98D
:10462000003030B583EAE374A4EBE374002BA0B24E
:1046300018DB012300E0134603EB8302520094428F
:10464000F9DA0B4D90FBF3F285FB03E403FB120058
:10465000DB173032D3EBA40380B201F8012BF1D188
:104660000B7030BD2D230B700131E2E7AC89FF1FC9
:1046700067666666134BB3F9003030B583EAE374BE
:10468000A4EBE374002BA0B218DB012300E0134677
:1046900003EB830252009442F9DA0B4D90FBF3F2E4
:1046A00085FB03E403FB1200DB173032D3EBA403DA
:1046B00080B201F8012BF1D10B7030BD2D230B70AE
:1046C0000131E2E77489FF1F67666666134BB3F931
:1046D000003030B583EAE374A4EBE374002BA0B29E
:1046E00018DB012300E0134603EB830252009442DF
:1046F000F9DA0B4D90FBF3F285FB03E403FB1200A8
:10470000DB173032D3EBA40380B201F8012BF1D1D7
:104710000B7030BD2D230B700131E2E79C89FF1F28
:1047200067666666134BB3F9003030B583EAE3740D
:10473000A4EBE374002BA0B218DB012300E01346C6
:1047400003EB830252009442F9DA0B4D90FBF3F233
:1047500085FB03E403FB1200DB173032D3EBA40329
:1047600080B201F8012BF1D10B7030BD2D230B70FD
:104770000131E2E77689FF1F67666666134BB3F97E
:10478000003030B583EAE374A4EBE374002BA0B2ED
:1047900018DB012300E0134603EB8302520094422E
:1047A000F9DA0B4D90FBF3F285FB03E403FB1200F7
:1047B000DB173032D3EBA40380B201F8012BF1D127
:1047C0000B7030BD2D230B700131E2E7A489FF1F70
:1047D00067666666054B1B881BB9054B1868086041
:1047E0007047044B18680860704700BF889CFF1F23
:1047F000C8F70000C4F70000164B1B880BB31BB2B0
:1048000030B583EAE374A4EBE374002BA0B21CDBA5
:10481000012300E0134603EB830252009442F9DACD
:104820000D4D90FBF3F285FB03E403FB1200DB1755
:104830003032D3EBA40380B201F8012BF1D10B701D
:1048400030BD064B1868086070472D230B7001318E
:10485000DEE700BFA29CFF1F6766666694F7000054
:10486000164B1B880BB31BB230B583EAE374A4EB81
:10487000E374002BA0B21CDB012300E0134603EB22
:10488000830252009442F9DA0D4D90FBF3F285FB5E
:1048900003E403FB1200DB173032D3EBA40380B236
:1048A00001F8012BF1D10B7030BD064B1868086080
:1048B00070472D230B700131DEE700BFF29CFF1F14
:1048C0006766666694F70000164B1B880BB31BB235
:1048D00030B583EAE374A4EBE374002BA0B21CDBD5
:1048E000012300E0134603EB830252009442F9DAFD
:1048F0000D4D90FBF3F285FB03E403FB1200DB1785
:104900003032D3EBA40380B201F8012BF1D10B704C
:1049100030BD064B1868086070472D230B700131BD
:10492000DEE700BF7E9DFF1F67666666CCF700006E
:10493000174B1B881BB31BB270B583EAE375A5EB5D
:10494000E375002BACB21EDB012300E0034603EB52
:10495000830040008542F9DA0E4E94FBF3F086FBAB
:1049600003E503FB1044DB173030D3EBA503A4B2FF
:1049700001F8010BF1D108480B70106070BD074BB6
:104980001868086070472D230B700131DCE700BF09
:10499000E89CFF1F67666666A4F7000094F70000B6
:1049A000164B1B880BB31BB230B583EAE374A4EB40
:1049B000E374002BA0B21CDB012300E0134603EBE1
:1049C000830252009442F9DA0D4D90FBF3F285FB1D
:1049D00003E403FB1200DB173032D3EBA40380B2F5
:1049E00001F8012BF1D10B7030BD064B186808603F
:1049F00070472D230B700131DEE700BFE89BFF1FDE
:104A00006766666694F70000164B1B880BB31BB2F3
:104A100030B583EAE374A4EBE374002BA0B21CDB93
:104A2000012300E0134603EB830252009442F9DABB
:104A30000D4D90FBF3F285FB03E403FB1200DB1743
:104A40003032D3EBA40380B201F8012BF1D10B700B
:104A500030BD064B1868086070472D230B7001317C
:104A6000DEE700BFDC9BFF1F6766666694F7000009
:104A7000164B1B880BB31BB230B583EAE374A4EB6F
:104A8000E374002BA0B21CDB012300E0134603EB10
:104A9000830252009442F9DA0D4D90FBF3F285FB4C
:104AA00003E403FB1200DB173032D3EBA40380B224
:104AB00001F8012BF1D10B7030BD064B186808606E
:104AC00070472D230B700131DEE700BF6E9DFF1F85
:104AD0006766666694F70000174B1B881BB31BB212
:104AE00070B583EAE375A5EBE375002BACB21EDB72
:104AF000012300E0034603EB830040008542F9DA1E
:104B00000E4E94FBF3F086FB03E503FB1044DB172A
:104B10003030D3EBA503A4B201F8010BF1D1084862
:104B20000B70106070BD074B1868086070472D232C
:104B30000B700131DCE700BF829DFF1F6766666670
:104B4000D0F7000094F70000074B1B88022B06D01B
:104B5000012B0CBF054B064B186808607047054BCE
:104B600018680860704700BFEA9BFF1FD8F7000075
:104B7000DCF70000D4F70000054B1B881BB1054B88
:104B8000186808607047044B18680860704700BFD9
:104B9000809DFF1FE4F70000E0F7000008B57020DB
:104BA00001F056FF044B1988884204D07020BDE8FC
:104BB000084001F033BF08BD689DFF1F08B5742091
:104BC00001F046FF044B1988884204D07420BDE8E8
:104BD000084001F023BF08BDBC9CFF1F38B5FCF79F
:104BE0003BFF0D4B1B7833B90C4B1020198801F09B
:104BF00015FF012038BD0A4D0A4C2B782288B3FAE4
:104C000083F382F008025B09114642202B70228058
:104C100001F004FF002038BD749DFF1FA69CFF1FFC
:104C2000449DFF1F249CFF1F184B1A8852B3184A3B
:104C3000128830B50A80B3F90030002B83EAE374A0
:104C4000A4EBE374BCBF2D238B70A0B2ACBF0231C8
:104C50000331012300E0134603EB83025200944228
:104C6000F9DA0C4D90FBF3F285FB03E403FB120031
:104C7000DB173032D3EBA40380B201F8012BF1D162
:104C80000B7030BD044B186808607047F89CFF1F1C
:104C9000E8F700006766666694F7000010B40A4BF8
:104CA0000A4C0A4693E8030083B0238802AC04E967
:104CB000030004EB8303104653F8081C052203B0DD
:104CC00010BC09F03BBE00BF24F10000CA9CFF1FCE
:104CD00030B40A4B0A4D0C4693E8070084B02B8889
:104CE00004AD05E9070005EB8303204653F80C1CCF
:104CF000042204B030BC09F021BE00BF2CF100003A
:104D0000689DFF1FF0B40C4D0C4F0E460FCD8CB0BC
:104D100001AC0FC40FCD0FC495E807003B8884E8B1
:104D200007000CAA02EB8303304653F82C1C042224
:104D30000CB0F0BC09F002BE38F10000EC9BFF1F84
:104D4000F0B40A4D0A4F0E460FCD86B001AC0FC429
:104D50002A683B88226006AA02EB8303304653F898
:104D6000141C042206B0F0BC09F0E8BD64F1000098
:104D7000909CFF1FF0B40A4D0A4F0E460FCD86B02F
:104D800001AC0FC42A683B88226006AA02EB8303A9
:104D9000304653F8141C0C2206B0F0BC09F0CEBD0E
:104DA00078F10000249DFF1FF0B40A4D0A4F0E4613
:104DB0000FCD86B001AC0FC42A683B88226006AADA
:104DC00002EB8303304653F8141C042206B0F0BCF7
:104DD00009F0B4BD8CF10000BC9CFF1F164B1B8872
:104DE0000BB31BB283EAE370A0EBE370002B30B58A
:104DF00084B21DDB012300E0134603EB8302520063
:104E00009042F9DA0D4894FBF3F280FB03E503FBD3
:104E10001244DB173032D3EBA503A4B201F8012B07
:104E2000F1D10B7030BD08460422054909F086BD5A
:104E30002D230B700131DDE70A9CFF1F6766666654
:104E4000ECF7000030B40A4B0A4D0C4693E807001B
:104E500084B02B8804AD05E9070005EB83032046E9
:104E600053F80C1C042204B030BC09F067BD00BF2D
:104E7000A0F10000F69CFF1F70B53C4D2B78064654
:104E8000002B35D11C4673780BB9204670BDFCF75A
:104E9000E3FD374A374B3848127831781B78007871
:104EA00002EB43034A1E03EB80030E2AEDD801A058
:104EB00050F822F01D4F00003F4F00008B4E0000C5
:104EC0001D4F00008B4E00008B4E00008B4E0000EB
:104ED0000B4F00008B4E00008B4E00008B4E0000ED
:104EE0008B4E00008B4E00008B4E0000074F0000E1
:104EF000AE21224803F0A0FC204803F0EDFE002381
:104F00002B700124BFE706F083F9AF211B4803F0A3
:104F100093FC1B4A012313702B70B6E783B9194821
:104F2000038804294FF6FF7103F1FF320CBF012300
:104F30000B46134403F07F03013303800FE073B18A
:104F4000013B114A32F813304BB10E4E0F48104955
:104F5000104A33800123002606700B701370084A34
:104F60000221012311702B70204670BD588AFF1F4B
:104F7000F89BFF1F589CFF1F7C9DFF1FA89DFF1FD4
:104F8000249EFF1F149CFF1FD09CFF1F459DFF1FE9
:104F9000869CFF1F309EFF1F10B5064B064C1A88DB
:104FA0002046012101F028FD21884220BDE8104063
:104FB00001F034BD269DFF1F249CFF1F10B5064B3A
:104FC000064C1A882046022101F016FD2188422055
:104FD000BDE8104001F022BD809CFF1F249CFF1FF4
:104FE00010B5064B064C1A882046042101F004FD3A
:104FF00021884220BDE8104001F010BDB49CFF1F85
:10500000249CFF1F10B5064B064C1A88204605212C
:1050100001F0F2FC21884220BDE8104001F0FEBC06
:10502000209DFF1F249CFF1F10B5064B064C1A88BD
:105030002046062101F0E0FC21884220BDE8104016
:1050400001F0ECBC289DFF1F249CFF1F10B5064BF0
:10505000064C1A882046002101F0CEFC218842200F
:10506000BDE8104001F0DABC769DFF1F249CFF1FB5
:1050700008B5122001F0ECFC054B1988884206D0D7
:10508000122001F0CBFCBDE8084001F0DFBB08BDF9
:10509000EC9BFF1F08B5582001F0DAFC054B19887E
:1050A000884206D0582001F0B9FCBDE8084001F064
:1050B000CDBB08BDF29CFF1F08B5142001F0C8FC51
:1050C000054B1988884206D0142001F0A7FCBDE8E2
:1050D000084001F0BBBB08BDE49CFF1FF0B480EAB0
:1050E000E075A5EBE0750028ACB21FDB1DBF2B23DC
:1050F0000B704E1C0E46012300E0134603EB8302A7
:1051000052009542F9DA0B4F94FBF3F287FB03054B
:1051100003FB1244DB173032D3EBA503A4B206F82D
:10512000012BF1D133700846F0BC70472D230B7072
:105130004E1CE0E767666666174B18880C2813D08C
:10514000192815D01A2817D01B2819D01C281BD0B5
:105150001D281DD01E2803D00C3800B2FFF7BEBF9B
:105160000E4A1068086070470D4A10680860704762
:105170000C4A1068086070470B4A10680860704756
:105180000A4A106808607047094A1068086070474A
:10519000084A1068086070475C9CFF1F0CF800000C
:1051A000F4F70000F8F70000FCF7000000F800003A
:1051B00004F8000008F80000034B1888A0EB8000FA
:1051C000400000B2FFF78ABF089EFF1F024BB3F9F1
:1051D0000000FFF783BF00BFC09CFF1F024B188871
:1051E000033800B2FFF77ABF849CFF1F024B188878
:1051F0000C3800B2FFF772BF3A9DFF1F024B1888B0
:10520000183800B2FFF76ABF2E9DFF1FC3681888C9
:10521000183800B2FFF762BF30B5134C85B00125D6
:105220002B463C2202212046009503F07BFB2046C2
:1052300003F052FD0022402180232046019100937B
:1052400011460A4B029504F0F5F9204603F050FE92
:1052500007480849084A0023036083800B608B805D
:105260001360938005B030BDA89DFF1FF8F10000CA
:10527000949DFF1F289EFF1F149EFF1F10B500EB7B
:10528000C00000F10F02D2B293B284B09C1E981CF1
:105290003D2303918DE819003921024804F02EF9CD
:1052A00004B010BDA89DFF1F014B01221A7070476A
:1052B000A19DFF1FF0B585B0684C694B0293694A08
:1052C0000192042300932046674B684F684E694D56
:1052D0004022802103F02EF92046674A6749684C36
:1052E00008F090FC674A684B9761684FD761684F38
:1052F0009F61684FDF61684FB761684FF761684F22
:10530000AF61684FEF61684FA7616848684FE76118
:10531000684F87616849694FC761694F8F61694A02
:10532000694FCF61694F9761694B6A4FD7616A4F87
:105330009F616A4E6A4FDF616A4F6B4DB7616B4F79
:10534000F7616B4F6B4CAF616B4FEF616B4F6C480C
:10535000A7616C4FE7616C4F6C4987616C4FC76107
:105360006C4F6D4A8F616D4FCF616D4F6D4B976183
:105370006D4FD7616D4F6E4E9F616E4FDF616E4F07
:10538000B7616E4D6E4FF7616E4FAF616E4C6F4FF0
:10539000EF616F4FA7616F486F4FE7616F4F876194
:1053A0006F49704FC761704F8F61704A704FCF6106
:1053B000704F9761704B714FD761714F9F61714E04
:1053C000714FDF61714FB761714D724FF761724F6D
:1053D000AF61724C724FEF61724FA7617248734FA9
:1053E000E761734F73498761734FC761734F744AA5
:1053F0008F61744FCF61744F744B9761744FD76155
:10540000744F754E9F61754FDF61754F754DB76174
:10541000754FF761754F764CAF61764F7648774997
:10542000EF61774F774DA761DFF808E2E561764FCE
:10543000764D774C774A784B8761C5618C61774EA2
:10544000774F784D784CC1F81CE0784878499761DF
:10545000D5619C61D861B16005B0F0BDA89DFF1F0A
:10546000A0860100801A0600FC8FFF1FED5100008E
:10547000908DFF1F9C8BFF1F1C89FF1F8D850000D7
:10548000448EFF1FE08CFF1F208EFF1F4541000050
:10549000DD51000051410000ED420000994F000035
:1054A00015430000BD4F00003D430000748CFF1FFA
:1054B000E14F000065430000EC89FF1F055000002C
:1054C000CD5100002C8CFF1F614100008D43000076
:1054D000C08FFF1F295000009D4C0000088CFF1F4B
:1054E00071410000B5430000BC8CFF1F4D5000000F
:1054F000B9510000988CFF1F4D4500006545000024
:10550000FC8DFF1F59450000D14C0000548BFF1F3C
:105510009D4B0000054D0000AC8EFF1F7150000038
:1055200061480000E48BFF1F95500000BD4500005E
:10553000108BFF1F81410000DD430000188FFF1F0B
:10554000B9500000C9480000C08BFF1F9141000006
:1055500031490000048DFF1FA1410000A149000056
:10556000808AFF1FB1410000414D0000508CFF1F99
:10557000C1410000294C0000D88DFF1FD14100001F
:10558000754D0000988FFF1FE1410000094A00009F
:105590006C8DFF1FF1410000714A0000A48AFF1FBB
:1055A00001420000A94D0000D08EFF1FBD4B00003E
:1055B000D94A0000B48DFF1F11420000395100008C
:1055C000C88AFF1F21420000DD4D00005C8AFF1FDA
:1055D00031420000454E0000688FFF1F414200002D
:1055E0001D460000788BFF1F5142000075460000E9
:1055F000348AFF1F61420000EC8AFF1F688EFF1F84
:10560000CD460000714200002547000081420000A5
:105610007D470000108AFF1FC889FF1F8C8FFF1F66
:10562000494B0000A1420000794B0000B14200004C
:10563000ED5B000091420000F0B5461C83B00D46C2
:105640000127032336B22AB2044631468DE888008A
:105650002448ADB203F0E8FE0C23AA1C12B200935A
:105660000197052321B21F4803F0DEFE1E4A1F4B9F
:1056700012881B68BA422AD023D3022A10D11C4CAC
:10568000A3F6CA0384FB03241C44DB17C3EB2414D6
:105690000A2CA8BF0A2424EAE474A2B223B202E0CE
:1056A00000231A461C460D35AA1A012000930190CA
:1056B00012B2314603230B4803F034FE204603B0F8
:1056C000F0BD0C4CA3F6FC0384FB0324DDE7084C7F
:1056D000A3F6980384FB03241C44DB17C3EBE40408
:1056E000D6E700BFA89DFF1F689DFF1FFC9CFF1F02
:1056F000898888881F85EB512DE9F0438FB283B0EC
:10570000DFF84C80BD1D461D2DB204B236B24FF0FD
:1057100001090AB22346314640460095CDF804906F
:1057200003F032FE2A463346214640468DE82002E9
:1057300003F02AFE07F10C020095334612B221460F
:10574000CDF80490404603F01FFE03B0BDE8F0839F
:10575000A89DFF1F2DE9F043804685B0002956D152
:105760000121304804F0A6F92F4998F8062098F84E
:10577000083011F80290994522DA4FEA89064D4621
:105780000C24D8F80C3027489B595F6822B20021BE
:1057900004F08CF9384609F013F8394602462148DE
:1057A00004F01EFB1F4804F031FB98F80830013567
:1057B0000934AB42A4B206F1040601DD422CE0D16B
:1057C000B9F1000F13D109F1060999450CDA3C2310
:1057D00001213B22039102930093019239233F223E
:1057E0003A21104803F08AFE05B0BDE8F0830F238C
:1057F00001213B22039102930093019239230C2251
:105800003A21084803F07AFE98F80830DBE70021D7
:105810003423009301913F230C22024803F082FDC0
:105820009EE700BFA89DFF1F289EFF1F10B5104CCC
:105830000121204604F044F92046012104F03AF900
:1058400020463422552104F031F92046022209492C
:1058500004F0C6FA20460522074904F0C1FA2046A2
:1058600004F0D4FA2046BDE8104003F041BB00BF6D
:10587000A89DFF1F10F8000014F8000070B50D4639
:10588000064608F09DFF00EB40008400002D36D056
:10589000284608F095FF00EB4000400023185B10FD
:1058A00003F16001091A282209B21748C3F1600404
:1058B00004F0FCF80121144804F0FCF8284608F034
:1058C0007FFF29460246104804F08AFA0E4804F089
:1058D0009DFA02210C4804F0EDF821B221220A4879
:1058E00004F0E4F8304608F06BFF31460246064803
:1058F00004F076FA0448BDE8704004F087BA6410FA
:10590000C4F16004E5E700BFA89DFF1F10B50D4B73
:105910001B5C51F82340237884B013B1012004B0FC
:1059200010BD04AA01A942F8103D2046A36998477A
:10593000A38A9B07F2D401A80099FFF79FFF0120DB
:1059400004B010BD949DFF1F2DE9F04F2F4DDFF8DF
:10595000CCB0DFF8C4A0DFF8C8900FCD91B003AC95
:105960000FC40FCD0FC40FCD0FC42B6823600025CB
:10597000A8462F462E4600E09846BAF80030244943
:105980005BF8232028461123FAF7FEFF00EBC00442
:1059900000EB840089FB00340444C017C0EB64347E
:1059A000C4F13C00C6F13C0207F14101012600B2FE
:1059B00008F1410300901BB2019612B209B21548DA
:1059C00003F0E2FC08EB060305F211153C2B26461A
:1059D000ADB24746D0D134226B210E4804F066F8B0
:1059E00000210C4804F066F80B4B1B8810AA02EB50
:1059F000830353F8344C204608F0E2FE0246054883
:105A0000214611B0BDE8F04F04F0EAB9ACF1000056
:105A10007CED0000A89DFF1FCE9CFF1F1CEF000027
:105A200009000280214B70B5B3F9003083EAE374BA
:105A3000A4EBE374002B82B0A1B22FDB68466D4665
:105A4000012300E0134603EB830252009442F9DA8B
:105A5000174E91FBF3F286FB03E403FB1211DB17F5
:105A60003032D3EBA40389B205F8012BF1D11946EA
:105A70002B70FFF703FF0F4B1B786BB101210E4812
:105A800004F018F8332274210B4804F00FF80122B7
:105A90000A49094804F0A4F902B070BD2D238DF81D
:105AA00000300DF101056846CAE700BFA69CFF1F44
:105AB00067666666449DFF1FA89DFF1FB8FB000038
:105AC00010B5424C424882B003F006F92378C3B9BE
:105AD00006213F4803F0EEFF2378012B37D90A2235
:105AE000022B11463A486BD003F0E0FF39490322FC
:105AF000374804F075F9364802B0BDE8104004F0AC
:105B000085B9354B1A7801210523002A35D1019139
:105B1000009311462E4803F087FC304B1A78002A78
:105B200036D0052301220192009300220A21284841
:105B300003F0F8FB2A4B1A78002A35D101210523FE
:105B4000019100931421224803F06EFCC0E7254C1C
:105B50002388092B32D9632B8CBF0A211F210A22EB
:105B60001B4803F0A3FF2188194804F09FF9184847
:105B700002B0BDE8104004F049B900220191009341
:105B80001146134803F0CEFB144B1A78002AC8D1F3
:105B900005230121019100930A210D4803F044FCE3
:105BA0000F4B1A78002AC9D00122052301920093D5
:105BB00000221421064803F0B5FB89E73021CEE727
:105BC00003F074FF0322084992E700BF309EFF1FD5
:105BD000A89DFF1F20F80000F89BFF1F589CFF1F87
:105BE0007C9DFF1F149CFF1F1CF80000F8B56D4D35
:105BF000287840B96C4B1B6899425CD36B4A0123EF
:105C000013702B70F8BD0C4600266948664F03F0F0
:105C100063F804F6AC53324665483B6031212E7080
:105C200003F044FF01216248624D03F049FF314611
:105C30005F4803F03FFF05225F495D4804F0D0F85C
:105C40005B4804F0E3F80C221021594803F02EFFC2
:105C50000B225A49564804F0C3F8052258495448C3
:105C600004F0BEF8524804F0D1F8564B50481C6876
:105C7000A4F69803C3EB031385FB03251D441021F1
:105C8000DB172022C3EB652503F010FF40F6CC3371
:105C90009C4205F124054FF022014FF004000BDC7B
:105CA000FFF7CAFC484B1C88064674B3012C46D04B
:105CB000022C41D00120F8BDFFF71EFD0922434907
:105CC0003B4804F08DF82A221021394803F0EEFEFB
:105CD0003F4C374884FB0534EB17C3EBA404214643
:105CE00004F0E4F801223B49314804F079F804EB70
:105CF0008401A5EB41012E4804F0D8F80122364971
:105D00002B4804F06DF80120F8BD344910222848D2
:105D100004F066F8264804F079F82A221021244875
:105D200003F0C4FE3146224804F0C0F807222C4993
:105D30001F4804F055F8CBE70C222A49E7E70C226C
:105D400029491B4804F04CF8194804F05FF82A224E
:105D50001021174803F0AAFE314615481C4E04F0E6
:105D6000A5F807221E49124804F03AF886FB0536CA
:105D7000EB17C3EBA60631460D4804F097F8224610
:105D800014490B4804F02CF806EB8601A5EB410101
:105D9000074804F08BF822460F49054804F020F824
:105DA0002046F8BD588AFF1F109EFF1F249EFF1F2C
:105DB000A89DFF1F3B773B9824F800002CF80000BB
:105DC00014F80000FC9CFF1F689DFF1F38F80000BE
:105DD0006766666624FD00009CFC000044F8000035
:105DE00058F8000070F8000060F800002DE9F0415C
:105DF000754C2278002A05460F4614BF4FF0010863
:105E00004FF000084ED1714E3368CB1AB3F5FA6FDC
:105E100004D86B78A3B94046BDE8F0816C4B6D485F
:105E20006D49DFF8D0E11A700123037009882370EF
:105E300026208EF8002000F0F1FD6B78002BEAD0D0
:105E40003760FBF709FE654A654B6649127828788A
:105E50001B78097802EB4303421E03EB81030E2AF1
:105E6000D9D801A151F822F0595F0000255F000048
:105E7000175E0000595F0000175E0000175E00000B
:105E8000175E00000D5F0000175E0000BF5E00009F
:105E9000175E0000175E0000175E0000175E00002E
:105EA000BB5E0000AF215048484E02F0C5FCFFF732
:105EB00007FE002337602370ABE705F0A9F94A48D5
:105EC00002F00AFF0221484803F0F4FD0F222321CB
:105ED000454803F0EBFD05224449434803F080FFA9
:105EE000414803F093FF1E2223213F4803F0DEFDCB
:105EF00005223F493C4803F073FF3B4803F086FF0F
:105F0000394802F0F5FF00F0ADFC84E7394D2B78FD
:105F1000012B50D9304B2620198800F07FFD00233B
:105F20002B7078E7002B3FF476AF013B324A32F812
:105F30001330002B3FF46FAF274C304825492D4AD2
:105F400023804FF001080023037081F8008082F85D
:105F50000080FFF7B5FD5EE793B1013B264A32F8BA
:105F6000131019B31C4B254D1A4C224A19800026D8
:105F7000012326202E702370137000F04FFD15E0D2
:105F8000154C1E4922880B7004284FF6FF7002F151
:105F9000FF310CBF012202460A440E4E154D02F09D
:105FA0007F0201320121228031702B70FFF788FDC2
:105FB0004FF001082FE70649064A01230020087028
:105FC00013702370A6E700BF588AFF1F209EFF1F93
:105FD000249EFF1F869CFF1F149CFF1FF89BFF1F22
:105FE000589CFF1F7C9DFF1FA89DFF1F80F800008D
:105FF00088F80000309EFF1FD09CFF1F459DFF1FAB
:106000002DE9F04F05468BB00F46AD4801211646ED
:1060100003F056FDAA8812F0010440F0B080DFF8CA
:10602000CC8298F80030002B7DD1AB79A54AD15CA9
:10603000A1B9DFF8BCA279781AF8039041B3397896
:106040000139072900F2B780DFE811F0F1005401AF
:10605000B5006C01B500B500B500E9007C78002CF6
:1060600000F0CA800139EC68387854F82170FC6877
:10607000411EB4F80080072900F2A780DFE811F084
:1060800074015901A5006C01A500A500A5009F00A1
:10609000DFF854A2DAF80020B21AB2F5967F75D96B
:1060A000894A107801281ABF012010701170874AA0
:1060B00018BF0146D05CC0EB0900C0B2FFF7DEF8A4
:1060C0000124CAF80060AB889B0770D57B78002B51
:1060D0006DD0FBF7C1FC7E4B7E4A7F481B7812785F
:1060E00039780078022515FB02330A2903EB800377
:1060F00000F04E810C295AD1002B58D003F1190021
:10610000764E774A013B0021400080B226F81310FA
:106110000123157088F8003000F080FC714B0322D9
:1061200020461A702FE0664802F0D6FD012164482F
:1061300003F0C0FC62482246214603F0B7FCAB885E
:10614000580725D42C68204608F03AFB2146024621
:106150005B4803F045FE5A4803F058FE092201232C
:106160008DE80C0000217F23554803F00DF9002134
:106170002846FFF7EFFA002388F8003055E7AB68B0
:106180003146384698470BB0BDE8F08F0846FAE72D
:106190002B6804A8984704A808F012FB04A902463B
:1061A000474803F01DFE464803F030FED6E7204680
:1061B0000BB0BDE8F08F00240AF8039083E70021BC
:1061C000D1543846FB699847FC68A4F80080002742
:1061D00025223C238DE8840041211822384803F011
:1061E000A1F8E968A879FFF791FB374A3E4B177091
:1061F0001E600BB0BDE8F08F3B490A68B21AB2F5D9
:10620000967FD4D9304F0E603E78012E00F0B480D6
:10621000E968184601233B70FFF778FBB3E7304A83
:10622000E9791170012288F800200024C4E72A7A55
:10623000013A4A45BFDD09F10104E4B2A145BAD0F3
:10624000224E16F803B0CBEB0900C0B20021FFF7D5
:1062500015F82B7A052BD9461BD9CBEB0402042A5F
:1062600040F3AE80A4F1040BBBF1000FC0F2B0808C
:10627000063B5B45A8BF5B465FFA83F9AA791348E2
:10628000B15C994205D000F8029001212846FFF741
:1062900061FAC9EB0400C0B201210B4EFEF7EEFF1C
:1062A00000213423019100930548317040230B22D3
:1062B0003F21A14603F036F80124AB797CE700BF0B
:1062C000A89DFF1F149EFF1F2E9EFF1F289EFF1FCD
:1062D000F89BFF1F589CFF1F7C9DFF1FD09CFF1F3A
:1062E000249EFF1F309EFF1F0C9EFF1F588AFF1F1A
:1062F000949DFF1F0FFA89F1E868604C50F8216007
:106300002168049134785E4904980860002C71D0AB
:10631000012C7FF450AF5B4A317A88F8004011704D
:10632000002449E7B9F1000F50D009F1FF34E4B27D
:1063300084E7B98A01F0040189B200293FF440AF33
:106340003B6A03929847039A00283FF43DAFAB792C
:10635000FC680021D15438E77B8A43453CD908F1D9
:1063600001081FFA88F830E73B8A43453BD208F121
:10637000FF381FFA88F828E725238DE818004248DF
:106380003C703C231822412102F0CCFF3046FAE653
:10639000002B3FF40CAF3D4A3D4E1188394A03F1C2
:1063A0001900013B400080B226F81310012388F841
:1063B0000030157000F032FB364B20461D70E2E6CF
:1063C000002A3FF755AF04F1FF3B4DE74C46F3E69B
:1063D0004FF000094B4651E7BB8ADA077FF5F5AE6F
:1063E000B7F81080F1E6BB8AD9077FF5EEAEB7F8B3
:1063F0001280EAE62849C85CC0EB090009F1010EE9
:10640000C0B201214FF0340B02F803E0FEF736FF73
:10641000B6681D48019440230B223F210124CDF88A
:1064200000B002F07FFF40230B223F211648CDF839
:1064300000B0019402F0F8FF2146134803F03AFB44
:10644000304608F0BDF9A0EB800000F15F0109B211
:106450000F220D4803F02AFB304608F0B1F931460F
:106460000246094803F0BCFC074803F0CFFCE9688A
:10647000A879FFF74BFAAB799EE600BF6C9EFF1F31
:106480000C9EFF1F249EFF1FA89DFF1F149CFF1F33
:10649000D09CFF1F309EFF1F289EFF1F2DE9F04755
:1064A000DFF808926D4B99F800601B68DFF800A2D6
:1064B00082B0003601934FF0030018BF0126019F00
:1064C0009AF8008004F05CFB0546042004F058FBB9
:1064D0000446052004F054FB800040EA44040620F2
:1064E00004F04EFB2C4364B25D4944EAC0000A78D4
:1064F00080F00F03DBB29A425A4A3CD01760002268
:1065000059480B7003788DF800808DF8012053B343
:10651000564A12684EF66021BA1A8A4219D8022BDE
:1065200059D0012B5FD0062B48D0032B63D0042B0E
:1065300069D0052B77D0072B7DD0082B00F0838006
:10654000092B68D016B14A4802F0D2FC02B0BDE86F
:10655000F087484A484C00230121237003701360E0
:10656000938089F800103A4669464448FFF748FD91
:106570003043C6B2E6E71268BA1A1E2A6BD99AF8F7
:106580000020934222D0394C3D488AF80030012B3C
:10659000276082EA030207609846B1D0042BAFD18E
:1065A00037480068381AB0F5C87FA9D9354C20683B
:1065B000381A3228A4D927601A46A1E73A46694614
:1065C0003148FFF71DFD3043C6B2BBE7012B4FF04A
:1065D0000002E3D1E4E73A4669462C48FFF710FD94
:1065E0003043C6B2AEE73A4669462948FFF708FD90
:1065F0003043C6B2A6E73A4669462648FFF700FD93
:106600003043C6B29EE73A4669462348FFF7F8FC96
:106610003043C6B296E73A4669462048FFF7F0FC99
:106620003043C6B28EE73A4669461D48FFF7E8FC9C
:106630003043C6B286E73A4669461A48FFF7E0FC9F
:106640003043C6B27EE73A4669461748FFF7D8FCA2
:106650003043C6B276E7002252E700BF6C9EFF1FB0
:10666000319EFF1F9C9DFF1F249EFF1F1C9EFF1F2E
:10667000A89DFF1F149EFF1F2F9EFF1FE4F6000022
:10668000349EFF1FA49DFF1F38F70000A8F60000EE
:1066900008F60000ECF100003CF60000F8F5000000
:1066A0004CF600008CF600008C8FFF1F588AFF1FED
:1066B000A09DFF1F28B11028044BA8BF1020186010
:1066C0007047024B01201860704700BF389EFF1FC3
:1066D00038B50F4D2B78013B01381B02C4B203F4CF
:1066E0007063200443F4404343F00C0300F4FE00C5
:1066F000184305F0ADFB2868013860F03F00C0B2D8
:1067000004F0D4FB2046BDE8384004F0CFBB00BF06
:10671000389EFF1F70B5124D2B78013B1B0203F40E
:106720007063064643F430430806320400F0FE402E
:1067300043F00B03034302F4FE0018430C4605F03C
:1067400087FB2868013860F04F00C0B204F0AEFB50
:10675000304604F0ABFB2046BDE8704004F0A6BB19
:10676000389EFF1F70B5124D2B78013B1B0203F4BE
:106770007063064643F410430806320400F0FE40FE
:1067800043F00903034302F4FE0018430C4605F0EE
:106790005FFB2868013860F06F00C0B204F086FB30
:1067A000304604F083FB2046BDE8704004F07EBB19
:1067B000389EFF1F38B5104D2B78013B1B0203F4A8
:1067C0007063044643F41043000443F0090300F4EB
:1067D000FE00184305F03CFB2868013860F06F00AC
:1067E000C0B204F063FB204604F060FB0020BDE86B
:1067F000384004F05BBB00BF389EFF1F38B50E4D1C
:106800002B78013B1B0203F47063044643F45043AE
:10681000000443F00D0300F4FE00184305F018FBDC
:106820002868013860F02F00C0B204F03FFB20461A
:10683000BDE8384004F03ABB389EFF1F08B5002081
:1068400005F0D0FB0028FAD108BD00BF08B56421CF
:106850000720FFF75FFF7F210B20BDE80840FFF70F
:1068600059BF00BF10B500217B20FFF753FF002464
:10687000E0B2FFF79FFF0134022004F0B7F9802C4B
:10688000F6D110BD10B504464FF4406004F0BEFAD6
:1068900004F016FB2CB1102C044BA8BF10241C6074
:1068A00010BD024B01241C6010BD00BF389EFF1FAD
:1068B00010B5044641F0E00004F0F8FA04F07F005F
:1068C00004F0F4FAC4F3C610BDE8104004F0EEBAC8
:1068D00038B5134D2B78044641F6FF72A0F50050F1
:1068E000824203F1FF33A8BF02461B0202F50052A9
:1068F00003F47063100443F4604343F00E0300F4A8
:10690000FE005204184302F0FE42104305F0A0FAC4
:10691000296801392046C9B2BDE83840FFF7C8BF31
:10692000389EFF1F38B504460D46F02004F0BEFA2D
:1069300035B1254414F8010B04F0B8FAAC42F9D192
:10694000F720BDE8384004F0B1BA00BF00B50B4BEA
:1069500083B00246998818680090032AADF80410A5
:1069600002D903B05DF804FB684606218DF80520C6
:10697000FFF7D8FF03B05DF804FB00BF5CFC00002C
:1069800000B50B4B024683B0186899880090131F1E
:106990004C2BADF8041002D903B05DF804FB684637
:1069A00006218DF80520FFF7BDFF03B05DF804FB5D
:1069B00064FC0000030203F4FE43C0F3C610184356
:1069C000704700BF03784078DB0103F47E5300F08A
:1069D0007F001843704700BF82B002AA114642F8F8
:1069E000040D002012F8013B03F07F03914243EABB
:1069F0000020F7D102B07047003210B403884FF086
:106A0000010404FA01F418BF012202FA01F123EA99
:106A100004020A43028010BC704700BF70B5CEB2BA
:106A20000C46054603F074FC864203D031462846E6
:106A300003F088FC0135284603F06AFC240A8442EE
:106A400005D021462846BDE8704003F07BBC70BDF0
:106A500038B5054603F05CFC4FF0000460F3070412
:106A6000681C03F055FC60F30F24A0B238BD00BFD2
:106A7000F8B504460020FFF7EBFF002C00F0098179
:106A80004FF4AF610220FFF7C9FF04204FF47A6191
:106A9000FFF7C4FF0B2004F073F8002840F0F884DF
:106AA0004FF496610620FFF7B9FF4FF4FA61082012
:106AB000FFF7B4FF4FF4AF610A20FFF7AFFF40F6D6
:106AC000FC010C20FFF7AAFF4FF496612220FFF78C
:106AD000A5FF4FF416612420FFF7A0FF7D212A2097
:106AE000FFF79CFF0C210E20FFF798FF01211020DB
:106AF000FFF794FF02211220FFF790FF00211420DE
:106B0000FFF78CFF00211620FFF788FF02211820D5
:106B1000FFF784FF01211A20FFF780FF02211C20CC
:106B2000FFF77CFF04211E20FFF778FF14212020AF
:106B3000FFF774FF01212620FFF770FF03212820B3
:106B4000FFF76CFF04212C20FFF768FF0F212E2098
:106B5000FFF764FF00213020FFF760FF0C21322097
:106B6000FFF75CFF00213420FFF758FF002136209B
:106B7000FFF754FF00213820FFF750FF00213A2093
:106B8000FFF74CFF00213C20FFF748FF00213E208B
:106B9000FFF744FF00214020FFF740FF0021422083
:106BA000FFF73CFF1F214420FFF738FF1321462049
:106BB000FFF734FF0E214820FFF730FF11214A2054
:106BC000FFF72CFF0A214C20FFF728FF00214E2061
:106BD000FFF724FF06215020FFF720FF022152205B
:106BE000FFF71CFF0C215420FFF718FF002156204F
:106BF000FFF714FF00215820FFF710FF01215A2052
:106C0000FFF70CFF03215C20FFF708FF0A215E203D
:106C1000FFF704FF00216020FFF700FF042162203E
:106C2000FFF7FCFE01216420FFF7F8FE002166203B
:106C3000FFF7F4FE0B216820FFF7F0FE7F216A20AA
:106C4000FFF7ECFE00216C20FFF7E8FE00216E202C
:106C5000FFF7E4FE00217020FFF7E0FE0021722024
:106C6000FFF7DCFE00217420FFF7D8FE232100206F
:106C7000FFF7D4FE0220FFF7EBFEB0F5805F03467E
:106C800016D34FF4AF610220FFF7C8FE4FF4AF6395
:106C90000EE04FF6FF7398423FF4F2AE232840F027
:106CA00003840220FFF7D4FEB0F5805F0346E8D2EC
:106CB000D24A04201380FFF7CBFEB0F5805F034675
:106CC00080F0D282CE4A06201380FFF7C1FEA0F5E5
:106CD0002F739BB2B3F57A6F024606D940F628218E
:106CE0000620FFF79BFE40F62822C64B08201A809C
:106CF000FFF7AEFEA0F52F739BB2B3F57A6F024695
:106D000006D940F6E4410820FFF788FE40F6E44249
:106D1000BD4B0A201A80FFF79BFEA0F5FA739BB2C9
:106D200040F6AC518B42024606D94FF4AF610A20BF
:106D3000FFF774FE4FF4AF62B44B0C201A80FFF7DC
:106D400087FEA0F5FA739BB240F6AC518B42024627
:106D500006D940F6FC010C20FFF760FE40F6FC026D
:106D6000AB4B0E201A80FFF773FE1828034600F283
:106D70009582A84A10201380FFF76AFE431E9BB23B
:106D80000F2B024604D901211020FFF747FE0122F4
:106D9000A14B12201A80FFF75BFE0A28034600F27F
:106DA00077829E4A14201380FFF752FE0128034683
:106DB00004D900211420FFF731FE0023984A162041
:106DC0001380FFF745FE7F28034600F25B82954A59
:106DD00018201380FFF73CFE0428034600F24C8283
:106DE000914A1A201380FFF733FE0C28034600F265
:106DF000E5828E4A1C201380FFF72AFE04280346F2
:106E000000F2D6828A4A1E201380FFF721FE09284D
:106E1000034600F2C782874A20201380FFF718FE3E
:106E20004628034600F2B882834A22201380FFF7E7
:106E30000FFEA0F5FA739BB240F6AC518B420246AE
:106E400006D94FF496612220FFF7E8FD4FF49662D1
:106E50007A4B24201A80FFF7FBFDA0F5FA739BB252
:106E600040F6AC518B42024606D94FF416612420FD
:106E7000FFF7D4FD4FF41662714B26201A80FFF7FE
:106E8000E7FD7F28034600F281826E4A28201380A6
:106E9000FFF7DEFD0628034600F272826A4A2A20C6
:106EA0001380FFF7D5FDA0F132039BB2B3F5967FB7
:106EB000024604D97D212A20FFF7B0FD7D22634BD5
:106EC0002C201A80FFF7C4FD0C28034600F25282E2
:106ED0005F4A2E201380FFF7BBFD1E28034600F2F9
:106EE00043825C4A30201380FFF7B2FD0928034635
:106EF00000F23482584A32201380FFF7A9FD1E2881
:106F0000034600F22582554A34201380FFF7A0FD86
:106F10007F28034600F21682514C36202380FFF76B
:106F200097FD7F28034600F2078238206380FFF731
:106F30008FFD7F28034600F2F9813A20A380FFF7F6
:106F400087FD7F28034600F2EB813C20E380FFF7BA
:106F50007FFD7F28034600F2DD813E202381FFF77D
:106F600077FD7F28034600F2CF8140206381FFF741
:106F70006FFD7F28034600F2C1814220A381FFF705
:106F800067FD384D28804420FFF762FD3028034616
:106F900000F2AE81344A46201380FFF759FD3028B5
:106FA000034600F29F81314C48202380FFF750FDBB
:106FB0003028034600F290814A206380FFF748FDA5
:106FC0003028034600F282814C20A380FFF740FD69
:106FD0003028034600F274814E20E380FFF738FD2D
:106FE0000128034604D900214E20FFF717FD002396
:106FF0001F4A50201380FFF72BFD3BE05A9CFF1FD8
:10700000849DFF1F109DFF1F569CFF1F6A9DFF1F41
:10701000C89CFF1F3A9DFF1FA69CFF1FEC9BFF1FF4
:10702000E49CFF1F7E9DFF1F909CFF1FF89CFF1F8D
:10703000249DFF1FA29CFF1F829DFF1F2A9DFF1FF3
:10704000929CFF1F149CFF1F849CFF1FCC9CFF1F62
:10705000CE9CFF1FE89CFF1FE89BFF1F5C9CFF1F4F
:10706000D09CFF1F249CFF1F2E9DFF1F549DFF1FC0
:10707000889CFF1F431E9BB20B2B024604D906219E
:107080005020FFF7CBFC0622CF4B52201A80FFF78F
:10709000DFFC0428034600F20D81CC4A5420138003
:1070A000FFF7D6FC431E9BB21D2B024604D90C21D0
:1070B0005420FFF7B3FC0C22C54B56201A80FFF773
:1070C000C7FC0128034604D900215620FFF7A6FC7F
:1070D0000023C04A58201380FFF7BAFC7F280346DC
:1070E00000F2E280BC4A5A201380FFF7B1FC431E35
:1070F0009BB2092B024604D901215A20FFF78EFCCE
:107100000122B64B5C201A80FFF7A2FC431E9BB203
:10711000102B024604D903215C20FFF77FFC0322D9
:10712000AF4B5E201A80FFF793FC431E9BB21D2BD2
:10713000024604D90A215E20FFF770FC0A22A94BFF
:1071400060201A80FFF784FC0228034600F2868044
:10715000A54A64201380FFF77BFC0128034604D96D
:1071600001216420FFF75AFC0123A04A622013800A
:10717000FFF76EFCC31E9BB2012B024604D904210B
:107180006220FFF74BFC0422994B66201A80FFF720
:107190005FFC7F28034600F27581964A68201380C1
:1071A000FFF756FC7F28034600F26681924A6A2068
:1071B0001380FFF74DFC7F28034600F257818F4A6A
:1071C0006C201380FFF744FC0228034600F248813C
:1071D0008B4A6E201380FFF73BFC1928034600F210
:1071E0003981884A70201380FFF732FC0228034659
:1071F00000F22A81844A72201380FFF729FC0628B6
:10720000034600F21B81814A74201380FFF720FCA3
:10721000042800F20D812B88DFF810E27C4F7D4AB4
:107220007D4D7E4E7E4C7F4903F0010CAEF800C0D0
:10723000C3F3400EA7F800E0C3F380071780C3F341
:10724000C007794A2F70C3F30017C3F34015C3F387
:107250008013378025800B801080F8BD00216020CE
:10726000FFF7DCFB002373E74FF47A610420FFF79C
:10727000D5FB4FF47A6325E502211820FFF7CEFBFA
:107280000223ADE500211620FFF7C8FB00239EE591
:1072900002211220FFF7C2FB022382E50C210E20FF
:1072A000FFF7BCFB0C2364E500215820FFF7B6FB79
:1072B000002317E702215220FFF7B0FB0223ECE680
:1072C0000A214C20FFF7AAFB0A2385E611214A2058
:1072D000FFF7A4FB112377E60E214820FFF79EFB62
:1072E0000E2369E613214620FFF798FB13235AE685
:1072F0001F214420FFF792FB1F234BE60021402073
:10730000FFF78CFB002338E600213E20FFF786FBC9
:1073100000232AE600213C20FFF780FB00231CE627
:1073200000213A20FFF77AFB00230EE600213820E7
:10733000FFF774FB002300E600213620FFF76EFB09
:107340000023F2E500213420FFF768FB0023E3E58A
:107350000C213220FFF762FB0C23D4E50021302002
:10736000FFF75CFB0023C5E50F212E20FFF756FB3E
:107370000F23B6E504212C20FFF750FB0423A7E5DB
:1073800003212820FFF74AFB032387E5012126205C
:10739000FFF744FB012378E514212020FFF73EFB93
:1073A000142341E504211E20FFF738FB042332E5B6
:1073B00002211C20FFF732FB022323E501211A20C2
:1073C000FFF72CFB012314E57489FF1FAC89FF1F15
:1073D0009C89FF1F809DFF1FF29CFF1FFA9BFF1FD0
:1073E0007689FF1FA489FF1FEA9BFF1FCA9CFF1F0E
:1073F000C09CFF1FDC9BFF1F0A9CFF1F389CFF1FC8
:10740000F69CFF1F129DFF1F689DFF1F6E9DFF1FB3
:10741000269DFF1F809CFF1F449DFF1FB49CFF1FE4
:10742000209DFF1F289DFF1FBC9CFF1F769DFF1FF7
:1074300074200021FFF7F2FA0020ECE60021722010
:10744000FFF7ECFA0023DEE600217020FFF7E6FAF2
:107450000023CFE600216E20FFF7E0FA0023C0E60C
:1074600000216C20FFF7DAFA0023B1E67F216A20C1
:10747000FFF7D4FA7F23A2E60B216820FFF7CEFAAC
:107480000B2393E600216620FFF7C8FA002384E669
:1074900040F628210620FFF7C1FA40F6E441082013
:1074A000FFF7BCFAFFF706BB17287FF6E9AA1928F1
:1074B0007FF658AB1B287FF675AB1C283FF48AABD0
:1074C0001E287FF68FAB1F283FF494AB20283FF493
:1074D000ADAB21283FF4B6AB22287FF4C7ABFFF752
:1074E000B9BB00BFF8B5872006F0C6FB204B214A88
:1074F000054603CB1368C5F803001A0C7620C5F8BF
:1075000007102B80AA70FFF755FA2E46002426F8A4
:107510000B0FA0B2FFF79CFAFFF74CFA0234762C5F
:1075200026F8020FF5D16C1E05F182064FF0FF30F0
:1075300014F8013F082758400F4B40F300017A1E12
:107540000B4012F0FF0783EA5000F5D1B442EFD1AF
:10755000C043FFF741FA3A46C5F883008721284621
:1075600004F0C4FC2846BDE8F84006F08DBB00BF1F
:1075700070FC00006CFC00002083B8EDF0B50E4BF1
:107580000E4C054693E8070085B024682E88AD7838
:1075900001AB83E80700270C184600220B21ADF849
:1075A00004408DF80670ADF80C608DF80E5004F0B4
:1075B0009DFC05B0F0BD00BF7CFC00006CFC000031
:1075C000F0B5124B124D1E68124F0FCD87B06C46AE
:1075D0000FC495E8030044F8040B38683B79CDF8F4
:1075E0000D00320C232021808DF802208DF81130FF
:1075F000ADF80060FFF7DEF90022ADF80B001221B4
:10760000684604F073FC07B0F0BD00BF6CFC0000DE
:1076100088FC000014F80000002004F0E3BC00BF68
:1076200002F02EBE70B5124C82B0002540230646F3
:1076300029462046009301958023202201F072FE06
:1076400020222946204602F031FA2046012102F08C
:1076500037FA304607F0B4F831460246204602F0C9
:10766000BFFB204602B0BDE8704001F041BC00BF46
:10767000A89DFF1FF0B5862983B075D90546441E25
:1076800000F182064FF0FF3014F8012F0827504018
:10769000404A40F300017B1E0A4013F0FF0782EAD4
:1076A0005000F5D1B442EFD1C043FFF795F9014640
:1076B000D5F883000190019A914202D0B2F17F2F58
:1076C0000BD105F10B00FFF77DF976280BD032487E
:1076D000FFF7A8FF002003B0F0BD3048FFF7A2FF7E
:1076E000384603B0F0BD05F10D00FFF76BF9232814
:1076F00040D1002440F6AC5613E004281AD00628E6
:1077000021D008281FD00A2828D00C2822D1A1F582
:10771000FA7292B2B24201D8FFF780F90234762CA5
:107720000ED004F10D002844FFF74CF9022C01465D
:10773000A0B2E2D1B1F5805FEED30234762CF0D165
:10774000012003B0F0BDA1F52F7292B2B2F57A6FAD
:10775000E4D8E1E7222801D0242811D1A1F5FA725A
:1077600092B2B242DAD8D7E70D48FFF75BFF0020AC
:1077700003B0F0BD0B48FFF755FF002003B0F0BD8C
:107780002A28C9D1A1F1320292B2B2F5967FC5D8AA
:10779000C2E700BF2083B8EDCCFC0000B8FC0000BD
:1077A000A0FC0000E0FC000003290CD970B5461CC9
:1077B00082B005460C46304603222A4907F06EF88F
:1077C00010B102B070BD70470B2C05D905222649B7
:1077D000281D07F063F840B12448FFF723FF244831
:1077E00002B0BDE87040FFF7C9BE05F109010322F0
:1077F00001A807F0A3F801A803221E4907F04EF8DC
:10780000D8B103221C4901A807F048F808B301A821
:1078100003221A4907F042F8B0B91948FFF702FFEE
:10782000A11E89B23046FFF725FF0028C9D01548B0
:1078300002B0BDE87040FFF7F5BE1348FFF7F2FE57
:10784000FFF750FE1148F3E71148FFF7EBFE114830
:10785000C6E71148FFF7E6FE02B0BDE87040FFF74B
:10786000AFBE00BF6CFC000024F80000F8FC000074
:107870000CFD000010FD000038FD000050FD000070
:1078800054FD000068FD000014FD000028FD00000C
:107890007CFD000090FD00003CFD00002DE9F04360
:1078A000174D2B6883B081460F469046F3B1154EB5
:1078B00034880A1992B218461146328006F05AFDF1
:1078C00028603A464946204402F06CFDB8F1000FAA
:1078D00009D031882868FFF767FF286806F0D4F9D7
:1078E00000232B60338003B0BDE8F083054E019385
:1078F0000846318006F0C0F9019B28601C46E0E78D
:10790000409EFF1F3C9EFF1F10B51F4C4FF4FA70A6
:10791000FCF768FB204601F0DFF900221146204603
:1079200002F0C4F82046012102F0CAF820460021E6
:1079300002F0C0F80B221549204602F051FA204609
:1079400002F064FA0F221249204602F049FA20465A
:1079500002F05CFA0F490722204602F041FA204665
:1079600002F054FA204601F0C3FA0B4B0B4A1A609E
:107970004FF4FA70FCF736FBFFF722FE0848BDE82B
:107980001040FFF74FBE00BFA89DFF1F94FD0000F1
:10799000A0FD0000B0FD0000F89FFF1F9D780000D3
:1079A000B8FD00000020704790F8392090F83800AA
:1079B000101A704790F8383090F839209A4205D95B
:1079C0005A1C034480F83820187E70474FF0FF306F
:1079D000704700BF90F8383090F839209A4286BF3F
:1079E0001B18187E4FF0FF30704700BF704700BF74
:1079F00038B50546B0F85E0090B195F85D30144694
:107A0000C3F1210294420CD805F13B0018442246F0
:107A100002F0C8FC95F85D30234485F85D302046BF
:107A200038BD012014462871EEE700BFB0F85E3083
:107A30006BB190F85D30202B07D8C218013380F865
:107A40005D30012082F83B10704701230371002054
:107A5000704700BF0023426980F8383080F8393021
:107A600080F85C3080F85D3080F85E3080F85F3000
:107A700006CA30B40D68046943662A4383660A6007
:107A8000A370426990F861301649146813441D7A56
:107A90005B7B01EBC5051B026D6803F4E06343F0FB
:107AA00064032B6090F8623013449D7CDB7D01EB16
:107AB000C5011B02496803F4E06343F064030B60F3
:107AC00021685368194205D0036927225A70036957
:107AD00004229A71036920225A71036980229A70E4
:107AE00030BC7047EC08010043690CCB12681A42A5
:107AF0000CD0094B99420AD9084B9942036994BFAB
:107B00001A220D225A70036904229A717047036980
:107B100027225A70F7E700BF7F1A06003F420F0086
:107B200010B50269D378DBB2D90604463DD51021E1
:107B30005806D17038D503F0040303F0FF02002B80
:107B400051D03D49626E00230B7084F85D30002AED
:107B50005BD0904794F85D30002B56D02369D0223B
:107B60009A70236994F83B201A712369012284F8E2
:107B70005C200222DA7010BD304B84F860009C4219
:107B80004AD02F4B9C4252D094F8391013791F29B8
:107B9000DBB207D82848007820B16018013184F89A
:107BA000391003760223D37010BD5906C3D49178DF
:107BB00001F0100101F0FF000029DDD013F00103F6
:107BC0001ED194F85C1094F85D00884281BF4B1C74
:107BD000091984F85C3091F83B3013712369D02285
:107BE0009A702269DEE7236984F83920C0229A70EE
:107BF0002369114A1979012111700222DA7010BD2E
:107C0000C023937022691379CCE70122002384F802
:107C10005D2084F83B30A1E7626994F8613009493E
:107C200013440322187A02F043FD2269ACE762692B
:107C300094F861300449F3E7449EFF1FFC8FFF1F57
:107C40006890FF1FA97C0000B57C00000369DB7809
:107C500003F0200373B190F860300133DBB2012BE5
:107C600080F860301AD9426990F861301344187A6C
:107C700002F09ABD70B5426903F0FF0590F86130DB
:107C800013440446187A02F08FFDA36E5BB184F8AA
:107C9000385094F83900BDE87040184790F85F30CC
:107CA000002BE0D0704770BD0148FFF7CFBF00BF89
:107CB000FC8FFF1F0148FFF7C9BF00BF6890FF1F7F
:107CC0002DE9F047374FDFF8E0903B68026982B05A
:107CD00006460093DDF800800021A025D3789B069E
:107CE0005BD53B680193019BC8EB03030F2BF5D9D0
:107CF00049B1102BF2D000209070336980229A7025
:107D000002B0BDE8F087726996F86130134405212E
:107D1000187A02F043FF726996F86130134401212A
:107D200093F812A0504602F039FF09240021504672
:107D300002F020FF2B46013BFDD10121504602F00D
:107D400019FF2B46013BFDD1013CEFD1706996F83C
:107D5000611001444FF4A0720C7A4B7B09EBC40113
:107D60001B02496803F4E06343F064030B6096F878
:107D700062300344997CDB7D09EBC1011B02496839
:107D800003F4E06343F064030B60013AFDD1326910
:107D9000D3789B064FF00101A3D4012002B0BDE8C7
:107DA000F08700BF6C9EFF1FEC080100F0B503696F
:107DB0001222DA700269937803F0200385B004463A
:107DC0000D46002B5ED0B42393703C4922690B68AA
:107DD0000093009E05E00B680193019B9B1B042B05
:107DE00042D8D37803F0200303F0FF00002BF2D039
:107DF00094F85D30002B31D04FF0000E4FF0020CA4
:107E000004EB0E0393F83B3013710B680393039F4D
:107E1000206907E09B060DD50B680293029BDB1BD4
:107E2000052B28D8C378DBB203F0020202F0FF066C
:107E3000002AEFD080F803C02669F378DBB2DF06B2
:107E400032462DD49F062BD5DB0731D40EF1010E1F
:107E500094F85D305FFA8EFE7345D1D800201DBBCB
:107E6000002384F85E3004E09070236980229A70C9
:107E7000042005B0F0BD86702369802204209A702A
:107E800005B0F0BD03F0FF06FFF71AFF10B904209C
:107E900005B0F0BD236984F85F60B0229A7094E762
:107EA0008023B3700420DAE726698023B370D7E714
:107EB000BEF1000F0CBF02200320F6E76C9EFF1FEF
:107EC0002DE9F04106690025122780F8385080F826
:107ED0003950F770D0F810C09CF802E00EF0200E78
:107EE00088B00446884615461E46BEF1000F49D0AC
:107EF000B4238CF80230784B21691A680092DDF8BF
:107F000000E006E01A6801920198CEEB0000042818
:107F100030D8C87800F0200000F0FF070028F1D02A
:107F20004FEA480242F00102D2B20A711A68029284
:107F3000DDF808E0206906E01A6803920399CEEBA9
:107F4000010105292AD8C17801F0020101F0FF07DB
:107F50000029F1D04FF0020C80F803C02269D178DB
:107F600011F0110722D12DBB002E0CBFA0238023BE
:107F7000937003E08F70236980229A70384608B0AE
:107F8000BDE8F0810EF0FF07FFF79AFE0028F5D05C
:107F9000236984F85F70B0229A70ACE78770236918
:107FA000802238469A7008B0BDE8F0818023937033
:107FB0000027E3E7012D75D0A021917021690A798E
:107FC000BE4667464FF0A80C1A680492049805E074
:107FD0001A680592059A121A052A4AD8CA7802F038
:107FE000020202F0FF08002AF2D0CF702169CA789D
:107FF000D2B212F0100F08465AD1920658D5013D60
:10800000EDB2012D49D0BEF11F0F3BD90A79012DE8
:10801000DAD11A680692069D05E01A680792079A57
:10802000521B052A46D8C27802F0020202F0FF0174
:10803000002AF2D00223C3702269D378DBB2D906BA
:108040003AD49B0634D5B023BEF11F0F93703FD8AE
:10805000226904EB0E0312791A760EF1010E5FFA13
:108060008EFE16B1236980229A7084F839E0774633
:1080700084E781F80280236980229A70774684F829
:1080800039E07BE704EB0E0291F8048082F8188057
:108090000EF1010E5FFA8EFEB9E781F802C0216988
:1080A0000846B0E7A82191702069BE460279B0E782
:1080B000774663E78170DEE71021A023D170013B92
:1080C000FDD12269937803F0F7037746937055E763
:1080D00023691B79C5E700BF6C9EFF1F0148FFF7AE
:1080E0001FBD00BFFC8FFF1F0148FFF719BD00BF78
:1080F0006890FF1F704700BF38B5144C0378012209
:108100005B000546204684F83B3084F85E2084F806
:108110005D20FFF78BFC20460021FFF747FE0B4C4C
:108120002978012320461A46FFF7CAFE0128F6D116
:1081300094F8383094F839209A4205D9E21801337E
:1081400084F83830107E38BDFF2038BDFC8FFF1F0B
:1081500038B51B4C037801225B000546204684F8A5
:108160003B3084F85E2084F85D20FFF75FFC2046FA
:108170000021FFF71BFE124C297820460123022222
:10818000FFF79EFE0228F6D194F8382094F83910B3
:108190008A420FD2531CDBB2A018994284F83830BF
:1081A000007E0AD9234402321B7E84F8382040EA3C
:1081B000032038BD4FF6FF7038BD40F47F4038BD16
:1081C000FC8FFF1F0C2901D90020704702314900A4
:1081D00001F0FE01FFF7BCBF70B50C4C03781646EA
:1081E00001255B00204684F83B3084F85E5084F81B
:1081F0005D50FFF71BFC31462046FFF717FC294670
:108200002046BDE87040FFF7D1BD00BFFC8FFF1FC7
:10821000F8B505460F461646412421463A462846FB
:10822000FFF7DAFF611C0234C9B232462846E4B2D5
:10823000FFF7D2FF592CF0D1F8BD00BF38B5044686
:108240000D463548FFF706FC632280212046257045
:10825000FFF7C2FF012002F0C9FC204600225E2188
:10826000FFF7BAFF20465D21FFF746FF242801D023
:10827000002038BD204606220C21FFF7C9FF20460A
:1082800001222B21FFF7A8FF204601222C21FFF716
:10829000A3FF20460E222D21FFF79EFF204600223D
:1082A0002E21FFF799FF204601222F21FFF794FF8F
:1082B000204605223021FFF78FFF20460122312181
:1082C000FFF78AFF204600223221FFF785FF204674
:1082D00000223321FFF780FF204600223421FFF7E0
:1082E0007BFF204600223521FFF776FF2046002243
:1082F0005B21FFF771FF204610225C21FFF76CFF26
:10830000204620225D21FFF767FF20468F225E2155
:10831000FFF762FF012038BDFC8FFF1F10B4047F00
:108320004160022CC26002D010BC01F0D7BB836850
:1083300010BC184790E80C00F0B41C685968256818
:10834000164F174E29432160164D17491760D66006
:1083500015611160417A154A5C180A3194F824407D
:1083600053F8215002EBC40149680D60017A5C1892
:1083700003EB8101247ECD6902EBC40149680D60E5
:10838000817A581803EB810390F83000596B02EBA7
:10839000C002F0BC53681960704700BF01401F0065
:1083A000011000380110007800001F80EC08010067
:1083B000704700BFF0B50C1EBDF8146034DBB0F997
:1083C00006701919B942C4BF3B1B1BB2002BA6464D
:1083D0001CDD002A1146B8BFD11D02F00705CC10E4
:1083E000826A012007FB04E1A840012E0A44C0B2C2
:1083F0001ED00CD3022E09D1013B12FA83F3013AAD
:1084000012F8011F41409A421170F9D1F0BDC043EA
:10841000013B12FA83F3C0B2013A12F8011F014086
:1084200093421170F9D1F0BD23441BB20024C6E77A
:10843000013B12FA83F3013A12F8011F01439A42F9
:108440001170F9D1F0BD00BFF8B50D1E0EDB14465A
:108450001F46064601F03AFBA84207DD002C05DB6B
:10846000304601F037FBA04201DCF8BDF8BD3046D4
:1084700001F02AFB022853D003284BD0012806D153
:108480006540F3886C406540013B5D1B2DB2012FB8
:1084900003D02AD3022F14D0F8BD002C2246B6F9FF
:1084A0000630B06AB8BFE21D42F3CF0202FB0355AB
:1084B00004F00704435D012101FA04F41C43445510
:1084C000F8BD002C2246B6F90630B06AB8BFE21DEE
:1084D00042F3CF0202FB035504F00704435D012180
:1084E00001FA04F45C404455F8BD002C2246B6F96C
:1084F0000630B06AB8BFE21D42F3CF0202FB03555B
:1085000004F00704435D012101FA04F423EA0404A2
:108510004455F8BD3389013B591B25460CB2B6E7DB
:10852000F18832890139013A4D1B141B2DB224B256
:10853000ADE700BF2DE9F041079E9DF91880089D29
:1085400004461F4600F0C0FF0D4B0E480E4984F84C
:108550003380FF22002F08BF1F4684F82F200023FE
:1085600084F8302084F8312084F832202060A66519
:10857000E565676261652362A3622046BDE8F0811C
:10858000FC8FFF1F44FE00000110013810B50446A7
:10859000806A034B236008B105F076FB204610BDCE
:1085A00044FE0000F8B5436ADBB190F82C200125A9
:1085B000AA4083F83B2083F85E5083F85D50044660
:1085C000406A03680E461B6800219847606A03688A
:1085D00031461B6898472946606ABDE8F840FFF7B6
:1085E000E5BBC26BC56C1368046A23EA050313601C
:1085F0004CB122684FF00043D3625163D36A002B21
:10860000FCDA936BF8BD836B466B0825802410E081
:108610003768426C3A4332601F68826C3A431A6092
:108620001A68876C013D22EA07024FEA54041A6077
:1086300007D02142ECD13268476C22EA070232604F
:10864000EAE7F8BD70B50446406A0D4600282BD015
:10865000A16DFFF749FA002D20460CBFA621A721E6
:10866000FFF7A0FF606A20B1E16DBDE87040FFF741
:108670003BBA216C226D0868236A02430A6093B1F9
:10868000DA7A82B1D00703D5224A99691160DA7A81
:10869000910703D5204AD9691160DA7A520702D5C9
:1086A0001E4A1B6A136070BD236A002B2BD0D97A37
:1086B000626DE1B172B6D97ACE0706D51848D9688D
:1086C0000668314099610160D97A880706D5154856
:1086D000196906683140D9610160D97A4E0705D51C
:1086E00011485969066831401962016062B61B6819
:1086F000D968914207D00D4818600D49DA6042F000
:10870000804018611960226C216D136823EA01030F
:108710001360A0E700E100E004E100E008E100E010
:1087200080E100E084E100E088E100E001403F00FA
:1087300000003F80436A2DE9F04105460E46904611
:10874000002B3ED090F82C100124A14083F83B1060
:1087500083F85E4083F85D40406A036800211B682F
:1087600008F1FF379847FFB2B8F1000F23D0374424
:10877000A046013E686A16F8011F03681B68984707
:108780000134B742E4B216D0202CF3D10121686A3B
:10879000FFF70CFB95F82C206B6A520083F83B2006
:1087A00083F85E8083F85D80686A036800211B6837
:1087B00098470124DEE7686A0121BDE8F041FFF730
:1087C000F5BAC26BC16C136823EA010306EB080417
:1087D00013604FF00048A6420ED02B6A16F801EB4A
:1087E00063B11A68C2F82C80C2F834E0D36A002B57
:1087F000FCDAA642936BF0D1BDE8F081AB6BD5F803
:1088000034C008208021DCF800206F6C1EEA010FC4
:1088100014BF3A43BA43CCF800201A68AF6C3A430D
:108820001A601A68AF6C013822EA07024FEA510158
:108830001A60E8D1CFE700BF70B50446406A0D4624
:10884000002828D0A16DFFF74FF920462946FFF7F1
:10885000A9FE606A20B1E16DBDE87040FFF744B940
:10886000216C226D0868236A02430A6093B1DA7AA8
:1088700082B1D00703D5234A99691160DA7A91074A
:1088800003D5214AD9691160DA7A520702D51F4A05
:108890001B6A136070BD236A002B2BD0D97A626DDE
:1088A000E1B172B6D97ACE0706D51948D9680668FB
:1088B000314099610160D97A880706D51548196950
:1088C00006683140D9610160D97A4E0705D5124852
:1088D0005969066831401962016062B61B68D9683F
:1088E000914207D00D4818600D49DA6042F080408F
:1088F00018611960226C216D136823EA010313606B
:10890000A3E700BF00E100E004E100E008E100E0CF
:1089100080E100E084E100E088E100E001403F0008
:1089200000003F802DE9F041044686B0806A9DF842
:1089300030801E460F461546B4F90830002800F076
:108940004281DA1D48BF03F10E02B4F90630D2109D
:1089500003FB02F2002105F0BBFCB4F90820202A39
:1089600000F39280B4F90610A34B0120203A73392A
:1089700002EBD27201EBD1714FF0200E0290732006
:108980008DE8014042F34F0241F34F01204600F0D1
:1089900051FE606A84F82D70002800F04D81002D92
:1089A00040F08A80B4F90830202B14BF3D253C25C7
:1089B00084F82C50B8F1000F40F0858006B394F98C
:1089C0003300002818DBC0B2012102F0E7F80121D2
:1089D00094F8330002F0CEF8012002F007F90021EC
:1089E00094F8330002F0C6F80A2002F0FFF80121E3
:1089F00094F8330002F0BEF8606A002800F082802C
:108A0000A16DFFF771F804227C492046FFF792FE22
:108A1000217A0139C9B22046FFF7C4FD7849042202
:108A20002046FFF787FE94F92D30012B14BF142147
:108A300010212046FFF7B6FD042272492046FFF7B9
:108A400079FEB4F90630802B00F09280602B00F0A4
:108A5000A680D9212046FFF7A5FD94F92D30012BE2
:108A600014BFF12122212046FFF79CFD204606225B
:108A70006549FFF75FFE606A50B3E16DFFF734F8B8
:108A8000012006B0BDE8F081B4F906105F4B01206B
:108A9000403A52394FF0400E029002EBD27252200F
:108AA00001EBD1718DE8014042F34F0241F34F01D8
:108AB000204600F0BFFD6CE76DB284F82C50B8F191
:108AC000000F3FF47BAFFEF7C5FF002E94D076E792
:108AD000216C226D0868236A02430A6073B1DA7A56
:108AE00062B1D00703D54A4A99691160DA7A9107D1
:108AF0007CD4520702D5474A1B6A1360012006B096
:108B0000BDE8F081236A002B2BD0D97A626DE1B1E8
:108B100072B6D97ACF0706D53F48D968056829408B
:108B200099610160D97A8E0706D53C4819690568B4
:108B30002940D9610160D97A4D0705D5384859696E
:108B4000056829401962016062B61B68D9689142C4
:108B500007D0344818603449DA6042F08040186128
:108B60001960226C216D136823EA010313604AE740
:108B7000B4F90830202B00F08680402B7FF469AFD9
:108B80002A4920460322FFF7D5FD94F92D30012B09
:108B900014BFCF219F212046FFF704FD59E7B4F908
:108BA0000830102B7FF455AF214920460322FFF7F0
:108BB000C1FD94F92D30012B14BFAF2110212046A7
:108BC000FFF7F0FC45E7DA1D48BF03F10E02B4F9E8
:108BD0000630D21003FB02F21046059205F04CF865
:108BE000A06200283FF44DAF059AB3E6114AD96957
:108BF0001160DA7A7DE700BF9CFE00007C00010076
:108C00008000010084000100880001009000010044
:108C100000E100E008E100E080E100E084E100E044
:108C200088E100E001403F0000003F8098FE000026
:108C30005003010004E100E0012194F83100244FC9
:108C400001F0ACFF94F83200012101F0A7FF94F984
:108C5000312094F9323057F83220E26357F833303C
:108C6000206A23640125E56425651A682A431A6091
:108C700078B1B8F1000F3FF428AFFFF75BFB002E8F
:108C80003FF4BAAE9BE6042212492046FFF752FD9C
:108C9000DFE6294694F82F0001F080FF294694F87A
:108CA000300001F07BFF94F92F2094F9303057F811
:108CB0003220626357F833306564A5641A68A36391
:108CC00022F001021A60002E3FF496AE77E600BF54
:108CD000EC08010094FE0000B0F90820D31D48BF45
:108CE00002F10E03B0F90620806ADB1002FB03F2EA
:108CF000002105F0EDBA00BFF0B50029BDF8145011
:108D00002EDBB0F90660B1422ADA002A59DBB0F94D
:108D1000087014461C44BC42C4BFBB1A1BB2002BD3
:108D20001EDDD2B2D408D0F828E016FB041112F0F0
:108D30000702DBB20EEB010421D0C2F10807FAB240
:108D4000374F9342BF5C0CD2C3EB020CFF2646FAAE
:108D50000CF6012D07EA06073FD005D3022D36D0C9
:108D6000F0BD012D39D030D21EF8016026EA070788
:108D70000EF801709342F3D3B0F906100C449A1A1E
:108D8000D2B2072A10D9022D36D0002D14BFFF26EB
:108D9000002613462670083BB0F90610DBB2072BFD
:108DA0000C44F7D802F00702002AD9D01D4B012D40
:108DB0009B5C1DD017D3022DD2D122785340237053
:108DC000F0BD13441BB20022A1E7022D25D11EF8ED
:108DD000016077400EF80170CCE71EF80160374360
:108DE0000EF80170C6E7227822EA03032370F0BD73
:108DF000227813432370F0BD11462378DB432370A0
:108E00000839B0F90630C9B207291C44F5D812F068
:108E10000702A5D0034B9B5CCFE73444AFE700BF0C
:108E200034FE000024FE000070B4C47DBDF80C5078
:108E3000022C18D0032C1FD0012C0BD0002A03DBEE
:108E4000B0F90840944201DC70BC7047039570BCD7
:108E5000FFF7B0BAC4880395013CA41A0A4621B2B0
:108E600070BCFFF749BF0689C488013E641AB21A74
:108E7000E41A12B221B2E1E704890395E41A641AF4
:108E8000114622B270BCFFF737BF00BF70B4C57D7A
:108E9000BDF80C60022D1AD0032D12D0012D03D085
:108EA000039670BCFFF728BFC488E41AA41A0A46C8
:108EB00021B2002A03DBB0F90840944213DC70BCF5
:108EC00070470489013C641A114622B2F1E7C48854
:108ED00005890396013CAD1AED1A621A11B22AB245
:108EE00070BCFFF709BF039670BCFFF763BA00BF01
:108EF0002DE9F8430446406A002863D0A16DFEF7CF
:108F0000F3FD052274492046FFF714FCA1790139CD
:108F1000C9B22046FFF746FBB4F90820E588A66AE7
:108F2000D31D48BF02F10E03DB10626A15FB03F587
:108F30001FFA85F8002A7BD094F82C300125AB402D
:108F400082F83B3082F85E5082F85D50606A0368B8
:108F500040211B6808F1FF379847BFB2B8F1000FF6
:108F600023D03744A846013E606A16F8011F036803
:108F70001B6898470135B742EDB216D0202DF3D1CA
:108F80000121606AFEF712FF94F82C20636A5200F8
:108F900083F83B2083F85E8083F85D80606A036815
:108FA00040211B6898470125DEE70121606AFEF732
:108FB000FDFE606A002800F08D80E16DBDE8F84399
:108FC000FEF792BD236A002B2BD0D97A626DE1B1F6
:108FD00072B6D97ACE0706D54048D96805682940C7
:108FE00099610160D97A8D0706D53D4819690568F0
:108FF0002940D9610160D97A480705D539485969AE
:10900000056829401962016062B61B68D9689142FF
:1090100007D0354818603549DA6042F08040186161
:109020001960226C216D136823EA0103136068E75D
:10903000E26BE36C1168276A0B4306EB08091360C7
:109040004FF0004E4E450DD016F801CB2FB33A68C5
:10905000C2F82CE0C2F834C0D36A002BFCDA4E45CB
:10906000936BF1D1226C236D11680B43136097B1A0
:10907000FB7A83B1D90703D51D4BBA691A60FB7A15
:109080009A0703D51B4BFA691A60FB7A5B0702D576
:10909000194B3A6A1A60BDE8F883A36BD4F83480A0
:1090A00008208021D8F80020656C1CEA010F14BF4D
:1090B0002A43AA43C8F800201A68A56C2A431A60FC
:1090C0001A68A56C013822EA05024FEA51011A60BC
:1090D000E8D1B7E7276AC5E72CFE000080E100E091
:1090E00084E100E088E100E001403F0000003F80B3
:1090F00000E100E004E100E008E100E02DE9F04FCC
:1091000085B09946BDF93870BDF83CA0BB1AC1EBDB
:10911000090B002BB8BF5B42BBF1000FB8BFCBF10E
:10912000000B5B450D4616460093804648DC4D45D6
:109130003A4633464CDC194613460A46C5EB09014C
:109140009B1A89B2002B0CB2B8BF5B4204EBD474FB
:10915000BE42ACBF4FF0FF3201224D450391029257
:109160004FEA640429DC9BB201930DE0D8F800704B
:10917000BF69B847019BE41AA3B21CB20135002CA9
:109180002DB211DBA94518DB009B5B452A465346EF
:1091900031464046EADCD8F8002053469769294614
:1091A00032464046B847E5E7029A1644039AA94575
:1091B00002EB030436B224B2E6DA05B0BDE8F08F64
:1091C0004A462B46B94635464D4517461E46B2DD42
:1091D000304629463E464D4607468946AEE700BF23
:1091E00010B404682469A44610BC604730B4046815
:1091F000BDF808500295A46BA44630BC604700BF80
:1092000030B40468BDF808500295E46BA44630BC45
:10921000604700BF70B40468BDF90C60BDF8105021
:1092200003960495246CA44670BC6047704700BF49
:1092300010B582B0B0F90C200191016800920022B3
:109240000C6CB0F90A301146A04702B010BD00BF47
:10925000704700BF01F003010129C17506D0032941
:1092600004D0C28803894281838170470289C38800
:1092700042818381704700BF2DE9F0410568134E9C
:109280006F6986B0B7420446BDF8308010D1013B0B
:1092900013441BB20093CDF804800B46AD6A204600
:1092A000A8472368DB6AB3420AD106B0BDE8F08163
:1092B000059304920391B84703A925680EC9E6E710
:1092C000204606B0BDE8F041184700BF2D920000CF
:1092D0002DE9F0410568124E6F6986B0B742044629
:1092E000BDF830800FD1013BCDF804800B440092D3
:1092F0001BB2AD6A2046A8472368DB6AB3420AD195
:1093000006B0BDE8F081059304920391B84703A924
:1093100025680EC9E7E7204606B0BDE8F0411847CA
:109320002D9200002DE9F04F0568DFF858B06F6905
:1093300085B05F450646BDF93890BDF83CA00C46A7
:10934000904615D11F19BC420CDACDF800A0214679
:1093500001342D6A4B464246304624B2A847BC42EF
:109360003568F2DBEB6A5B4507D105B0BDE8F08FED
:109370000393B8473568039BE4E7304605B0BDE882
:10938000F04F18472D9200002DE9F04387B0994225
:109390000546BDF93840BDF83C6025D0A24212D048
:1093A0000768DFF88080D7F81490C14532D18DE886
:1093B00050002846BC6AA0472B68DB6A434524D18D
:1093C00007B0BDE8F083994202DD0846194603461E
:1093D00028680E96C46B01335B1A1BB22846A4465C
:1093E00007B0BDE8F0436047A24202DD13462246C3
:1093F0001C4628680E96631C846B9B1A1BB2284679
:10940000A44607B0BDE8F0436047284607B0BDE872
:10941000F0431847059304920391C84703A92F68A6
:109420000EC9C4E72D9200002DE9F04FD0F800E0FE
:10943000DFF89090DEF814B083B0CB450446BDF958
:109440003080BDF834A00D4617461E4631D1CDF808
:1094500000A0DEF824B0294633463A462046D847D5
:109460002368CDF800A008F1FF323A44D3F824B0C5
:10947000294612B233462046D8472368CDF800A0CB
:109480002946D3F820B03A4643462046D8472068BC
:10949000CDF800A0711E29444346056A09B23A4638
:1094A0002046A8472368DB6A4B4506D103B0BDE8D8
:1094B000F08FD847D4F800E0C9E7204603B0BDE8F4
:1094C000F04F18472D920000F0B4002401264FF60B
:1094D000FF75094F07600471C475C4810482447626
:1094E000C4618675067685824582C180028141818C
:1094F0008281F0BC704700BF5C0301002DE9F04F92
:1095000085B00668BDF84450BDF93880CDF80080BC
:1095100004460195D6F848B00392BDF93C60BDF908
:10952000407089469A46D84723680195009742467D
:109530005146D3F8488020463346C0472068039BF5
:109540000E930F95856C4B463A4631462046AC4605
:1095500005B0BDE8F04F60472DE9F04F87B01746E2
:10956000BDF9404000912546E91D059344BF2B46B7
:1095700003F10E010268BDF8486053690294C910F6
:1095800003912B49BDF9444001968B42824645D157
:10959000002C3CDD029B3C445E1EB6B24FF000093D
:1095A00023B2049301364D46029B002B28DD059B18
:1095B000002403EB090806E0EDB22B0604F10104D8
:1095C00011D4A6421CD0A1B211F0070F23B24FEA6A
:1095D0004505F1D1002BB8BF0733DB10013418F873
:1095E00003502B06EDD5009BD2F818B019443A462B
:1095F00009B2019B5046D847A642DAF80020E2D1D2
:10960000039B01379944049B3FB2BB42CCD1D36A40
:10961000074A934206D107B0BDE8F08F9847DAF8C1
:109620000020B5E7504607B0BDE8F04F184700BF2F
:109630002D92000070B4BDF90C60BDF91050BDF85A
:10964000144003960495059470BCFFF785BF00BFD6
:109650002DE9F04F93B090460591C1691090BDF887
:1096600070000790BDF874909DF878A004930029CD
:1096700000F0CD800A7A0AC9894604998A1AD2B2C2
:1096800003EBC203BAF1010FDA780B9293F90520CC
:109690001E8893F802B00F9293F9064079D913B25D
:1096A000099323B20C93109B1A68A94B1193194686
:1096B00053698B4240F0A6800B9B002B55D01FFABC
:1096C00088F300210D93C8462344DDF840900691AD
:1096D0000E930F460C46BBF1000F3FD0BDF818109B
:1096E0000C9B03971FFA8AF0CB1813FB00F304902E
:1096F0000E9801440D98034409B21BB20A910893D5
:10970000002505E00135EBB264009B45E4B222D9A7
:10971000039B2B44590703D1731C18F806409EB2D3
:109720002306EFD5099BBDF81000E91811FB00F1E5
:109730000598BAF1010F0FFA8AF301441CD007987B
:1097400001900093D26909B217464846089AB84773
:10975000D9F80020D6E7039F5F44FFB2069B0B9920
:1097600001330693DBB29942B5D8D36A119A93427A
:1097700043D113B0BDE8F08F0F9B191893690A9A73
:1097800029441F4609B2079B4846B847D9F800202C
:10979000B8E700230C93099385E70A9A0D9B0132E1
:1097A000013B52B213F0FF030A920D936FD1DDF823
:1097B0001890079BDDF83C80DDF820A04B4517D0C2
:1097C000BAF1010F00F0C8800B9A109DCDF80490FB
:1097D0000BEB8B014FEACB030A4400931146DEF8F2
:1097E0001C405346424609B22846A047D5F800E03F
:1097F000DEF82C30119A9342BBD0109813B0BDE81C
:10980000F04F1847109D284698472A6854E7109A49
:109810000598B2F90A308342ABDDB2F90C3043450A
:10982000A7DD062313FB0A03002BA2DD08EBCA0306
:10983000002B9EDD537E2BB9049BAF2B02D9013345
:10984000DBB20493109BD3F800E0414B11931A460E
:10985000DEF81430934240F08E801FFA88F30E93A6
:1098600008339BB2BDF81420059305230D93002304
:109870000A93CDF83C800FFA8AF3DDF84080CDF8EA
:1098800018900B921FFA8AFBCDF820A099460A9AED
:10989000BDF810000B9C0E9D0523194611FB0023FB
:1098A0002C481146C75C039702FB0B4214FA81F364
:1098B00012B21BB209920C932C462E461CE0089B58
:1098C0000999012B2AB24B4640462DD0079F01979C
:1098D000CDF80090DEF81CA0D047D8F800E0039B3C
:1098E0005B0801340393059BA4B25D445E44A3422C
:1098F000ADB2B6B23FF451AF039BD807DFD4079B9C
:10990000069A9342EBD0089B012B16D0069B01933D
:10991000CDF80090DEF81CA009994B4632B24046C3
:10992000D047D8F800E0DAE7DEF818A0079B0C99DA
:1099300022B2D047D8F800E0D1E7DEF818A00C99A1
:109940001346404622B2D047D8F800E0C7E700BF30
:109950002D920000AC0301000B99109DCDF80090F2
:109960000531DEF8204009B2424608232846A047C8
:10997000D5F800E03CE7109C20469847D4F800E07A
:109980006BE700BFF0B5C36985B004462BB30A2965
:1099900068D00D294AD01A7A914247D3587A884222
:1099A00044D35D688A1A05EBC205AA78002A50D014
:1099B000E87800284DD0207E00283AD095F905E0BF
:1099C000B4F90E00A67DB4F90A70724406FB0202D7
:1099D000BA4262DCB4F9102030E00A2956D00D29D1
:1099E00024D0027E002A4BD0B0F90E00A57DB4F938
:1099F0000A60062212FB0502B2423EDD228AE381A2
:109A000002EBC50212B218462282A78A668A029524
:109A10000B468DE8C00001462046FFF719FEA37DE6
:109A2000E28903EB430302EB4303E381012005B02A
:109A3000F0BDA67DB4F90E00B4F91020B4F814E01E
:109A4000678A02960B468DE8804001462046FFF764
:109A5000FFFD2979E389A27D012001FB0233E38127
:109A600005B0F0BD0022C2819A7A817D038A01FB94
:109A700002330382012005B0F0BDB4F91020C4E721
:109A8000857DB4F91020B0F90E00BEE7028A817D11
:109A9000C38102EBC1030382C8E70020E0819B7A07
:109AA000228A03FB062212B22282C7E7C181028208
:109AB000704700BF002908BF01218175704700BFB2
:109AC00081824182704700BFC07D7047B0F90A00B3
:109AD000704700BFB0F90C00704700BF10B4EFF33F
:109AE000108272B6437F33B9017F012907D0032961
:109AF0000FD00123437702B962B610BC7047124CF5
:109B00002168A1B1114943610B6883610860586104
:109B1000EFE70F4C216881B10E4943610B68836107
:109B2000086058610C4B4FF080511960E1E7074B1A
:109B30004161816120601860DBE7064B4161816112
:109B400020601860EEE700BF589EFF1F549EFF1F65
:109B5000489EFF1F4C9EFF1F04ED00E070B5EFF321
:109B6000108272B60C4C206880B10C4E00254369FF
:109B7000236073B19D6102B962B6457783689847E7
:109B8000EFF3108272B620680028F0D102B962B6F5
:109B900070BD3360EFE700BF489EFF1F4C9EFF1F64
:109BA000FFF7DCBF184A30B41468002C27D00368D4
:109BB00021688B420ED2CB1A00218460C1602360E1
:109BC000E06010600223037530BC704711688B425F
:109BD000144608D3A2685B1A0360002AF6D182609B
:109BE000C460A060EEE7D268C2608460E060C568CF
:109BF000CB1A0222A8602360027530BC70478460D3
:109C0000C4601060DEE700BF509EFF1FF8B5224E13
:109C100034682CB32368002B3AD1204F1D4604E052
:109C20003468ECB12368002B32D1A36803B1DD6046
:109C300020693360036825751B68BB4221D1037F0F
:109C40004560022BC46020D0FFF748FF6368002BFB
:109C5000E6D023602046FFF7A5FF3468002CE1D151
:109C6000EFF3108372B60E4A00211068116003B939
:109C700062B628B18468FFF795FF20460028F9D125
:109C8000F8BD224600219847E0E783689847DDE762
:109C9000013B2360E4E700BF509EFF1F1D830000CF
:109CA000609EFF1F024A136801331360FFF7AEBFC7
:109CB0006C9EFF1F704700BF0368F0B4FBB1002526
:109CC00001249D60DC601B4C1A601C44241104F1CB
:109CD00044056A11032692009E60174F0679174BC0
:109CE00047F8241002F1604202F5614205F01F05B9
:109CF000012000FA05F5E6541560F0BC7047104CE1
:109D0000236843F40003236000BF0E4B0E4DA4F5FF
:109D10008734A4F59E7401261E60234604609C6867
:109D2000002CD0D01033AB420360F8D10023036085
:109D30001846E2E7008FFCBFD490FF1F44E400E028
:109D40003C80044000700340407103400168A9B1A9
:109D50000B4BF0B40B441B110A4E0B4F0B4D46F846
:109D6000237003F1440202F01F0401235211A340A7
:109D7000002445F822308C600460F0BC704700BFBE
:109D8000008FFCBFD490FF1FB59C000080E100E075
:109D9000024A034B012111601B6818470C710340F4
:109DA000D490FF1F024A034B012111605B681847E2
:109DB0001C710340D490FF1F024A034B0121116024
:109DC0009B6818472C710340D490FF1F024A034B35
:109DD00001211160DB6818473C710340D490FF1FDC
:109DE000F8B50E4671B17AB10746144600253B68B6
:109DF00016F8011B1B6838469847013C0544F6D10C
:109E00002846F8BD0846F8BD1046F8BD00B5064A1C
:109E1000036812885B6883B001A9ADF804200222B0
:109E2000984703B05DF804FBAC080100F0B50746A5
:109E30008BB0002A33D0012A08BF0A2251B3212453
:109E400000E0F4B2B1FBF2F502FB1511C8B209292A
:109E500000F1300198BFC8B20AA988BF3730214449
:109E600088BFC0B201F8240C661E2946002DE8D137
:109E700033B1013CE4B20AAB23442D2203F8242C75
:109E80003B6801AA11195B683846C4F12202984761
:109E90000BB0F0BD30228DF825202124E8E70368BF
:109EA000C9B21B6898470BB0F0BD00BF0029BABF0C
:109EB00049422D2300230A22FFF7B8BF374A384909
:109EC00013681B06FCD40B6813F08003F8D172B63C
:109ED00034490A78002A5FD0334A3448F0B4344C0D
:109EE000176806682568D4680C303E441432006850
:109EF0001268304F35442C4420440244C2F34E02D1
:109F00002D4E2E482E4D2F4C42F400423A603768B9
:109F100006682D682C4A24680C303E44006812689C
:109F20002A4F35442C4420440244C2F34E02284EAA
:109F30002848294D294C42F400423A6037680668A7
:109F40002D68274A24680C303E4400681268254F6B
:109F500035442C4420440244C2F34E02224E23488E
:109F6000234D244C42F400423A60376806682D685D
:109F7000214A24680C303E440068126835442C4461
:109F800020440244C2F34E021C4842F400420260E4
:109F90000B7062B6F0BC704762B6704724B00340E5
:109FA00024B00B40659EFF1F38B003403CB0034017
:109FB00040B003402CB0034058B003405CB00340B5
:109FC00060B0034064B003406CB0034030B0034065
:109FD00038B00B403CB00B4040B00B4044B00B409D
:109FE0004CB00B402CB00B4058B00B405CB00B4059
:109FF00060B00B4064B00B406CB00B4030B00B4015
:10A0000030B42948294A2A4B2A4D6024E1210470A2
:10A0100011701B78284C082B30D00A2B2748284970
:10A0200037D00C2B0CBF35223D2212232A6023602F
:10A0300002600B60234B24491B78244ABBB10123E7
:10A040000B601360224B23491B78234A012B26D92E
:10A05000042B0FD9082B1ED9102B94BF86238723DE
:10A060000B6013601D4B01221A7030BC70470B60EF
:10A070001360E7E784230B601360F3E700F58E209D
:10A080000F490830012213232A60236002600B600D
:10A09000D0E73922F7E785230B601360E2E78023DE
:10A0A0000B601360DEE700BF00400740014007403F
:10A0B000E490FF1F08B003400CB0034008B00B4011
:10A0C0000CB00B40689EFF1F20B0034020B00B4037
:10A0D000E590FF1F24B0034024B00B40659EFF1F96
:10A0E0000C2830B417D91023984228BF18461C46B4
:10A0F000104A114D1178181A8C42287018D00F4947
:10A1000013700B7823B10E490E4A00230B601360C5
:10A1100030BCFFF775BF0A2802D90C231C46E7E7BD
:10A12000082802D90A231C46E2E708231C46DFE779
:10A1300030BC7047E490FF1F649EFF1F659EFF1FA9
:10A1400024B0034024B00B4028282FD8334B2DE9EE
:10A15000F0411E5CFF2E2BD0314B1B78002B2AD1F7
:10A1600032062CD472B62F4D2F4C2F460123266079
:10A170002B7062B672B623681B060CD43B781BB9F1
:10A18000F4E72B78002BF1D062B602F09BF972B69F
:10A1900023681806F5D5254B1B6800222A7062B685
:10A1A000234A107843FA00F0BDE8F08100207047A0
:10A1B0000020BDE8F081FFF781FE3206D2D572B6ED
:10A1C0001C4DDFF87C801C4C06F04007FFB206F007
:10A1D0003F06D8F80030DFB123F01003C8F8003094
:10A1E00001232660134A2B7062B672B623681906E3
:10A1F0000CD413781BB9ECE72B78002BE9D062B6AE
:10A2000002F060F972B623681B06F5D50B4BC3E765
:10A2100043F01003C8F80030E2E700BFB0080100C7
:10A22000659EFF1F679EFF1F00B0034010B00340F4
:10A23000649EFF1F669EFF1F00B00B4010B00B40D6
:10A240000CB00B400A4A0B49136843F48053136067
:10A250000B7843B9084BC0221A70084B80F30C00EE
:10A2600000B218807047044B80221A70F5E700BFD7
:10A270002C800440689EFF1F21C00C4000C00C4091
:10A28000F0B51B4B1B4E596818689A68DB6885B09F
:10A290006C460FC4337899071DD5174A174C1378AD
:10A2A000174913F0700318BF1370164A164B802716
:10A2B000177000263320032226706D4608701A702E
:10A2C00072B6043C45F001052046A84762B62378E3
:10A2D00013F0700309D10D4B064901E0013B02D098
:10A2E0000A78D207FAD505B0F0BD237005B0F0BDED
:10A2F000DC080100010002400000024004000240AE
:10A300000B000240070002400A000240410D03001A
:10A31000B0F5006F0AD210B5094B1B78DB07044675
:10A3200006D504F1A0500078C0B210BD00207047DF
:10A33000FFF7A6FF04F1A0500078C0B210BD00BF27
:10A3400001000240B0F5006F17D238B50F4B1B78F3
:10A35000DA070D46044611D504F1A0500378AB424C
:10A360000AD00B4A137813F0700318BF1370074A12
:10A3700005701378DB07FCD538BD7047FFF780FF09
:10A3800004F1A0500378AB42EBD1F5E701000240A5
:10A390000000024008B5F6F771F9F7F771FD02F019
:10A3A00091F8FAE7844641EA000313F003036DD104
:10A3B000403A41D351F8043B40F8043B51F8043B88
:10A3C00040F8043B51F8043B40F8043B51F8043B8F
:10A3D00040F8043B51F8043B40F8043B51F8043B7F
:10A3E00040F8043B51F8043B40F8043B51F8043B6F
:10A3F00040F8043B51F8043B40F8043B51F8043B5F
:10A4000040F8043B51F8043B40F8043B51F8043B4E
:10A4100040F8043B51F8043B40F8043B51F8043B3E
:10A4200040F8043B51F8043B40F8043B51F8043B2E
:10A4300040F8043B403ABDD2303211D351F8043BCE
:10A4400040F8043B51F8043B40F8043B51F8043B0E
:10A4500040F8043B51F8043B40F8043B103AEDD27D
:10A460000C3205D351F8043B40F8043B043AF9D2CE
:10A47000043208D0D2071CBF11F8013B00F8013BA1
:10A4800001D30B8803806046704700BF082A13D3AE
:10A490008B078DD010F003038AD0C3F10403D21AC6
:10A4A000DB071CBF11F8013B00F8013B80D331F8FA
:10A4B000023B20F8023B7BE7043AD9D3013A11F87A
:10A4C000013B00F8013BF9D20B7803704B784370E5
:10A4D0008B7883706046704708B5104C08E023689D
:10A4E00059050DD423681A050FD42368DB0411D451
:10A4F00023685803F3D500F08DFE23685905F1D584
:10A5000002F044F823681A05EFD502F0D5F8236865
:10A51000DB04EDD500F0F0FCEAE700BF3480044036
:10A5200008B5FFF7D9FF00BF014B10221A80704712
:10A5300000200540704700BF094908B50B6830B1DD
:10A540006A461844A2F58052904202D2086018462A
:10A5500008BD03F063FB0C2303604FF0FF3008BD20
:10A56000E890FF1FFEE700BFEFF3138070B9EFF331
:10A5700010836BB9EFF305825AB94FF48070EFF393
:10A5800011832BB1984228BF184670474FF0FF3017
:10A5900070470F2A01D81846F1E7014BD05CEEE76F
:10A5A000F0E300E0F0B44D1E2E46002400E001343C
:10A5B000B0FBF2F302FB1300092800F130078ABF59
:10A5C0003730F8B2C0B206F8010F1846002BEED1B2
:10A5D0000A1953704CB1107815F8016F28700133C7
:10A5E000E01A834202F80169F5DB0846F0BC7047C7
:10A5F000704700BF10B40F4B53F8302092F88042E0
:10A600002CB1012369B182F8803010BC704703EB94
:10A61000C0035B681A6841B922F002021A6010BCDC
:10A62000704782F8003110BC704742F003021A6094
:10A6300010BC7047EC0801001C4A02EBC003012962
:10A640005B6811D004291BD052F83000002280F83A
:10A65000802229B1022920D0032922D01A60704714
:10A660004FF480721A60704752F830004FF4A272B3
:10A6700080F880121A601A6822F020021A6070476F
:10A6800052F830104FF4A272012081F880021A6053
:10A690001A6842F020021A60704740F203121A60F2
:10A6A00070474FF481721A60704700BFEC080100D8
:10A6B000212848D8F8B5042A44D8DFE802F0484BEE
:10A6C0004E0345004FF410262B4B03EBC0030D4601
:10A6D0005C68216811F4E06148D0284B284A294978
:10A6E000C3F89C2104F140422748C3F8A411A2F505
:10A6F0009221264FC3F8A0017C292548C3F8A871F0
:10A70000C3F8AC012CD9A2F594237C2B2AD9A2F54D
:10A7100096237C2B28D9A2F598237C2B29D9A2F546
:10A720009A227C2A27D81B4872B6236823F4702308
:10A7300043F08072C4F384011643236040F8215033
:10A74000266062B6F8BD70474FF43026BCE74FF480
:10A750000026B9E74FF44026B6E74FF42026B3E7CA
:10A760000D48E1E70D48DFE70D48DDE7FFF764FF3F
:10A77000B3E70C48D8E7F8BDEC0801000082FF1FE2
:10A78000F188FF1F9988FF1FC588FF1F6D88FF1F75
:10A790004188FF1FC491FF1FEC90FF1F2491FF1FF2
:10A7A0007491FF1FA491FF1F1A4B03EBC00010B45C
:10A7B000426802F14043A3F592217C2923D9A3F5F5
:10A7C00094217C290DD9A3F596217C291FD9A3F5C5
:10A7D00098217C2919D9A3F59A237C2B11D80E4CEA
:10A7E00000E00E4C72B613680D4823F08773C2F375
:10A7F000840123F4803343F08073136044F8210014
:10A8000062B610BC7047074CECE7074CEAE7074C10
:10A81000E8E700BFEC080100C491FF1F2491FF1F6F
:10A82000F1A50000EC90FF1FA491FF1F7491FF1F82
:10A8300030B4054B054D064C002210211A602A60E9
:10A840002060196030BC704714D0034004D003402E
:10A8500000D00340282838B52ED0002904464FDD0B
:10A860005F4B1B78012505FA03F28A4202D82128A2
:10A8700037D938BD0338C2B2012A3AD9202C4AD080
:10A88000192C48D0574A126802FB011222FA03F32E
:10A890001D2800F29B80DFE800F0928B847D99995F
:10A8A000766F99999999999999999968615A539953
:10A8B0004C99999999999945494B1B780B2B08D933
:10A8C0000C2B1CBF0C3B19410846BDE83840FFF774
:10A8D000B9BCC3F10C0399400846BDE83840FFF706
:10A8E000B1BC2946FFF786FE2946BDE83840FFF790
:10A8F000A3BE3D4A126802FB011222FA03F3C7E726
:10A900002128B6D80021FFF775FE20460121BDE8B9
:10A910003840FFF791BE354A126802FB011222FA55
:10A9200003F3B5E73249334A0B604FF451731360B8
:10A9300038BD3149314A0B604FF45173136038BD53
:10A940002F49304A0B6040F24443136038BD2E4912
:10A950002E4A0B6040F24443136038BD2C492D4A07
:10A960000B6040F24443136038BD2B492B4A0B6007
:10A9700040F24443136038BD29492A4A0B6040F233
:10A980004443136038BD2849284A0B6040F24443D1
:10A99000136038BD2649274A0B6040F244431360D8
:10A9A00038BD2549254A0B6040F24443136038BD49
:10A9B0002349244A0B604FF45173136038BD224978
:10A9C000224A0B604FF45173136038BD212C3FF6BF
:10A9D00050AF7F29D4BF00210121204693E700BF5B
:10A9E000CC91FF1F088003400890034008800B4073
:10A9F00010800B4048A0044018800B404CA004403D
:10AA00001880034008B004401080034004B00440A4
:10AA10004080034018C004403880034014C0044004
:10AA20002880034010B00440208003400CB0044054
:10AA30003080034010C00440488003401CC00440E4
:10AA4000189003403490044010900340309004402C
:10AA500038B1102828BF1020044AC3B210781370F0
:10AA60007047024A0123107813707047CC91FF1F82
:10AA70002DE9F8430E4680463249334D304603F007
:10AA800053F847F6122300281ABF1D464FF002095B
:10AA90004FF00109002425FA04F002F04FFE4FF0B8
:10AAA0005E51074602F0A2FE0146304603F050F820
:10AAB00030B90134072CEED1E80902F03FFE074619
:10AAC0003146384602F046FF4FF07C5102F084FDDB
:10AAD00003F078F84FF6FF729042A8F1030328BF05
:10AAE0001046012B29D9B8F1170F17D8174B23FAA5
:10AAF00008F303F0010383F0010223B9B8F1190F41
:10AB00000FD0BDE8F883124B124D13491A6044EA86
:10AB1000C9042A6008601C60BDE8F883B8F1200F02
:10AB2000ECD10E4B0E4D0F49002244EAC9041A60C5
:10AB30002A6008601C60BDE8F8830B4B0B4D0C4984
:10AB4000F2E700BF001BB740006CDC026006F000BB
:10AB500000800340048003400880034000800B40D5
:10AB600004800B4008800B40009003400490034099
:10AB700008900340212801D8FFF73CBD704700BF73
:10AB8000212806D8044B53F8303093F80002C0B2A5
:10AB900070470020704700BFEC080100212801D851
:10ABA000FFF74ABD704700BF72B60C490C4B0D4A07
:10ABB0001B680868126862B6520102D5322B88BF42
:10ABC00001300949C3F5BB334FF47A72FF33A1FB5F
:10ABD000031302FB00F000EB931070476C9EFF1F05
:10ABE00018E000E004ED00E0ABAAAAAA2DE9F843C2
:10ABF000054672B6204F214B214A1B683C681268FB
:10AC000062B6520102D5322B88BF013495B3C3F529
:10AC1000BB331C4EDFF86490DFF86480FF334FF4E1
:10AC20007A72A6FB031302FB04F404EB931472B6CE
:10AC3000D9F800103A68D8F800E062B6C1F5BB3325
:10AC4000FF33A6FB03031EF0806FC4EB93134FF496
:10AC50007A7002D0322988BF013200FB0233B3F58B
:10AC60007A7F04D3013D05D004F57A74DFE701F063
:10AC700029FCDCE7BDE8F8836C9EFF1F18E000E0CC
:10AC800004ED00E0ABAAAAAAF8B52D4B2D49DFF8D8
:10AC9000D0E0DFF8D0C02C4E2C4D2D4C2D4A2E4F3D
:10ACA0004FF4000018604FF0807018604FF0007093
:10ACB00018604FF0806018604FF00060186000204E
:10ACC000086028234BF6FF71CCF80010CEF8003056
:10ACD000336013602B6023603B60B3629362092290
:10ACE00045F8242CC4F8D80F05F57F65C7F8D41FA4
:10ACF00007F5FF2707F5FA67C6F8F83F2B6006F55A
:10AD0000FF26C4F8D42F05F5FD2504F5FF2438608F
:10AD100006F2F4761148316005F5FF6504F5FD642F
:10AD20002B6023600260FFF76BF91920FFF75EFFCD
:10AD300000F0B6FF40F21310BDE8F840FFF756BF31
:10AD400008E100E0048003401480034024800340B5
:10AD50002C8003401C8003403480034000800B4063
:10AD60000C800340088003402DE9F84F214B1B68FD
:10AD700007460BB101221A70DFF888901E4D99F832
:10AD80000040DFF884801D4E0134272C8ABF4FF02D
:10AD9000000A5FFA84FA5446AB462B78A34216D1D8
:10ADA000FFF7E2FB40281FDC33791B06F5D59BF843
:10ADB00000300133272B86BF00221346DAB218F881
:10ADC0000330DBB2F3712A702B78A342E8D00C4930
:10ADD0000A4BFFB208F804700120AC22087089F811
:10ADE00000A0DA70BDE8F88FFF28D6DD01F06AFB1D
:10ADF000D3E700BFE49EFF1FE19EFF1F00C0064097
:10AE0000E09EFF1FE89EFF1F789EFF1F1C4BDFF890
:10AE100094C01A681B49F0B542F480521A4D1A606A
:10AE2000DFF884E0194F1A4E1A4C00238CF80030DA
:10AE30004FF451722B701F2840F213358EF80030FA
:10AE40003B70337025600A6012D819460124124AFB
:10AE5000124D11701248547000212C274026937215
:10AE60004FF4003491701174D7702E700460F0BDEF
:10AE7000C0F34431C0F3471400F01F03E7E700BFFD
:10AE8000348004400CC00440759EFF1FE19EFF1FEC
:10AE9000E09EFF1F08C0044000C0064031E400E00F
:10AEA00004E100E0749EFF1FE89EFF1F034B1B6838
:10AEB000DB0401D5FFF758BF704700BF3480044062
:10AEC00010B5044C237823B101F0FCFA2378002B51
:10AED000FAD110BDE09EFF1F054A064B10781B7883
:10AEE000C0B2DBB2984238BF4030C01A704700BFD2
:10AEF000749EFF1F759EFF1F30B42B4B1A7994066A
:10AF00001FD52A48DA790378294901333F2B09787C
:10AF1000C8BF00238B42D2B203D0264CD9B2E25430
:10AF20000170254A116861B1244A1278D2B2934265
:10AF300036BFC2F140029B1A9B18272BC4BF0123C6
:10AF40000B70194AD378DBB2180611D45A060DD506
:10AF5000154B1B795B0609D5194B1A491B68002252
:10AF60000A7003B11A70104B2C22DA7030BC704793
:10AF700011790906EAD5144910480C780178C9B24C
:10AF80008C420DD04A1C272A84BF00210A460F4D4F
:10AF9000054C98BFD1B2AA5CD2B2E2710170D5E77C
:10AFA0006C21D170D2E700BF00C00640749EFF1F25
:10AFB000759EFF1FA09EFF1F709EFF1FE19EFF1F3B
:10AFC000E49EFF1FE09EFF1FE89EFF1F789EFF1F6D
:10AFD00021282FD8184B195CFF292BD0174B184A62
:10AFE000DFF870C003EBC000F0B54368DFF868E03D
:10AFF000144F154D154E00241C60DEF80030012062
:10B0000043F020038840CEF8003014604FF4A07362
:10B0100038602E60C2F800C0013BFDD113689B056B
:10B02000FCD42023013BFDD1094B09B233F81100B8
:10B0300080B2F0BD00207047FC090100EC0801005F
:10B040000050044008500440045004400000020333
:10B050000051044080014A0038800440431E032B05
:10B0600014D872B60A4951F8230068B170B4094C7B
:10B07000058834F81320466841F82360521B24F8F1
:10B08000132062B670BC704762B6704700207047EC
:10B09000449FFF1F88A1FF1F013803280BD872B6F9
:10B0A000074B53F8203043B100205B680130002B80
:10B0B000FBD162B67047002070471846F9E700BF21
:10B0C000989FFF1F30B472B62B4A13781D0706D520
:10B0D0002A4B196A002936D0996A002941D0537841
:10B0E0001C0706D5254B196C00293ED0996C002908
:10B0F00039D09378190705D5204B196E002936D021
:10B10000996E89B1D3781B0707D51C4BD3F88020E3
:10B110007AB3D3F8882011213AB162B6184B0022D5
:10B120001A7030BC00F04ABE0D21154C154D227826
:10B1300043F8315003EBC1030830013A58602270E4
:10B1400062B630BC704704220D4C0F4D217843F895
:10B15000325003EBC20308304A1E5860227062B6B8
:10B16000EFE70521E1E70921DFE70822ECE70C2200
:10B17000EAE71022E8E700BF200A01000080FF1F75
:10B18000C19FFF1FC800400088004000431E032BE2
:10B190001DD81B4A400140F0100030B4104472B674
:10B1A000184CE25C032A1BD8DFE802F002121517E4
:10B1B00003220D88E25410F0080F14BFC82388231F
:10B1C00043EA054308310360416062B630BC704712
:10B1D00008300222EDE70522EBE708300422E8E719
:10B1E000094A52F8230038B1084A52F82300416056
:10B1F00042F8231062B6E9E742F82310034AF7E762
:10B200000080FF1FD09FFF1F989FFF1FA89FFF1F59
:10B2100000BE70472DE9F04FDFF818B3DFF818A330
:10B2200087B044E0AD4F4FEA930807EBC809013EF1
:10B23000D9F8042003F00803F6B2A2F1080003F0E5
:10B24000FF04002B40F0018157F838301B0C99B2F5
:10B2500022F8081C002B00F0EF80A14B22F8064CCE
:10B2600042F8044C53F82620002A00F0CF819D4D6F
:10B2700055F8263058609C4C45F8260034F81630B6
:10B28000194424F8161000F079FD002800F0C2815E
:10B29000964A974B19F0080F00F1080018BF1346A3
:10B2A000C9F8040047F8383008238BF800309BF8C1
:10B2B0000040E4B265071CD58E4B1B78B3B18E49B4
:10B2C0000A7802F0FF0322B1013BDBB20B7003B935
:10B2D00000BE8A490A7802F0FF032AB1013BDBB2C3
:10B2E0000B70002B00F0688100F066FE04238BF8E1
:10B2F000003004F0080303F0FF02002B00F0C980C7
:10B300009AF80030DBB21E098CD19A08DFF8CC9194
:10B3100059F8321009EBC200C1F3830101394068CA
:10B320000C2900F28580DFE801F07A7A8383838339
:10B3300083834683838307000168714D4068714FA2
:10B34000714E6860296088B240F281610024674BC9
:10B3500049F832304FF0010E88423C60C9F8104085
:10B36000C9F8184086F800E05C4A00F2E780B0F5C2
:10B37000D06F80F01B82B0F5817F00F0D98100F2A0
:10B380006981802800F02A82822840F0D781A9882C
:10B3900001F07F01042900F2D1815C485C4A8900F8
:10B3A00008441470547001788C0740F1608382F86F
:10B3B00000E0022173E1534F3A682AB3554B524ED5
:10B3C000554819883478057840298E4645F002089A
:10B3D00028BF4FF0400E002C84F001043470CEEBF7
:10B3E00001010CBF8824C82409EBC80689B285F086
:10B3F000010544EA0E447260198049F838407244ED
:10B400000570002965D03A603D4B1A88B2F5A06FEF
:10B410000ED100219A785970404B1A7008E03849D3
:10B420003F4C0D68A54200F09880304949F8321031
:10B430003C4A0123137037E72C4A2D4B19F0080FB3
:10B4400018BF134647F838302EE700F0B7FC364AED
:10B45000364952F82630002B00F0E38058688C5DA6
:10B4600042F8260003F10802C9F80420032C05D88D
:10B47000DFE804F02C02292602228A551A8819F0E6
:10B48000080F0CBF8823C82343EA024347F838302B
:10B490000AE7E00700F19380210600F1D180A207BE
:10B4A00006D5234A234913780220DBB213700870B3
:10B4B000E30602D51F4B10221A7007B0BDE8F08FCB
:10B4C00004228A55DAE705228A55D7E703228A55EE
:10B4D000D4E7BEF1400F18BF002294E70080FF1FA1
:10B4E000449FFF1FF09EFF1F88A1FF1FC800400060
:10B4F00088004000CC9FFF1F559FFF1F40A0FF1FEB
:10B50000B89FFF1FEC9EFF1F549FFF1FC0200740E6
:10B51000C49FFF1F009FFF1FC09FFF1F9820074071
:10B520002109000394200740989FFF1FD09FFF1F11
:10B53000882007408020074090200740B0F5106F1A
:10B5400000F07C8140F2A38040F62112904240F04E
:10B550007B82A54A012313706AE74C68A3498C4299
:10B560007FF463AF0178A9297FF45FAF4178452963
:10B570007FF45BAF8178C2297FF457AFC1786B2924
:10B580007FF453AF9A489B4E0178347881F00105DF
:10B59000002C41F0020105700CBF8820C82084F007
:10B5A000010449F8310009EBC101934834700025CA
:10B5B00005244D60047038E700F064FF94E68F4B7B
:10B5C00089488B491A614FF0020E80F800E08C4FD9
:10B5D0000A708C49196099608B4E8C4D8C4C9A6125
:10B5E0000D213970FF213170DFF84CE22970227093
:10B5F000884D894A8EF800109F27012406F8047CA4
:10B600005D600470DA6007B0BDE8F08F43F8260093
:10B61000824D30E6824A47F83800137801331370C0
:10B6200042E68B5D032B00F2BA8001A252F823F0B0
:10B63000A9B20000A9B2000089B6000083B60000DC
:10B640006F49724B80220D2008701A70A2077FF597
:10B650002FAF26E740F20232904240F0ED81AA88F7
:10B6600002F07F02042A69D86D88002D66D16449F2
:10B67000CDF804E0920011440A7842F002020A7008
:10B68000C1E101238B550FE600238B550CE6B0F585
:10B69000086F53D16349644A097811707146ED8887
:10B6A0008D4280F0E88252480478402DAE4644F046
:10B6B000020C28BF4FF0400E02EB0E0309EBCC0149
:10B6C000029301234A604FEA0E48CEEB0501019335
:10B6D0000025C82242EA080384F0010249F83C3000
:10B6E00035700270DFF814C1424BDFF8048149BBAA
:10B6F000BEF1400F7FF42DAF42F0020C09EBCC03FA
:10B70000029ADFF8F8E05A608DBB0D0445F0880519
:10B710009DF804304EF83C500A44337004701346D0
:10B7200040297FF416AF0021404A3B60118010E7AA
:10B73000AA8802F07F02042A40F28B81304A0F234C
:10B74000137006E74029D7D942F002020CEBC20081
:10B75000029E4660BDB19DF8045035481D703346C9
:10B76000403988F8004040334CF83200DCE79DF85F
:10B77000043033700D04029B047045F0C8050B447F
:10B780004EF83C50CCE79DF804501D70029B1D48BC
:10B7900088F80040403940334CF83200C4E719F0D3
:10B7A000080F0CBF022303238B557DE521494A680E
:10B7B000002AC3D06C88B5F804E003E00C314A6875
:10B7C000002ABBD00B88A342F8D14B887345F5D132
:10B7D000240A032C0CBF1178098960E7124A022160
:10B7E000147054705BE700BF942007400100040010
:10B7F000C09FFF1F549FFF1F559FFF1F0080FF1F0B
:10B80000C020074088004000882007408020074073
:10B8100098200740049FFF1F589FFF1FF09EFF1FA7
:10B82000C19FFF1FCC9FFF1FC49FFF1F009FFF1FD3
:10B83000C8004000240A01008C200740B248116A69
:10B84000AC7804700C0600F19881D9F82820AF4933
:10B85000100600F1DB81D9F83020AC49120600F166
:10B86000D081D9F83820A949130600F1C581D9F84B
:10B870004020A649150600F1BA81D9F84820A3490D
:10B88000140600F1AF81D9F85020A049100600F14C
:10B89000A481D9F858209D49120600F19981D9F860
:10B8A00060209A49130600F18E81D9F868209749E3
:10B8B000150600F18381D9F870209449140600F12F
:10B8C0007881D9F878209149100600F16D81D9F876
:10B8D00080208E49120600F16181D9F888208B49B9
:10B8E000130600F15581D9F890208849150600F11A
:10B8F0004981D9F898208549140600F1FF808448D1
:10B90000844A854901908548854D864C04970023DB
:10B910000596029580460F4616461D4603943068EC
:10B9200028B1446800F04AFA2046002CF9D10023DF
:10B930003360029B38681A46002342F8253028B14C
:10B94000446800F03BFA2046002CF9D100223A600E
:10B95000019A98F800301146002241F8042B039A0E
:10B960000191023B4FF0000122F81510032B07D87C
:10B97000DFE803F05D025D024FF0010388F800305C
:10B980000135042D06F1040607F1040708F101084A
:10B99000C5D1654C654D2278654B049F059E0021FD
:10B9A000100729701A7000F19280624962780A705B
:10B9B0000021C9F83010C9F838101107DFF84C81A0
:10B9C0006ED4A2785C49DFF844810A700021120726
:10B9D000C9F85010C9F858104BD4E27857494B4C6D
:10B9E0000A7013074FF00001C9F87010C9F87810F9
:10B9F00000F1AE8033780193002283F00105C9F88D
:10BA00009020C9F898200021029188468E460A4667
:10BA10004B48047844F0020C09EBCC030393019BE0
:10BA2000002B039B5A600CBF8822C82252E64FF0BD
:10BA3000000388F80030A3E7B0F5A06F7FF47EAE76
:10BA4000012300250193DEE740F621229042F7D042
:10BA500074E66D88002D7FF471AE3A49CDF804E0AC
:10BA6000920011440A7822F002020A70CBE7022108
:10BA700015E600F083F9002800F0EB800830324A28
:10BA8000C8F86400C8F8602000F078F9002800F0D9
:10BA9000DA8008302D4AC9F86C00C9F868209CE7A4
:10BAA00000F06CF9002800F0E0800830264AC8F861
:10BAB0004400C8F8402000F061F9002800F0CF8071
:10BAC0000830224AC9F84C00C9F8482079E700F04C
:10BAD00055F9002800F0A58008301B4AC9F8240059
:10BAE000C9F8202000F04AF9002800F094800830BE
:10BAF000164AC9F82C00C9F8282056E7D1F89C004E
:10BB0000083800F05BF9FAE6CC9FFF1F0080FF1FAA
:10BB1000A89FFF1F449FFF1F989FFF1FD09FFF1FDD
:10BB2000F09EFF1F88A1FF1F200A0100C19FFF1F79
:10BB3000C4200740C8200740CC200740D020074041
:10BB4000C09FFF1FC020074088004000C800400081
:10BB500000F014F9002870D008304F4AC4F884006F
:10BB6000C4F8802000F00AF9002860D008304B4A61
:10BB7000C9F88C00C9F888203CE7506A083800F002
:10BB80001DF962E6D1F89400083800F017F9B0E624
:10BB9000D1F88C00083800F011F9A4E6D1F884003F
:10BBA000083800F00BF998E6C86F083800F006F97D
:10BBB0008DE6486F083800F001F982E6C86E083853
:10BBC00000F0FCF877E6486E083800F0F7F86CE60D
:10BBD000C86D083800F0F2F861E6486D083800F0EA
:10BBE000EDF856E6C86C083800F0E8F84BE6486C0B
:10BBF000083800F0E3F840E6C86B083800F0DEF8DB
:10BC000035E6486B083800F0D9F82AE6C86A0838E3
:10BC100000F0D4F81FE62A78C9F8280001322A700B
:10BC2000C3E62A78C9F8200001322A705AE72A7838
:10BC3000C9F8880001322A70DCE62A78C4F880004E
:10BC400001322A708EE72A78C9F8680001322A701A
:10BC5000C3E62A78C8F8600001322A7014E72A780F
:10BC6000C9F8480001322A70ABE62A78C8F84000CB
:10BC700001322A701FE740298E4628BF4FF0400E40
:10BC800002EB0E0302930123CEEB01014FEA0E48B3
:10BC900000250193BCE600BF88004000C8004000BA
:10BCA000F8B500F08FFD294B29482A4C2A4F2B4D1F
:10BCB000DFF8BCC0DFF8BCE0294E00221A605A60F1
:10BCC0009A60DA601A615A619A61DA611A625A629C
:10BCD0009A62DA621A635A639A63DA631A645A647C
:10BCE0009A64DA641A655A659A65DA651A665A665C
:10BCF0009A66DA661A675A679A67DA67C3F8802025
:10BD00000168C3F8842041F480210160C3F3072156
:10BD10002170C3F30740134938701B0E2B70FF23AB
:10BD20008CF80030104D8EF8003010480B70012355
:10BD3000337084F8642070264FF40074102207F8E2
:10BD40002C3C2E70046081F8F820F8BD0080FF1FA5
:10BD5000348004409C200740B0200740B4200740B6
:10BD6000942007401020074049E400E008E100E08B
:10BD70008020074088200740704700BF72B60D48FA
:10BD80000268B2FA82F30F2B10DC4FF00041D94069
:10BD900022EA0102026062B6074803EBC303DB003C
:10BDA000C2180021C15010465160704762B6002091
:10BDB000704700BFD091FF1FBC83FF1F0D4B0E4A81
:10BDC000C31AA2FB03231B090F2B0CD80B4A1278B2
:10BDD00052B972B60A484FF00041026821FA03F3E3
:10BDE0001A43026062B67047064A1278002AF0D001
:10BDF000FFF768B9BC83FF1F398EE338C19FFF1F6F
:10BE0000D091FF1FCC9FFF1F38B50E4B0E4C1B6807
:10BE1000218805468BB1B1F5917F05D20B4A4B1CA9
:10BE200055549BB2238038BD002208489847002112
:10BE3000064A55540123238038BDB1F5917FEDD3D7
:10BE400038BD00BFF89FFF1F92A1FF1F98A1FF1FE1
:10BE50002DE9F843214E224F3168012380463B7083
:10BE6000B1B1204D4B8801EB8302013300240F2B2D
:10BE7000C2F808802C7004D84B8000233B70BDE8CA
:10BE8000F88340230B800320FFF780F93460F4E748
:10BE9000DFF8549099F80030002BF0D0114D45F6A2
:10BEA000215408E0013C12D02B7883B900F00AFB42
:10BEB00099F800307BB10320FFF7EEF80528F1D8A0
:10BEC000FFF75CFF014630600028EBD0CAE7012392
:10BED0002B70BDE8F883BDE8F88300BF14A0FF1FF6
:10BEE000E89FFF1F18A0FF1FCC9FFF1F1201F8B58E
:10BEF000D5B2A1B3012943D04378044600781B068C
:10BF000043EA004040F4704045F004068F1E304381
:10BF1000FFF79EFF022F04F1020314D9053414F831
:10BF2000023C14F8032C14F8010C1B0443EA02230E
:10BF3000334343EA0060033FFFF78AFF022F2346A3
:10BF400004F10304EBD8022F23D0012F0DD045F4C8
:10BF5000774040F00500BDE8F840FFF779BF14488E
:10BF60002843BDE8F840FFF773BF187845F477051C
:10BF700045F0060545EA0020BDE8F840FFF768BF38
:10BF800003780C4845EA03452843BDE8F840FFF72D
:10BF90005FBF1A78587845F0774545F0070545EAC0
:10BFA000022545EA0040BDE8F840FFF751BF00BF59
:10BFB00006F0F70007F000F738B5084B1C7824B9F5
:10BFC000074D296809B14B8803B938BD9B000B8028
:10BFD0000320FFF7DBF82C6038BD00BFE89FFF1F90
:10BFE00014A0FF1F2DE9F041AD4E33680746002B2A
:10BFF00000F092801D885A88910803EB8101043279
:10C00000AA428C6842D25A8004F00F064FEA1428E4
:10C01000A449A6F1080208F00F00C4F30313062A8E
:10C0200000F101050B701AD9B31E012B5FFA88F0DD
:10C030004ED9052E48D0042E00F0A481731F022B88
:10C040007FD90F2E0ED1F72842D8F02802D0964B78
:10C050001B883BB1FFF7D8FE0020BDE8F08127B177
:10C06000BD4202D00020BDE8F081082EC4F30333A6
:10C0700000F08780092E11D00A2E40F094800A2B00
:10C08000F0D18A4B8A4A1B68A02181E01846FFF74D
:10C0900095FE0420FEF7E2FF3060B5E7092BE1D101
:10C0A000270E00F07B81834B814A1B689021C4F3EB
:10C0B00007461170EDB2FCB2002B00F09D802246C5
:10C0C00031462846984797E0F02843D9F72841D0D1
:10C0D000F1380E28C6D801A353F820F093C200000F
:10C0E00077C2000065C2000065C0000065C00000A6
:10C0F00057C2000065C0000037C3000065C00000E3
:10C1000001C300001BC300003FC2000065C0000067
:10C1100027C200000BC20000674B1B78002BA1D088
:10C120000420FEF79BFF0346306000289AD0058864
:10C13000002D7FF460AFFFF741FE35602846BDE873
:10C14000F081FFF761FEC4F30740FFF75DFE072EA5
:10C1500002D1200EFFF758FE534B584A1988584811
:10C160001468584D524A017000270E0AF0201F80B3
:10C170002E7010700CB301225348A0470120BDE877
:10C18000F081082B7FF46EAF504B494A1B68802129
:10C19000C4F307461170EDB2240E6BB32846224655
:10C1A0003146984728E00B2E11D10B2B7FF45AAF64
:10C1B000474B3F4A1B68B021EAE7464B1B68002B00
:10C1C00000F0FB80404898470120BDE8F0810C2E2C
:10C1D00040F000810C2B7FF445AF3F4B344A1B6885
:10C1E000C0211170EDB2C4F30746002B00F0C880E7
:10C1F00028463146240E98473849314A314B0D7054
:10C2000016701C700120BDE8F081354B1B68002BB7
:10C2100000F0D6809847C4F30746254BEDB2240EB4
:10C2200083F80080E8E72F4B1B68002BF2D12E4BE0
:10C230001B68A3B1FE209847C4F30746EDE72B4BDC
:10C240001B68002BE6D1284B1B6843B1FC209847A4
:10C25000C4F30746E1E7264B1B68002BDAD1C4F391
:10C260000746DAE7234B1B68C4F30746002BD4D0FC
:10C2700030469847D1E7204B1A68002AEFD0260CA9
:10C28000630C06F07F0003F47E531843F6B2904728
:10C29000C3E71A4B1B68C4F30746002BE8D1BCE781
:10C2A00020A0FF1F96A1FF1F92A1FF1FFC9FFF1F51
:10C2B00090A1FF1F30A0FF1FCC9FFF1FF89FFF1F03
:10C2C00094A1FF1F95A1FF1F98A1FF1F28A0FF1F8A
:10C2D0002CA0FF1F10A0FF1FEC9FFF1F97A1FF1FA7
:10C2E000D89FFF1FDC9FFF1FE09FFF1F1CA0FF1FA9
:10C2F0000CA0FF1F24A0FF1FF49FFF1F08A0FF1F1B
:10C300003F4B1B68002B85D13E4B1B68002BA6D0F2
:10C31000FA209847C4F307467FE73B4B1B68002B86
:10C320007FF478AF374B1B68002B98D0FB209847E1
:10C33000C4F3074671E7354B1B68002B7FF46AAFE7
:10C34000304B1B68002B8AD0F8209847C4F307466F
:10C3500063E70E2B7FF486AE2D4A2E4B1268E02148
:10C360001970002A47D0260C610C06F07F0301F4F7
:10C370007E511943EDB2A1F5005128469047F6B21F
:10C38000240E39E7FFF740FDC4F30740FFF73CFDFB
:10C39000200EFFF739FD0020BDE8F0811E4B1D4A3D
:10C3A0001B6880211170EDB2C4F3074683B131469A
:10C3B00028463A4698473C461EE70120BDE8F081F2
:10C3C000104B1B68002B3FF44AAFFF20984746E70D
:10C3D0001C4611E70D2EBCD10D2B7FF443AE0F4B45
:10C3E0000C4A1B68D0211170EDB2C4F30746002B34
:10C3F0007FF4FEAEC4E7C4F30746EDB2240EFBE6BD
:10C4000004A0FF1FE09FFF1FE49FFF1FD49FFF1F9B
:10C41000F09FFF1F90A1FF1F28A0FF1F00A0FF1F7C
:10C4200038B5164D2868E0B101884488A14213DD73
:10C4300003191B7A83B104F10803C2180C1B0023F3
:10C4400002E012F8011F21B10133A342F9D12046C5
:10C4500038BD1C46204638BDFFF7B0FC00202860E0
:10C4600038BD074B1B780BB9002038BD0220FEF702
:10C47000F5FD28600028D7D1F6E700BF3CA0FF1FDC
:10C48000CC9FFF1F0D4B1B78BBB910B50C4C21681E
:10C4900003F0FF024B883F2B07DC07330B4401F10D
:10C4A000470003F8012F8342FBD140230B8001207A
:10C4B000FEF76CFE0023236010BD704734A0FF1F01
:10C4C00038A0FF1F38B5224C237803B138BD0123B3
:10C4D0002370FFF7A5FF70BB00F048F840BB00F0E9
:10C4E000DBF810BBFEF7F8FCE0B900232370EFF394
:10C4F0000583002BEAD1EFF3108172B6154B186853
:10C50000E0B1154C2278CAB945691D60012323703A
:10C51000C5B1AA6101B962B600254577836898471D
:10C520002570D3E700F020F8DFE700F01BF8D9E72B
:10C5300000F016F8D3E7FFF71FFCCDE70029C5D1BF
:10C5400062B638BD054B1D600029E5D1E3E700BFA9
:10C5500041A0FF1F589EFF1F5C9EFF1F549EFF1FA0
:10C56000704700BF704700BF704700BF054A064BC9
:10C5700010781B78C0B2DBB2984238BF4030C01A86
:10C58000704700BF48A0FF1F49A0FF1FF0B4384B01
:10C590001A7912F0300F2CD072B6997D01F0FF029B
:10C5A00000293DD062B6334F334938780D78334E89
:10C5B0001C46C0B2EDB2431C402BE17928BF0023DA
:10C5C000AB4202F1FF32C9B21CBFF154184612F05F
:10C5D000FF02F0D12A4B1B68C2B23A704BB1A8429D
:10C5E00036BFC5F14005401B40192728C4BF0122B2
:10C5F0001A701F49CA78D2B2150616D452060DD544
:10C600001B4B1B795B0609D51E4B1F491B6800227B
:10C610000A7003B11A70164B3C22DA70F0BC7047F6
:10C620004022D9795A7462B6E3E70B791C06E5D546
:10C63000164B174E1C783378E4B2DBB29C420ED016
:10C64000144D01E0A3420AD00133402B28BF002340
:10C650000879E85CC0B2C871087D0728F2D9DBB25E
:10C66000034933700B79180644BF7C23CB70C5E7B0
:10C6700000A0064048A0FF1F49A0FF1F8CA0FF1F7D
:10C6800044A0FF1FD0A0FF1FCCA0FF1FD4A0FF1FFE
:10C69000CDA0FF1F4CA0FF1F054A064B10781B784A
:10C6A000C0B2DBB2984238BF4030C01A704700BFFA
:10C6B00048A1FF1FDDA0FF1FF0B4384B1A7912F01C
:10C6C000300F2CD072B6997D01F0FF0200293DD0C9
:10C6D00062B6334F334938780D78334E1C46C0B2BA
:10C6E000EDB2431C402BE17928BF0023AB4202F19D
:10C6F000FF32C9B21CBFF154184612F0FF02F0D14C
:10C700002A4B1B68C2B23A704BB1A84236BFC5F182
:10C710004005401B40192728C4BF01221A701F4939
:10C72000CA78D2B2150616D452060DD51B4B1B790A
:10C730005B0609D51E4B1F491B6800220A7003B116
:10C740001A70164B3C22DA70F0BC70474022D9793F
:10C750005A7462B6E3E70B791C06E5D5164B174E03
:10C760001C783378E4B2DBB29C420ED0144D01E069
:10C77000A3420AD00133282B28BF00230879E85CA4
:10C78000C0B2C871087D0728F2D9DBB20349337003
:10C790000B79180644BF7C23CB70C5E700B0064078
:10C7A00048A1FF1FDDA0FF1F08A1FF1FD8A0FF1F8A
:10C7B0004CA1FF1FDCA0FF1F50A1FF1F49A1FF1FBD
:10C7C000E0A0FF1F70B584B072B6194B194D1A481E
:10C7D000702241260F2480211A702E701A46047090
:10C7E000197013781B06FCD5144B186862B6144BED
:10C7F000144C984298BF00EB800001A998BF4000FC
:10C800000A22FDF7CFFE01A92046002311F8012BD3
:10C8100001333AB10A2B20F8022FF7D116232370E7
:10C8200004B070BD5B00DBB2237004B070BD00BF0C
:10C8300000000240070002400600024008000240DB
:10C840007F9698009C92FF1F2DE9F043DFF8EC8063
:10C850008BB006460F4600F073F898F900300133AC
:10C8600004460D4637D03046394600F0DFF900283F
:10C8700031D02BA3D3E900233046394600F026FE01
:10C88000814668BB28A3D3E900233046394600F02F
:10C89000FFFD00B398F90030254ACDF8209004241C
:10C8A00000200021022BCDE90467CDE90267009446
:10C8B0000192CDE906012CD0684600F0BDF940B3E5
:10C8C000089B1BB101F0AAF9089B0360DDE9060192
:10C8D0000BB0BDE8F083204629460BB0BDE8F083DD
:10C8E000134A98F90030019203210022CDE9046730
:10C8F000CDE90267009108922BB90E4B4FF06042D0
:10C90000CDE90623D8E70C490020022BCDE906012A
:10C91000D2D101F083F922230360D1E7AFF3008085
:10C92000EF39FAFE422E864051302DD5104987C08E
:10C93000900A0100FFFFEF470000F07FB292FF1F57
:10C940002DE9F04FB04F21F00042BA4283B00C46BF
:10C950004FEAD17605460DD9AC4FBA4225D9C1F37D
:10C960001303034340F0EF800EB10020014603B0F3
:10C97000BDE8F08FA64B9A4200F2CC80A54B9A42BC
:10C9800000F2DE808AA3D3E9002300F05DF90022E3
:10C99000A14B00F09BFD002800F0058128462146B0
:10C9A00000229D4B00F050F9E1E783A3D3E9002377
:10C9B00000F08CFD002840F0CB802846214680A363
:10C9C000D3E9002300F064FD0028CED1934B284624
:10C9D00003EBC60821467CA3D3E9002300F0E6FA66
:10C9E000D8E9002300F030F900F07AFD804600F02D
:10C9F00077FA77A3D3E9002306460F4600F0D6FA6C
:10CA000002460B462846214600F01CF972A3D3E9E2
:10CA10000023CDE900013046394600F0C7FA8246CE
:10CA20008B4652465B46DDE9000100F00BF90546F6
:10CA30000C462A4623462846214600F0B7FA68A34A
:10CA4000D3E9002306460F4600F0B0FA66A3D3E907
:10CA5000002300F0F7F832463B4600F0A7FA64A343
:10CA6000D3E9002300F0F0F832463B4600F09EFA8E
:10CA700061A3D3E9002300F0E5F832463B4600F01D
:10CA800095FA5FA3D3E9002300F0DEF832463B4677
:10CA900000F08CFA02460B462846214600F0D2F8F8
:10CAA00006460F462846214632463B46B8F1000F5F
:10CAB00056D000F07BFA324604460D463B46002035
:10CAC0004FF0804100F0BEF802460B462046294652
:10CAD00000F096FB02460B465046594600F0B2F86D
:10CAE000DDE9002300F0AEF80B4602464A4900207B
:10CAF00000F0A8F86FF47F7398454FDA08F57A785C
:10CB000001EB085100224FF0B87300F04FFA03B068
:10CB1000BDE8F08F424B9A423FF658AF414BF400CC
:10CB20002344D3E9002300F08DF83F4BC6F1010800
:10CB30001C44CDE90001D4E900ABC6EB080870E75E
:10CB40004FF0000875E702460B4600F07DF80EE74F
:10CB500017A3D3E900231046194600F027FA06E789
:10CB600000F024FA0022804689464FF08043304688
:10CB7000394600F067F802460B464046494600F049
:10CB80003FFB2A46234600F05DF802460B46002094
:10CB9000214900F057F803B0BDE8F08F01EB0851D0
:10CBA00003B0BDE8F08F804643E700BFAFF30080DD
:10CBB0009C7500883CE4377EEF39FAFE422E8640B1
:10CBC00051302DD5104987C0FE822B654715F73FA0
:10CBD0000000E0FE422EE63F763C7935EF39EA3D33
:10CBE000D0A4BE726937663EF16BD2C541BDBB3E73
:10CBF0002CDE25AF6A56113F93BDBE166CC1663F51
:10CC00003E5555555555C53F412E8640FFFFEF7F98
:10CC1000422ED63FFFFF2F3E0000F03F980A010052
:10CC2000B1A2F03FB80A0100A80A010041F000419A
:10CC300001F58010C00F70470020704781F000415F
:10CC400002E000BF83F0004330B54FEA41044FEAF1
:10CC5000430594EA050F08BF90EA020F1FBF54EA8C
:10CC6000000C55EA020C7FEA645C7FEA655C00F028
:10CC7000E2804FEA5454D4EB5555B8BF6D420CDDF9
:10CC80002C4480EA020281EA030382EA000083EA7C
:10CC9000010180EA020281EA0303362D88BF30BD1C
:10CCA00011F0004F4FEA01314FF4801C4CEA113172
:10CCB00002D0404261EB410113F0004F4FEA0333D1
:10CCC0004CEA133302D0524263EB430394EA050F5C
:10CCD00000F0A780A4F10104D5F1200E0DDB02FACB
:10CCE0000EFC22FA05F2801841F1000103FA0EF25F
:10CCF000801843FA05F359410EE0A5F120050EF125
:10CD0000200E012A03FA0EFC28BF4CF0020C43FA55
:10CD100005F3C01851EBE37101F0004507D54FF062
:10CD2000000EDCF1000C7EEB00006EEB0101B1F5B2
:10CD3000801F1BD3B1F5001F0CD349085FEA3000F8
:10CD40004FEA3C0C04F101044FEA445212F5800F03
:10CD500080F09A80BCF1004F08BF5FEA500C50F1A0
:10CD6000000041EB045141EA050130BD5FEA4C0C83
:10CD7000404141EB010111F4801FA4F10104E9D10C
:10CD800091F0000F04BF01460020B1FA81F308BF03
:10CD90002033A3F10B03B3F120020CDA0C3208DDCF
:10CDA00002F1140CC2F10C0201FA0CF021FA02F1AA
:10CDB0000CE002F11402D8BFC2F1200C01FA02F11A
:10CDC00020FA0CFCDCBF41EA0C019040E41AA2BF3F
:10CDD00001EB0451294330BD6FEA04041F3C1CDA07
:10CDE0000C340EDC04F11404C4F1200220FA04F027
:10CDF00001FA02F340EA030021FA04F345EA0301D1
:10CE000030BDC4F10C04C4F1200220FA02F001FA92
:10CE100004F340EA0300294630BD21FA04F0294614
:10CE200030BD94F0000F83F4801306BF81F48011AD
:10CE30000134013D4EE77FEA645C18BF7FEA655C20
:10CE400029D094EA050F08BF90EA020F05D054EAF2
:10CE5000000C04BF1946104630BD91EA030F1EBFF7
:10CE60000021002030BD5FEA545C05D140004941FB
:10CE700028BF41F0004130BD14F580043CBF01F5EE
:10CE8000801130BD01F0004545F0FE4141F47001D4
:10CE90004FF0000030BD7FEA645C1ABF19461046AF
:10CEA0007FEA655C1CBF0B46024650EA013406BFB0
:10CEB00052EA033591EA030F41F4002130BD00BF6F
:10CEC00090F0000F04BF0021704730B54FF480642C
:10CED00004F132044FF000054FF0000150E700BFAD
:10CEE00090F0000F04BF0021704730B54FF480640C
:10CEF00004F1320410F0004548BF40424FF00001F9
:10CF00003EE700BF42004FEAE2014FEA31014FEA3B
:10CF100002701FBF12F07F4393F07F4F81F060518A
:10CF2000704792F0000F14BF93F07F4F704730B5F9
:10CF30004FF4607401F0004521F0004120E700BF8C
:10CF400050EA010208BF704730B54FF000050AE013
:10CF500050EA010208BF704730B511F0004502D514
:10CF6000404261EB41014FF4806404F132045FEA16
:10CF7000915C3FF4DCAE4FF003025FEADC0C18BFBB
:10CF800003325FEADC0C18BF033202EBDC02C2F1B1
:10CF9000200300FA03FC20FA02F001FA03FE40EA43
:10CFA0000E0021FA02F11444C1E600BF70B54FF043
:10CFB000FF0C4CF4E06C1CEA11541DBF1CEA135525
:10CFC00094EA0C0F95EA0C0F00F0DEF82C4481EA8D
:10CFD000030621EA4C5123EA4C5350EA013518BFAD
:10CFE00052EA033541F4801143F4801338D0A0FB9A
:10CFF00002CE4FF00005E1FB02E506F00042E0FB47
:10D0000003E54FF00006E1FB03569CF0000F18BF4C
:10D010004EF0010EA4F1FF04B6F5007F64F54074F4
:10D0200004D25FEA4E0E6D4146EB060642EAC62187
:10D0300041EA55514FEAC52040EA5E504FEACE2EF4
:10D04000B4F1FD0C88BFBCF5E06F1ED8BEF1004FF7
:10D0500008BF5FEA500E50F1000041EB045170BD73
:10D0600006F0004646EA010140EA020081EA0301B7
:10D07000B4EB5C04C2BFD4EB0C0541EA045170BDB3
:10D0800041F480114FF0000E013C00F3AB8014F12D
:10D09000360FDEBF002001F0004170BDC4F1000476
:10D0A000203C35DA0C341BDC04F11404C4F12005F7
:10D0B00000FA05F320FA04F001FA05F240EA020052
:10D0C00001F0004221F0004110EBD37021FA04F688
:10D0D00042EB06015EEA430E08BF20EAD37070BD42
:10D0E000C4F10C04C4F1200500FA04F320FA05F0A1
:10D0F00001FA04F240EA020001F0004110EBD370A3
:10D1000041F100015EEA430E08BF20EAD37070BD12
:10D11000C4F1200500FA05F24EEA020E20FA04F3EB
:10D1200001FA05F243EA020321FA04F001F000419A
:10D1300021FA04F220EA020000EBD3705EEA430E0B
:10D1400008BF20EAD37070BD94F0000F0FD101F03A
:10D150000046400041EB010111F4801F08BF013C73
:10D16000F7D041EA060195F0000F18BF704703F0B1
:10D170000046520043EB030313F4801F08BF013D38
:10D18000F7D043EA0603704794EA0C0F0CEA1355F4
:10D1900018BF95EA0C0F0CD050EA410618BF52EAAE
:10D1A0004306D1D181EA030101F000414FF00000B4
:10D1B00070BD50EA410606BF1046194652EA4306C2
:10D1C00019D094EA0C0F02D150EA013613D195EA36
:10D1D0000C0F05D152EA03361CBF104619460AD17E
:10D1E00081EA030101F0004141F0FE4141F4700188
:10D1F0004FF0000070BD41F0FE4141F4780170BD78
:10D2000070B54FF0FF0C4CF4E06C1CEA11541DBFDC
:10D210001CEA135594EA0C0F95EA0C0F00F0A7F8DE
:10D22000A4EB050481EA030E52EA03354FEA01310B
:10D2300000F088804FEA03334FF0805545EA13131E
:10D2400043EA12634FEA022245EA111545EA1065E6
:10D250004FEA00260EF000419D4208BF964244F17D
:10D26000FD0404F5407402D25B084FEA3202B61A9C
:10D2700065EB03055B084FEA32024FF480104FF470
:10D28000002CB6EB020E75EB030E22BFB61A7546E4
:10D2900040EA0C005B084FEA3202B6EB020E75EB77
:10D2A000030E22BFB61A754640EA5C005B084FEADF
:10D2B0003202B6EB020E75EB030E22BFB61A7546AC
:10D2C00040EA9C005B084FEA3202B6EB020E75EBB7
:10D2D000030E22BFB61A754640EADC0055EA060E78
:10D2E00018D04FEA051545EA16754FEA06164FEABB
:10D2F000C30343EA52734FEAC2025FEA1C1CC0D167
:10D3000011F4801F0BD141EA00014FF000004FF0F3
:10D31000004CB6E711F4801F04BF01430020B4F1B4
:10D32000FD0C88BFBCF5E06F3FF6AFAEB5EB030C6C
:10D3300004BFB6EB020C5FEA500C50F1000041EB69
:10D34000045170BD0EF0004E4EEA113114EB5C0436
:10D35000C2BFD4EB0C0541EA045170BD41F4801109
:10D360004FF0000E013C90E645EA060E8DE60CEA11
:10D37000135594EA0C0F08BF95EA0C0F3FF43BAF2E
:10D3800094EA0C0F0AD150EA01347FF434AF95EAE5
:10D390000C0F7FF425AF104619462CE795EA0C0FC9
:10D3A00006D152EA03353FF4FDAE1046194622E796
:10D3B00050EA410618BF52EA43067FF4C5AE50EA70
:10D3C00041047FF40DAF52EA43057FF4EBAE12E760
:10D3D0004FF0FF3C06E000BF4FF0010C02E000BF41
:10D3E0004FF0010C4DF804CD4FEA410C7FEA6C5C24
:10D3F0004FEA430C18BF7FEA6C5C1BD001B050EAC7
:10D40000410C0CBF52EA430C91EA030F02BF90EAB1
:10D41000020F0020704710F1000F91EA030F58BF70
:10D42000994208BF90422CBFD8176FEAE37040F0D2
:10D43000010070474FEA410C7FEA6C5C02D150EA70
:10D44000013C07D14FEA430C7FEA6C5CD6D152EA2B
:10D45000033CD3D05DF8040B704700BF84461046F0
:10D4600062468C461946634600E000BF01B5FFF7EF
:10D47000B7FF002848BF10F1000F01BD4DF808EDBF
:10D48000FFF7F4FF0CBF012000205DF808FB00BF90
:10D490004DF808EDFFF7EAFF34BF012000205DF8EA
:10D4A00008FB00BF4DF808EDFFF7E0FF94BF012037
:10D4B00000205DF808FB00BF4DF808EDFFF7CEFF38
:10D4C00094BF012000205DF808FB00BF4DF808ED77
:10D4D000FFF7C4FF34BF012000205DF808FB00BF48
:10D4E0004FEA410212F5001215D211D56FF478738C
:10D4F000B3EB625212D94FEAC12343F0004343EA2F
:10D50000505311F0004F23FA02F018BF4042704709
:10D510004FF00000704750EA013005D111F0004093
:10D5200008BF6FF0004070474FF00000704700BF29
:10D530004FEA4102B2F1E04324BFB3F5001CDCF135
:10D54000FE5C0DD901F0004C4FEAC0024CEA50706D
:10D55000B2F1004F40EB830008BF20F0010070479C
:10D5600011F0804F21D113F13872BCBF01F000409F
:10D57000704741F480114FEA5252C2F11802C2F1D1
:10D58000200C10FA0CF320FA02F018BF40F0010052
:10D590004FEAC1234FEAD32303FA0CFC40EA0C0004
:10D5A00023FA02F34FEA4303CCE77FEA625307D141
:10D5B00050EA01331EBF4FF0FE4040F44000704778
:10D5C00001F0004040F0FE4040F40000704700BF12
:10D5D00080F0004002E000BF81F0004142001FBF28
:10D5E0005FEA410392EA030F7FEA226C7FEA236C31
:10D5F0006AD04FEA1262D2EB1363C1BFD218414026
:10D6000048404140B8BF5B42192B88BF704710F0BB
:10D61000004F40F4000020F07F4018BF404211F05E
:10D62000004F41F4000121F07F4118BF494292EAC6
:10D63000030F3FD0A2F1010241FA03FC10EB0C00F2
:10D64000C3F1200301FA03F100F0004302D549427F
:10D6500060EB4000B0F5000F13D3B0F1807F06D32C
:10D6600040084FEA310102F10102FE2A51D2B1F124
:10D67000004F40EBC25008BF20F0010040EA030019
:10D680007047490040EB000010F4000FA2F10102C6
:10D69000EDD1B0FA80FCACF1080CB2EB0C0200FA50
:10D6A0000CF0AABF00EBC25052421843BCBFD0409E
:10D6B0001843704792F0000F81F4000106BF80F418
:10D6C00000000132013BB5E74FEA41037FEA226CDB
:10D6D00018BF7FEA236C21D092EA030F04D092F0A6
:10D6E000000F08BF0846704790EA010F1CBF0020DA
:10D6F000704712F07F4F04D1400028BF40F0004037
:10D70000704712F100723CBF00F50000704700F056
:10D71000004343F0FE4040F4000070477FEA22627D
:10D7200016BF08467FEA23630146420206BF5FEA4E
:10D73000412390EA010F40F4800070474FF000034E
:10D7400004E000BF10F0004348BF40425FEA000C15
:10D7500008BF704743F0964301464FF000001CE0BD
:10D7600050EA010208BF70474FF000030AE000BF13
:10D7700050EA010208BF704711F0004302D5404251
:10D7800061EB41015FEA010C02BF844601460020C3
:10D7900043F0B64308BFA3F18053A3F50003BCFADE
:10D7A0008CF2083AA3EBC25310DB01FA02FC63448B
:10D7B00000FA02FCC2F12002BCF1004F20FA02F292
:10D7C00043EB020008BF20F00100704702F1200285
:10D7D00001FA02FCC2F1200250EA4C0021FA02F2E6
:10D7E00043EB020008BF20EADC7070474FF0FF0CEB
:10D7F0001CEAD0521EBF1CEAD15392EA0C0F93EAE6
:10D800000C0F6FD01A4480EA010C400218BF5FEA87
:10D8100041211ED04FF0006343EA501043EA5111FA
:10D82000A0FB01310CF00040B1F5000F3EBF4900F4
:10D8300041EAD3715B0040EA010062F17F02FD2AF8
:10D840001DD8B3F1004F40EBC25008BF20F00100DB
:10D85000704790F0000F0CF0004C08BF49024CEAF2
:10D86000502040EA51207F3AC2BFD2F1FF0340EA84
:10D87000C250704740F400004FF00003013A5DDCF5
:10D8800012F1190FDCBF00F000407047C2F1000236
:10D89000410021FA02F1C2F1200200FA02FC5FEA23
:10D8A000310040F1000053EA4C0308BF20EADC706D
:10D8B000704792F0000F00F0004C02BF400010F4DF
:10D8C000000F013AF9D040EA0C0093F0000F01F08C
:10D8D000004C02BF490011F4000F013BF9D041EAAE
:10D8E0000C018FE70CEAD15392EA0C0F18BF93EAB0
:10D8F0000C0F0AD030F0004C18BF31F0004CD8D1DA
:10D9000080EA010000F00040704790F0000F17BF60
:10D9100090F0004F084691F0000F91F0004F14D0A6
:10D9200092EA0C0F01D142020FD193EA0C0F03D1FE
:10D930004B0218BF084608D180EA010000F0004001
:10D9400040F0FE4040F40000704740F0FE4040F4DC
:10D95000400070474FF0FF0C1CEAD0521EBF1CEA7B
:10D96000D15392EA0C0F93EA0C0F69D0A2EB030299
:10D9700080EA010C49024FEA402037D04FF0805333
:10D9800043EA111143EA10130CF000408B4238BFF8
:10D990005B0042F17D024FF4000C8B4224BF5B1A06
:10D9A00040EA0C00B3EB510F24BFA3EB510340EA54
:10D9B0005C00B3EB910F24BFA3EB910340EA9C0002
:10D9C000B3EBD10F24BFA3EBD10340EADC001B0172
:10D9D00018BF5FEA1C1CE0D1FD2A3FF650AF8B4216
:10D9E00040EBC25008BF20F0010070470CF0004C23
:10D9F0004CEA50207F32C2BFD2F1FF0340EAC2504E
:10DA0000704740F400004FF00003013A37E792F00E
:10DA1000000F00F0004C02BF400010F4000F013A6C
:10DA2000F9D040EA0C0093F0000F01F0004C02BF67
:10DA3000490011F4000F013BF9D041EA0C0195E7D0
:10DA40000CEAD15392EA0C0F08D142027FF47DAF69
:10DA500093EA0C0F7FF470AF084676E793EA0C0F59
:10DA600004D14B023FF44CAF08466EE730F0004C57
:10DA700018BF31F0004CCAD130F000427FF45CAFE7
:10DA800031F000437FF43CAF5FE700BF4FF0FF3C55
:10DA900006E000BF4FF0010C02E000BF4FF0010CA8
:10DAA0004DF804CD4FEA40024FEA41037FEA226C71
:10DAB00018BF7FEA236C11D001B052EA530C18BF93
:10DAC00090EA010F58BFB2EB030088BFC81738BFF8
:10DAD0006FEAE17018BF40F0010070477FEA226CE6
:10DAE00002D15FEA402C05D17FEA236CE4D15FEAE2
:10DAF000412CE1D05DF8040B704700BF8446084616
:10DB00006146FFE70FB5FFF7C9FF002848BF10F1D6
:10DB1000000F0FBD4DF808EDFFF7F4FF0CBF01201B
:10DB200000205DF808FB00BF4DF808EDFFF7EAFFA5
:10DB300034BF012000205DF808FB00BF4DF808ED60
:10DB4000FFF7E0FF94BF012000205DF808FB00BF55
:10DB50004DF808EDFFF7D2FF94BF012000205DF8DB
:10DB600008FB00BF4DF808EDFFF7C8FF34BF0120E8
:10DB700000205DF808FB00BF4FEA4002B2F1FE4F03
:10DB80000FD34FF09E03B3EB12620DD94FEA00237F
:10DB900043F0004310F0004F23FA02F018BF404258
:10DBA00070474FF00000704712F1610F01D142023F
:10DBB00005D110F0004008BF6FF0004070474FF0F3
:10DBC0000000704742000ED2B2F1FE4F0BD34FF06F
:10DBD0009E03B3EB126209D44FEA002343F00043E3
:10DBE00023FA02F070474FF00000704712F1610F06
:10DBF00001D1420202D14FF0FF3070474FF00000D8
:10DC0000704700BF0B460146184600F001B800BF40
:10DC100013460A460146022000F0C4BE014B1868B4
:10DC2000704700BFE096FF1F70B50F4E0F4D761B7B
:10DC3000B61018BF002405D0013455F8043B9847AE
:10DC4000A642F9D10A4E0B4D761B02F03FFFB610EB
:10DC500018BF002406D0013455F8043B9847A6426B
:10DC6000F9D170BD70BD00BFD80A0100D80A01000B
:10DC7000EC0A0100D80A0100024B0146186800F0C6
:10DC80000BB800BFE096FF1F024B0146186800F07A
:10DC90004DBF00BFE096FF1F2DE9F04F01F10B05CE
:10DCA000162D83B0064640F29F8035F0070500F13F
:10DCB000BF80A94200F2BC8000F058FBB5F5FC7FA4
:10DCC000C0F09C826B0A00F0BA80042B00F28381C2
:10DCD000A80900F1390E4FEA4E033830C44F07EB64
:10DCE0008303A3F108015C68A14207D1ACE0002ADC
:10DCF00080F2AC80E468A14200F0A680636823F063
:10DD000003035A1B0F2AF2DDB9493C6901F1080EE1
:10DD1000744500F0B381636823F003035A1B0F2A94
:10DD200000F39981002AC1F814E0C1F810E080F2F4
:10DD30009E80B3F5007F80F06781DB0803F1010C62
:10DD400001229B1002FA03F34A6851F83C80C4F8A0
:10DD5000088001EBCC091A43A9F10803E3604A608B
:10DD600041F83C40C8F80C40831001249C40944288
:10DD700000F28A80144206D120F0030064001442AD
:10DD800000F10400FAD007EBC009CC468046DCF86D
:10DD90000C108C4507D173E1002A80F28181C9689B
:10DDA0008C4500F06D814B6823F003035A1B0F2A4A
:10DDB000F2DD0C46D1F80CC054F8088F4B1945F031
:10DDC00001054D6042F00101C8F80CC03046CCF8A6
:10DDD00008807B613B61C3F80CE0C3F808E0596040
:10DDE0009A5000F0C5FA1FE0102921D800F0BEFAC1
:10DDF0001025062302207E4F07EB8303A3F10802C0
:10DE00005C68944200F045816368E168A56823F08E
:10DE10000303234430465A68E96042F001028D60F2
:10DE20005A6000F0A5FA0834204603B0BDE8F08F30
:10DE300000240C232046336003B0BDE8F08F80231C
:10DE40004FF0400E3F2049E770465DE72344E1680C
:10DE50005A68A56842F00102E96030468D605A6058
:10DE600000F086FA0834204603B0BDE8F08F234462
:10DE700030465A6842F001025A6000F079FA0834DC
:10DE8000204603B0BDE8F08FBC68636823F0030848
:10DE9000A84504D3C5EB08030F2B00F38C80554B2A
:10DEA000DFF860911A68D9F8003001332A4404EB96
:10DEB000080A00F0608102F580520F3222F47F627E
:10DEC00022F00F0211463046019200F04BFCB0F1F7
:10DED000FF3F8346019A00F05881824500F2FC80A2
:10DEE000454B1968DA451144196000F05381D9F89F
:10DEF0000000DFF810E101301BBFCAEB0B0A5144F0
:10DF0000CEF800B019601BF0070100F01781C1F1D5
:10DF10000800C1F58051834408315A44C2F30B0212
:10DF2000C2EB010949463046019300F01BFC431C3B
:10DF3000019B00F03F81CBEB00024A4442F001021A
:10DF40001968C7F808B04944BC42CBF804201960EE
:10DF5000DFF8A49016D0B8F10F0F40F2FD80626890
:10DF6000A8F10C0323F00703E01802F001024FF0C0
:10DF7000050E1A430F2B6260C0F804E0C0F808E0F9
:10DF800000F21C811D4BBC681A68914288BF196061
:10DF90001B4B1A689142626888BF196022F0030225
:10DFA0009542A2EB050301D80F2B04DC304600F0AC
:10DFB000DFF9002438E7621943F0010345F0010559
:10DFC00065603046BA60536000F0D2F908342046EC
:10DFD00003B0BDE8F08F142B71D9542B00F2A4804C
:10DFE000280B00F16F0E4FEA4E036E3076E600BF4D
:10DFF000E496FF1F5CA1FF1F60A1FF1F58A1FF1F38
:10E0000054A1FF1FF09AFF1F5A0A042A5ED9142A4E
:10E0100000F2B38002F15C0149005B3207EB810C36
:10E0200057F82110DFF8DC81ACF1080C8C4500F0CA
:10E0300088804A6822F00302934202D289688C45A4
:10E04000F7D1D1F80CC07A68C4F80CC0A160CCF844
:10E050000840CC6088E6631942F0010745F00105ED
:10E06000656030464B610B61C3F80CE0C3F808E013
:10E070005F609A50083400F07BF9D5E64A6873E691
:10E0800008F1010818F0030F0CF1080C7FF47FAEC3
:10E0900030E0DC68A34208BF02303FF435AEB3E69F
:10E0A0000B440C465A68C96854F8085F42F00102F4
:10E0B0005A603046E9608D6000F05AF9B4E603F129
:10E0C0005C0E03F15B004FEA4E0307E69A0902F18A
:10E0D000390149003832A1E7BC424A4B3FF400AF56
:10E0E0009C68626822F003025AE759F8083999459A
:10E0F00040F0828010F0030F00F1FF30F5D17B6813
:10E1000023EA04037B6064009C423FF6BDAE002C12
:10E110003FF4BAAE1C4240467FF435AE64001C4268
:10E1200000F10400FAD02EE6B3F5AA7F18D8E80B68
:10E1300000F1780E4FEA4E037730CFE54FF480516F
:10E14000EBE60121D8F80430921001FA02F21A43EA
:10E15000C8F80420614677E70123CBF8043025E7AF
:10E1600040F25452934220D8A80C00F17D0E4FEAA1
:10E170004E037C30B2E51032A4E6542A26D81A0B9E
:10E1800002F16F0149006E3248E7BC68626822F014
:10E19000030205E7CAF30B0000287FF4A8AE42444F
:10E1A000BB6842F001025A60ECE6FE234FF07F0E9E
:10E1B0007E2093E501224FF00009C1E604F1080139
:10E1C000304600F0B3FCD9F80010DBE6B2F5AA7FC8
:10E1D00005D8DA0B02F17801490077321EE740F2E8
:10E1E00054518A4205D89A0C02F17D0149007C32D3
:10E1F00014E7FE217E2211E77B6884E7E808431CD0
:10E200005B00F8E5E496FF1F8842F0B50DD98B1846
:10E2100098420AD28118002A51D09A1A13F8014D57
:10E2200001F8014D9342F9D1F0BD0F2A48D941EAD6
:10E2300000039B0746D100F1100401F110031546BD
:10E2400053F8106C44F8106C53F80C6C44F80C6CD8
:10E2500053F8086C44F8086C103D53F8046C44F80B
:10E26000046C0F2D03F1100304F11004E8D8A2F19F
:10E27000100323F00F0302F00F0E1033BEF1030F53
:10E280001944034421D91E1F0D467446043C55F819
:10E29000047B46F8047F032CF8D8AEF1040424F084
:10E2A000030404342344214402F0030262B1013B1D
:10E2B0000A4411F8014B03F8014F8A42F9D1F0BD2D
:10E2C0000346F3E70346F2E7F0BD7246EEE700BF10
:10E2D00070B4840746D0541E002A41D0CDB2034604
:10E2E00002E0621EE4B3144603F8015B9A07F8D11A
:10E2F000032C2ED9CDB245EA05250F2C45EA05455C
:10E3000019D903F110022646103E0F2E42F8105C78
:10E3100042F80C5C42F8085C42F8045C02F110021E
:10E32000F2D8A4F1100222F00F0204F00F04103210
:10E33000032C13440DD91E462246043A032A46F8FC
:10E34000045BFAD8221F22F003020432134404F0C3
:10E3500003042CB1C9B21C4403F8011BA342FBD136
:10E3600070BC704714460346C2E700BF704700BF49
:10E37000704700BF024B0A460146186800F002B819
:10E38000E096FF1F2DE9F04F174683B0002900F0FB
:10E39000C1800E46814607F10B05FFF7E7FF56F8EF
:10E3A00004EC162D2EF00304A6F1080840D8102224
:10E3B0001546AF4241D8944275DAC94B996808EBCB
:10E3C00004008842416800F0D98021F00103034431
:10E3D0005B68DB077DD51EF0010F35D03946484616
:10E3E000FFF75AFC0746E0B156F8043C23F001035E
:10E3F0004344A0F108029A4200F04481221F242ADB
:10E4000000F23181132A00F204810346324611687A
:10E4100019605168596092689A603146484600F028
:10E4200085FB4846FFF7A4FF384603B0BDE8F08FF0
:10E4300025F00705002D2A46BBDA0C230020C9F879
:10E44000003003B0BDE8F08F56F8083CC3EB080A73
:10E45000DAF8043023F0030C04EB0C039342BDDB29
:10E460005746DAF80C1057F8080F221F242AC1600B
:10E47000886000F21781132A40F212813168CAF8CD
:10E4800008107168CAF80C101B2A00F22B8108369C
:10E490000AF110023168116071685160B1689160D1
:10E4A0003E461C46D046631B0F2B1DD8D8F80430BF
:10E4B00003F0010323434444C8F80430636843F085
:10E4C000010363604846FFF753FF304603B0BDE8E1
:10E4D000F08F21F003012144914221DBC36882685F
:10E4E0000C46D3609A60DEE7D8F8042008EB0501FB
:10E4F00002F00102154343F001020B44C8F8045036
:10E500004A605A6842F0010208315A60484600F0F9
:10E510000DFBD7E7114603B0BDE8F04FFFF7BCBBDA
:10E520001EF0010F7FF45AAF56F8083CC3EB080AFF
:10E53000DAF8043023F0030C01EB0C0E96458BDB6C
:10E54000C36882685746D3609A6057F8081FDAF8A4
:10E550000C30CB60221F242A996000F29980132A84
:10E5600062D93368CAF808307368CAF80C301B2ABD
:10E5700000F2A08008360AF1100356E021F0030BE8
:10E58000A34405F11000834559DA1EF0010F7FF412
:10E5900025AF56F8081CC1EB080ADAF8041021F080
:10E5A000030CE34458453FF757AF5746DAF80C10D1
:10E5B00057F8080F221F242AC160886000F2B48037
:10E5C000132A40F2A5803168CAF808107168CAF8A9
:10E5D0000C101B2A00F2AF8008360AF110023168D5
:10E5E000116071685160B16891600AEB0501C5EB7B
:10E5F0000B0242F0010299604A60DAF8043003F03D
:10E6000001031D434846CAF80450FFF7B1FE3846DF
:10E610005CE733680360736843601B2A27D800F106
:10E62000080306F10802F2E63B4632681A60726897
:10E630005A60B2689A603E467446D04633E708EBAB
:10E640000501C5EB0B0B4BF0010299604A6056F8CF
:10E65000043C03F001031D43484646F8045CFFF701
:10E6600087FE304632E73146FFF7CEFDD5E6B36888
:10E670008360F368C360242A28D000F1100306F1F8
:10E680001002C4E650F8043C23F003031C440AE7DC
:10E69000314638467446D046FFF7B6FD3E4602E79F
:10E6A0003A46F7E6314638461C46D046FFF7ACFD01
:10E6B0003E46F8E6B368CAF81030F368CAF814307A
:10E6C000242A1BD010360AF11803AEE73369036120
:10E6D0007369436106F1180200F1180397E600BF61
:10E6E000E496FF1FB168CAF81010F168CAF8141058
:10E6F000242A0FD010360AF11802CBE63369CAF883
:10E7000018307369CAF81C3018360AF120038CE7F8
:10E710003A4664E73269CAF818207269CAF81C20C0
:10E7200018360AF12002B5E6314638460193FFF764
:10E730006BFD019B59E7B168CAF81010F168CAF87F
:10E740001410242A03D010360AF1180247E7326960
:10E75000CAF818207269CAF81C2018360AF120027B
:10E760003DE700BF38B5074C002305460846236047
:10E77000FBF7E2FE431C00D038BD2368002BFBD022
:10E780002B6038BDBCA2FF1FFFFFFFFFFFFFFFFF95
:10E79000FFFFFFFFFFFFFFFFFFFFFFFFFFFFFFFF89
:10E7A000FFFFFFFFFFFFFFFFFFFFFFFFFFFFFFFF79
:10E7B000FFFFFFFFFFFFFFFFFFFFFFFFFFFFFFFF69
:10E7C00090F800F06DE9024520F007016FF0000CB1
:10E7D00010F0070491F820F040F049804FF0000459
:10E7E0006FF00700D1E9002391F840F000F1080034
:10E7F00082FA4CF2A4FA8CF283FA4CF3A2FA8CF36C
:10E800004BBBD1E9022382FA4CF200F10800A4FAD2
:10E810008CF283FA4CF3A2FA8CF3E3B9D1E9042326
:10E8200082FA4CF200F10800A4FA8CF283FA4CF35D
:10E83000A2FA8CF37BB9D1E9062301F1200182FA17
:10E840004CF200F10800A4FA8CF283FA4CF3A2FA1D
:10E850008CF3002BC6D0002A04BF04301A4612BA2B
:10E86000B2FA82F2FDE8024500EBD2007047D1E92E
:10E87000002304F00305C4F100004FEAC50514F0BD
:10E88000040F91F840F00CFA05F562EA05021CBF8E
:10E8900063EA050362464FF00004A9E7002A41D06D
:10E8A00040EA010313F00303F0B425D1032A23D96E
:10E8B00004680D68AC421FD1043A35D0A4F101358B
:10E8C00025EA040414F0803F31D1071D0D1D0DE031
:10E8D00057F8043B0E68A3F10134B34224EA030461
:10E8E0000AD1043A20D014F0803F23D1032A2946CC
:10E8F000384605F10405EBD803780C789C4202F108
:10E90000FF320CD182B114B916E06AB17BB110F8B4
:10E91000013F11F8014FA34202F1FF32F5D0181B5D
:10E92000F0BC7047104670471046F0BC7047184660
:10E93000F0BC70470020F3E72046F1E740EA01030E
:10E940009B0770B42BD1032A29D90C4603462146D4
:10E9500054F8046BA6F1013525EA060515F0803F51
:10E9600006D1043A032A43F8046B2146EFD8A2B13A
:10E970000C781C70013A013301313CB16AB111F8D5
:10E98000014B03F8014B013A002CF7D12AB11A448C
:10E99000002103F8011B9A42FBD170BC704703466B
:10E9A000E5E700BF2DE9F047254C2568D5F848413B
:10E9B0000646884692469946C4B360681F2817DC0D
:10E9C000431C76B104EB80050122C5F888A0D4F879
:10E9D000881182401143022EC4F88811C5F80891AD
:10E9E0001ED00230636044F820800020BDE8F0872C
:10E9F000144B03B34FF4C870FFF73EF90446D0B18F
:10EA0000D5F84831002780E88800C5F848413846E5
:10EA10000123C4F88871C4F88C71002EE1D0D1E7CD
:10EA2000D4F88C110A43C4F88C21DAE705F5A674F2
:10EA3000C5F84841C1E74FF0FF30BDE8F08700BF9F
:10EA4000C80A010079DC0000024B13B1024800F053
:10EA500005B870470000000069EA00000023014685
:10EA60001A461846FFF79EBF38B5074D074C2C1BBA
:10EA7000A41005D0013C55F8043D9847002CF9D16D
:10EA8000BDE8384002F032B800000000000000008D
:10EA9000F8B5234F0C460646FFF768FCBB685D6877
:10EAA00025F00305291B01F6EF7121F47F6121F0A8
:10EAB0000F01A1F58054B4F5805F07DB00213046DB
:10EAC000FFF750FEBB682B44984204D03046FFF756
:10EAD0004FFC0020F8BD61423046FFF743FE013095
:10EAE0000DD0104BBA6819682D1B45F00105304652
:10EAF000091B55601960FFF73BFC0120F8BD0021A0
:10EB00003046FFF72FFEBA68831A0F2BDEDD064C66
:10EB10000449246843F00103001B53600860D5E7F3
:10EB2000E496FF1F60A1FF1FF09AFF1F002945D048
:10EB30002DE9F0410D468046FFF718FC55F8047C9E
:10EB40006A4927F00103A5F10804E2188E685068AD
:10EB5000B24220F0030062D0FE0750600BD455F89B
:10EB6000087CE41B01F1080EA56875453B446FD095
:10EB7000E768EF60BD6015186D68ED0742D543F09A
:10EB800001026260E350B3F5007F18D2DB085A1C23
:10EB90004D6851F83270A76001209B1000FA03F312
:10EBA00001EBC2001D430838E0604D6041F832407F
:10EBB000FC604046BDE8F041FFF7DABB70475A0AF7
:10EBC000042A53D89A0902F139077F0002F1380567
:10EBD00001EB870051F827204449083890424DD076
:10EBE000516821F003018B4202D292689042F7D122
:10EBF000D068E060A2608460D4604046BDE8F04127
:10EC0000FFF7B6BB95683A4FBD4203443FD0D0688A
:10EC1000E86043F0010285606260E350B3E7FF07FC
:10EC2000034407D455F8082CA41A1344A068E268DA
:10EC3000C26090602F4A126843F001009342606006
:10EC40008C60B6D32C4B40461968FFF721FFB0E724
:10EC500011184968C90744D49168D268CA6003444E
:10EC600043F0010091606060E350A2E7142A17D8D6
:10EC700002F15C077F0002F15B05A9E7AA104B686F
:10EC8000012505FA02F213434B600246B1E743F057
:10EC900001024C610C61E560A5606260E35088E7A9
:10ECA000542A06D81A0B02F16F077F0002F16E0595
:10ECB0008EE7B2F5AA7F06D8DA0B02F178077F005B
:10ECC00002F1770584E740F25450824206D89A0C4C
:10ECD00002F17D077F0002F17C0579E7FE277E25A2
:10ECE00076E743F001026260E35062E7E496FF1FBB
:10ECF000EC96FF1FEC9AFF1F5CA1FF1F0000D007DE
:10ED0000800CD80E0010C012EC130C17FA19141E48
:10ED10006022AC265C2B0C30BC34023AFF3FFFFF74
:10ED200000000000070000000C00000010000000C0
:10ED3000130000001A0000001F0000000000000087
:10ED4000070000000C00000010000000130000008D
:10ED5000180000001C0000000000CC10581BFC2113
:10ED6000AC26C62A7C2E3831F4334C36A438983A77
:10ED70005A3C543D803E7A3FFF3FFFFF0000FF03B7
:10ED8000FF07FF0BFF0FFF13FF17FF1BFF1FFF23E3
:10ED9000FF27FF2BFF2FFF33FF37FF3BFF3FFFFF17
:10EDA0000000D007100E88133219AA1E28237427DA
:10EDB0005C2B442F643284354038663A8C3C803E6C
:10EDC000FF3FFFFF0000900120031405D0075A0AFF
:10EDD000AC0DCC10B4146A18E81C342180252A2B01
:10EDE00070301437FF3FFFFF0000580246056608E9
:10EDF000540BD80E5C12E015FA19141E6022AC26D2
:10EE00005C2B0C30BC34023AFF3FFFFF0000C8000F
:10EE1000F4018403140508072E091C0CD80EF81100
:10EE2000AE159619401F1C25F22B5834FF3FFFFFEB
:10EE300000006400C8009001BC021A04DC059E07B3
:10EE4000F609800CA00F2413A2174C1D5424442F44
:10EE5000FF3FFFFF00000000070000000C00000063
:10EE60001000000013000000180000001A0000004D
:10EE7000070000000C00000010000000130000005C
:10EE8000180000001A0000001F00000000005802D7
:10EE900046056608540BD80E5C127017FC21F82A40
:10EEA00070305834DC37663A8C3C803EFF3FFFFFC1
:10EEB0000000580246056608540BA00FD4172823FB
:10EEC000F82A442F643284354038663A8C3C803EC0
:10EED000FF3FFFFF00007805220B0410B414321925
:10EEE000B01DFC214826FE29822D383126344637B4
:10EEF000663A223DFF3FFFFF0000540BEC13FA1966
:10EF000008201C253629EC2C0C302C33E8357238BF
:10EF1000663AF63B863D163FFF3FFFFF58ED000087
:10EF2000F8EE0000A0ED0000D4EE00007CED000043
:10EF3000E8ED0000C4ED00000CEE000030EE000033
:10EF40008CEE0000B0EE000040F00000FCEC000091
:10EF500000000000CDCC4C3DCDCCCC3D9A99193E63
:10EF6000CDCC4C3E0000803E9A99993E3333B33E5F
:10EF7000CDCCCC3E6666E63E0000000007000000F7
:10EF80000C0000001000000013000000180000003A
:10EF90001C00000000000000070000000C00000042
:10EFA00013000000180000001F00000024000000F3
:10EFB000000000000C000000180000002400000009
:10EFC000300000003C00000048000000000000008D
:10EFD000FBFFFFFFF4FFFFFFEFFFFFFFE8FFFFFF77
:10EFE000E3FFFFFFDCFFFFFF00000000F4FFFFFF77
:10EFF000E8FFFFFFDCFFFFFFD0FFFFFFC4FFFFFFC5
:10F00000B8FFFFFF2C011301FA00E100C800AF00B8
:10F0100096007D0064004B00320019004006780520
:10F02000B004E80384032003BC025802F4019001F9
:10F030002C01FA00C8009600640032001900FFFF9E
:10F04000000078053408540B800C3C0F5C12E0156E
:10F05000FA19141E6022AC265C2B0C30BC34023A28
:10F06000FF3FFFFFD4F000005A9CFF1F0000FF0F7E
:10F07000849DFF1F0000FF0F61370000A0F000001B
:10F08000CC9CFF1F32005E01000000000000000069
:10F090000137000054485200534E53004D41580070
:10F0A000544F5543482053454E53450045585452FC
:10F0B0004120434F4E54524F4C4C455200000000EB
:10F0C00050495443482042454E440000424954456B
:10F0D0000000000042524541544800FFACF00000DF
:10F0E0002A9DFF1FF401A00F929CFF1FF401A00FA7
:10F0F0000D370000CCF00000109DFF1FBC025C1219
:10F10000569CFF1FBC025C1245370000C0F0000097
:10F110006A9DFF1FF401A00FC89CFF1FF401A00F00
:10F1200029370000F4F80000FCF80000E8F80000BF
:10F13000ECF80000F0F8000094F70000ACF80000D4
:10F14000C8F80000CCF80000D0F80000D4F80000A7
:10F15000D8F80000DCF80000E0F80000B4F8000087
:10F16000E4F8000094F7000090F70000BCF80000FD
:10F17000C0F80000C4F8000094F70000ACF80000EC
:10F18000B0F80000B4F80000B8F8000098F80000EB
:10F190009CF80000A0F80000A4F80000A8F8000007
:10F1A000ACFD000090F8000094F8000004F90000A5
:10F1B00008F900000CF9000010F9000014F9000033
:10F1C00018F900001CF9000020F9000024F90000E3
:10F1D00028F900002CF9000030F9000034F9000093
:10F1E0000100000038F900000700000000000000E6
:10F1F00001000000D54400000000000000000000F5
:10F2000000000000000000000000000000000000FE
:10F2100000000000000000000000000000000000EE
:10F2200000000000000000000000000000000000DE
:10F2300000000000000000000000000000000000CE
:10F2400000000000000000000000000000000000BE
:10F2500000000000000000000000000000000000AE
:10F26000000000000000000000000000000000009E
:10F27000000000000000000000000000000000008E
:10F28000000000000000000000000000000000007E
:10F29000000000000000000000000000000000006E
:10F2A000000000000000000000000000000000005E
:10F2B000000000000000000000000000000000004E
:10F2C000000000000000000000000000000000003E
:10F2D000000000000000000000000000000000002E
:10F2E000000000000000000000000000000000001E
:10F2F000000000000000000000000000000000000E
:10F3000000000000000000000000000000000000FD
:10F310000000000000000000000000000001FFFFEE
:10F32000FFE3600007736000000000000001FFFFC2
:10F33000FFE360000EE360000000000000018000B9
:10F34000000360001DC36000000000000001BFFF5B
:10F35000FFE360003B836000000000000001BFFF8E
:10F36000FFE3600077036000000000000001B000D0
:10F3700000036000EE036000000000000001B00028
:10F3800000036001DC036000000000000001B00029
:10F3900000036003B8036000000000200001B0001B
:10F3A0000003600770036000000000600001BFFF01
:10F3B000FFE3600EE0036000000000600001BFFF9B
:10F3C000FFE3601DC00360000003006000018000D7
:10F3D0000003603B80036000000300E00001BFFF0A
:10F3E000FFE3607700036000000300C00001BFFF7F
:10F3F000FFE360EE00036000000380C00001B00086
:10F40000000361DC00036000000780C00001B00061
:10F41000000363B8000360000007C0C00001B00033
:10F4200000036770000360000006C0C00001B00068
:10F4300000036EE000036000000660C10101B0003F
:10F4400000037DC000036000000630C30301BFFF5E
:10F45000FFE37B8000036000000C30C30701BFFFA7
:10F46000FFE3770000036000000C1CC3060180006E
:10F4700000030E0000036000000C0CC20E01FFFF31
:10F48000FFE3FC0000036000000C0EC61E01FFFF3E
:10F49000FFE3F80000036000000C07C61E00000038
:10F4A0000000000000000000000C03C67600000011
:10F4B0000000000000000000000C01C7E600000092
:10F4C0000000000000000000000C00C7C6000000A3
:10F4D0000000000000000000000C00030600000017
:10F4E0000000000000000000000C00000000000010
:10F4F0000000000000000000000C00000000000000
:10F5000000000000000000000000000000000000FB
:10F5100000000000000000000000000000000000EB
:10F5200000000000000000000000000000000000DB
:10F5300000000000000000000000000000000000CB
:10F5400000000000000000000000000000000000BB
:10F5500000000000000000000000000000000000AB
:10F56000000000000000000000000000000000009B
:10F57000000000000000000000000000000000008B
:10F58000000000000000000000000000000000007B
:10F59000000000000000000000000000000000006B
:10F5A000000000000000000000000000000000005B
:10F5B000000000000000000000000000000000004B
:10F5C000000000000000000000000000000000003B
:10F5D000000000000000000000000000000000002B
:10F5E000000000000000000000000000000000001B
:10F5F0000000000000000000A8FA00000000050163
:10F600000B000000408DFF1F0544000006000000B5
:10F6100009000000F48EFF1F00000000BCFB00008A
:10F62000B0FB0000589DFF1F0000300000000000EC
:10F630000D520000C14200000000000034FA00003A
:10F6400000000101080000008C8EFF1F9CF90000E3
:10F65000000002010B0000003C8FFF1F00000000B3
:10F660008CFB000098FB0000889CFF1F000001003D
:10F6700001000000D5470000F54000000000000038
:10F6800001000000B0FA00000600000038F9000098
:10F690000000040508000000348BFF1F010000007B
:10F6A000A8FA0000090000000000000001000000AE
:10F6B000ED5D000001000000D0FA00000300000032
:10F6C00000000000D4FB0000B0FB0000549DFF1FB1
:10F6D00000003000000000000D520000C142000098
:10F6E000000000000000000001000000794E000052
:10F6F00000000000D8FA0000E0FA0000A69CFF1FFE
:10F700000100100006000000255A0000154100000D
:10F71000DD4B000000000000A4FB0000B0FB000077
:10F720005A9DFF1F00003000000000000D52000035
:10F73000C1420000000000007CFB0000000003014B
:10F7400006000000288DFF1F00000000E0FB000005
:10F75000B0FB00002E9DFF1F0000300000000000E5
:10F76000FD51000005410000000000000000000005
:10F7700094F9000060F90000A29CFF1F000009003E
:10F7800000000000F94700003541000000000000C3
:10F790004F4E00004F464600555342004241540030
:10F7A0004C4F5720000000004D454E552020202092
:10F7B000202020202058585820592E59560000004B
:10F7C00058000000524F54004D454C0044594E0023
:10F7D0006D73000042544800424954004C56520098
:10F7E0004E524D0052455600312F0000415400004A
:10F7F0004D4F4400504244004543420045435300AE
:10F800004C564C004C565000474C44004543480071
:10F81000762E0000312E342E370000005345540060
:10F82000434C52004E754556490000006669726DA2
:10F830007761726520762E0055534220706F776590
:10F8400072000000416C6B616C696E6520626174CE
:10F85000746572790000000030202520617420005A
:10F860004E694D4820626174746572790000000031
:10F870004C69506F206261747465727900000000F9
:10F88000444F4E275400000050414E4943000000B1
:10F890005450540048524E0048524D0035544800D0
:10F8A0004F43540035444E004F444E004D57000026
:10F8B00046500000434600005350000053570000DC
:10F8C00053454C005345450042520000564C000041
:10F8D000455800004D572B0042522B00564C2B0030
:10F8E00045582B00554E4F00414C4B004E4D4800A3
:10F8F0004C495000425254480000000050544348C4
:10F90000000000002D3400002D3300002D320000D7
:10F910002D3100004C494E002B3100002B320000ED
:10F920002B3300002B340000533100005332000011
:10F930005A3100005A3200005649425241544F0099
:10F94000444952454354494F4E000000434F4E54E2
:10F95000524F4C00535155454C4348204200000043
:10F960004C4556454C00000053454E5345204254EB
:10F9700045000000535155454C4348204C000000C1
:10F9800053454E5345204C565200000052455455A5
:10F99000524E000044455054480000005345545511
:10F9A00050204354524C530046494E474552494E0D
:10F9B000470000004C4556454C20434300000000E2
:10F9C00050494E4B59204B45590000004445474C87
:10F9D00049544348000000004841524D2053454CD3
:10F9E0000000000053455249455300004558435418
:10F9F000204841524D0000004841524D2052414E96
:10FA0000474500004558435420434320420000002E
:10FA1000455843542043432041000000504954437B
:10FA20004842454E44000000504F52542F474C442A
:10FA3000000000005345545550204252454154485F
:10FA40000000000056454C20424F4F535400000028
:10FA500056454C2044454C415900000043555256F0
:10FA60004500000056454C4F4349545900000000E2
:10FA70004252454154482041540000004343204233
:10FA8000205249534500000042525448204343202D
:10FA900042000000425254482043432041000000ED
:10FAA00041424F5554000000455854524153000004
:10FAB000524F5441544F52005345545550204354D3
:10FAC0004C000000534554555020425200000000A5
:10FAD00041444A55535400004D494449204348008D
:10FAE0004D4944492043484E4C00000042415420B7
:10FAF0005459504500000000574C204348414E00E7
:10FB0000574C20504F574552000000004641535477
:10FB100020424F4F54000000444143204F555400B1
:10FB200042434153204D4F4445000000335244208E
:10FB30005452494C4C00000053504543204B45590A
:10FB4000000000004741544520484F4C440000004D
:10FB50004C45474143592042520000004C45474123
:10FB600043592050420000004F4354415645000085
:10FB70005452414E53504F5345000000524F544190
:10FB8000544F522053455455500000005052494F95
:10FB900052495459000000004D4F4E4F20505249D9
:10FBA0004F000000524F54415445203400000000E3
:10FBB00053454D49544F4E4553000000524F544158
:10FBC0005445203300000000524F54415445203228
:10FBD00000000000524F5441544520310000000005
:10FBE000504152414C4C454C00FFFFFF01000000CA
:10FBF000C4FA0000040000002C0100000000000016
:10FC0000C8FB0000B0FB0000569DFF1F0000300045
:10FC1000000000000D520000C14200000000000082
:10FC200001000000B8FA000005000000000000001C
:10FC30005CFA00005CFA0000CE9CFF1F00000C0084
:10FC400003000000495900002541000000000000A9
:10FC500001000000A0FA00000800000000211102CD
:10FC600002000000002111020504FFFF003E7FFF9B
:10FC70004E75455649633031000000007676764E69
:10FC800075455649636363007676764E75455649E9
:10FC90006330346565767676767676767600000023
:10FCA000496E76616C696420636F6E666967206671
:10FCB0006F726D6174000000496E76616C6964203A
:10FCC000636865636B73756D00000000496E766153
:10FCD0006C696420636F6E6669672073697A65007A
:10FCE000496E76616C696420636F6E666967207621
:10FCF000657273696F6E0000496E76616C6964208D
:10FD00006D6573736167652E00000000653030001B
:10FD10006330300053656E64696E6720636F6E6692
:10FD200069672E2E2E000000436F6E666967207390
:10FD3000656E742E000000006330330053656E64FE
:10FD4000696E672076657273696F6E2E0000000021
:10FD500063303200526563656976696E6720636F50
:10FD60006E6669672E2E2E004E657720636F6E6675
:10FD700069672073617665642E000000556E6B6EB6
:10FD80006F776E206D6573736167652E00000000EC
:10FD900065303100436F6E666967206D676D740072
:10FDA000506F776572206F6666204E754556490024
:10FDB000746F20657869740052656164792E00FF64
:10FDC00034800440400000001211FFFFFF020200D7
:10FDD00000001310FFFFFF020200000018000000E7
:10FDE00034800440800000001EFFFFFFFF0200007F
:10FDF00000001DFFFFFFFF020000000019000000CF
:10FE000000000000000000002D7A0000F1790000E1
:10FE1000A5790000ED790000A9790000B57900000E
:10FE2000D5790000000103070F1F3F7F2200FF214B
:10FE300000FFFFFF0080C0E0F0F8FCFE00000000C3
:10FE40000000000085990000E19D0000A5790000F8
:10FE5000B1830000498400002D920000E191000070
:10FE600015920000ED91000001920000FD9000004D
:10FE70002D92000055920000458600008D8E0000F6
:10FE8000298E000025930000319200008993000024
:10FE900029940000DA02818FDA1281FF00006000ED
:10FEA00000000000000000000000000000E0000072
:10FEB000000000000000000000000001E000000061
:10FEC0000000000000000000000001F00000000041
:10FED00000000000000000000003F000000000002F
:10FEE000000000000000000007F00000000000001B
:10FEF0000000000000000007F80000000000000003
:10FF00000000000000000FF800000003C0007E00A9
:10FF10000001E0007F0FF800000003C000FE0000B9
:10FF200001E000FFEFF800000003C000FE00000148
:10FF3000E000FFFFF800000003C000F00000000F29
:10FF4000007FFE7FC0000003C000F00000000F0033
:10FF50003FFE7FF83FF1FBCFFCFEF3BC3DEFE01F1F
:10FF6000FE7FFF7FFBFFDFFEFEFFBC3DEFE01FC615
:10FF7000FFFF7FFBFFDFFEFEFFBC3DEFE00FE3C7AF
:10FF8000FE787BC3DE1EF0FFBC3DEF0007FF87FC61
:10FF9000787BC3DE1EF0F83C3DEF0001FFFFF00070
:10FFA0007BC3C01EF0F03C3DEF0001F37FE03FFB60
:10FFB000C3CFFEF0F03C3DEF0003E33F807FFBC387
:10FFC000DFFEF0F03C3DEF0007E73C00787BC3DE4E
:10FFD0001EF0F03C3DEF0007FFBE00787BC3DE1E45
:10FFE000F0F03C3DEF0007FFFE00787BC3DE1EF023
:10FFF000F03C3DEF000FFFFE007FFBFFDFFEF0F067
:020000021000EC
:100000003FFDEFE00FFFFF007FFBFFDFFEF0F03F63
:10001000FDEFE00FF9FF003E79F9CF9EF0F01F3DB4
:10002000E7E01FF1FF0000000000000000000000FA
:10003000001F80FF007FFFFFFFFFFFFFFFFFFFE0CC
:100040001C007F007FFFFFFFFEB46D888D18E0006D
:10005000001F007FFFFFFFFE95AD7DB577E000003C
:100060000F007FFFFFFFFEA5AD9D8D19E00000068C
:10007000007FFFFFFFFEB5ADEDB57EE0AED580A8F9
:10008000D300408D2000A1C8DB40A4A62EAFFFFF07
:1000900000000000000180000000000000000000DF
:1000A000038000000000000000000007C000000006
:1000B00000000000000007C0000000000000000079
:1000C000000FC00000000000000000001FE0000062
:1000D000000000000000001FE00000000000000021
:1000E00000003FE00000000000000000003FF000C2
:1000F00000000000000000007FF000000000000091
:10010000001FF87FF0000000000000003FFE7FF0BD
:10011000000000000000003FFF7FF0000000000032
:1001200000001FFFFBE0000000000000000FFFF9CF
:10013000FFC00000000000000FFFF9FFF800000002
:1001400000000007FFF1FFFF00000000000003FCBB
:1001500073FFFF80000000000001FE3FFFFF8000F2
:100160000000000000FF1E0FFF0000000000000064
:100170007FFE1FFC000000000000003FFFFFF800B2
:100180000000000000000FDFFFE0000000000000A2
:10019000001F19FFC0000000000000003F3CFF00EE
:1001A000000000000000007E7CF80000000000005D
:1001B00000007FFE7C0000000000000000FFFFFC4C
:1001C0000000000000000000FFFFFE000000000033
:1001D000000000FFFFFE0000000000000001FFEF34
:1001E000FE0000000000000001FFCFFE0000000044
:1001F00000000003FF07FE0000000000000003FCF9
:1002000007FE0000000000000003F003FE000000F5
:1002100000000000018000FE00000000000000005F
:1002200000007E000000000000000000003E000012
:1002300000000000000000000C00000000000007AB
:100240008000FC000003C0000000078001FC0000EB
:1002500003C0000000078001FC000003C000000094
:10026000078001E00000001E000000078001E000A0
:1002700000001E007FE3F79FF9FDE7787BDFC0FFFA
:10028000F7FFBFFDFDFF787BDFC0FFF7FFBFFDFD80
:10029000FF787BDFC0F0F787BC3DE1FF787BDE00B5
:1002A000F0F787BC3DE1F0787BDE0000F787803D0A
:1002B000E1E0787BDE007FF7879FFDE1E0787BDE81
:1002C00000FFF787BFFDE1E0787BDE00F0F787BC39
:1002D0003DE1E0787BDE00F0F787BC3DE1E0787B34
:1002E000DE00F0F787BC3DE1E0787BDE00FFF7FF42
:1002F000BFFDE1E07FFBDFC0FFF7FFBFFDE1E07F77
:10030000FBDFC07CF3F39F3DE1E03E7BCFC000000C
:10031000000000000000000000FFFFFFFFFFFFFFE4
:10032000FFFFFFC0FFFFFFFFFD68DB111A31C0FFB9
:10033000FFFFFFFD2B5AFB6AEFC0FFFFFFFFFD4BE6
:100340005B3B1A33C0FFFFFFFFFD6B5BDB6AFDC049
:10035000DA0281FF00000000000000008599000023
:10036000E19D0000A5790000B183000065A50000B3
:100370002D920000E191000015920000ED91000027
:1003800001920000FD9000002D92000055920000A7
:100390005192000079920000D19200002593000054
:1003A00031920000899300002994000000000000B1
:1003B000003E5B4F5B3E3E6B4F6B3E1C3E7C3E1CEB
:1003C000183C7E3C181C577D571C1C5E7F5E1C0031
:1003D000183C1800FFE7C3E7FF0018241800FFE7E8
:1003E000DBE7FF30483A060E2629792926407F05AB
:1003F0000507407F05253F5A3CE73C5A7F3E1C1CC1
:1004000008081C1C3E7F14227F22145F5F005F5F80
:1004100006097F017F006689956A6060606060946C
:10042000A2FFA29408047E040810207E2010080871
:100430002A1C08081C2A08081E101010100C1E0C7C
:100440001E0C30383E3830060E3E0E06000000000E
:100450000000005F00000007000700147F147F14F5
:10046000242A7F2A1223130864623649562050003A
:1004700008070300001C2241000041221C002A1C26
:100480007F1C2A08083E0808008070300008080811
:100490000808000060600020100804023E51494531
:1004A0003E00427F400072494949462141494D334F
:1004B0001814127F1027454545393C4A49493141B6
:1004C000211109073649494936464949291E000084
:1004D00014000000403400000008142241141414D9
:1004E0001414004122140802015909063E415D59C5
:1004F0004E7C1211127C7F494949363E41414122CE
:100500007F4141413E7F494949417F090909013EF7
:10051000414151737F0808087F00417F410020401E
:10052000413F017F081422417F404040407F021C30
:10053000027F7F0408107F3E4141413E7F09090947
:10054000063E4151215E7F09192946264949493213
:1005500003017F01033F4040403F1F2040201F3FD9
:100560004038403F6314081463030478040361595E
:10057000494D43007F4141410204081020004141A0
:10058000417F04020102044040404040000307084C
:100590000020545478407F28444438384444442848
:1005A000384444287F385454541800087E090218EF
:1005B000A4A49C787F0804047800447D4000204077
:1005C000403D007F1028440000417F40007C0478BB
:1005D00004787C080404783844444438FC18242403
:1005E0001818242418FC7C08040408485454542483
:1005F00004043F44243C4040207C1C2040201C3C00
:100600004030403C44281028444C9090907C4464F6
:10061000544C440008364100000077000000413689
:10062000080002010204023C2623263C1EA1A1610F
:10063000123A4040207A3854545559215555794141
:100640002254547842215554784020545579400C16
:100650001E527212395555555939545454593955F9
:100660005454580000457C410002457D420001453C
:100670007C407D1211127DF0282528F07C545545D0
:10068000002054547C547C0A097F4932494949323C
:100690003A4444443A324A4848303A4141217A3A4D
:1006A00042402078009DA0A07D3D4242423D3D4019
:1006B00040403D3C24FF2424487E4943662B2FFCC8
:1006C0002F2BFF0929F620C0887E09032054547976
:1006D000410000447D413048484A32384040227A47
:1006E000007A0A0A727D0D19317D2629292F2826C4
:1006F0002929292630484D402038080808080808CC
:100700000808382F10C8ACBA2F102834FA00007B24
:10071000000008142A142222142A14085500550037
:1007200055AA55AA55AAFF55FF55FF000000FF0026
:10073000101010FF00141414FF001010FF00FF1021
:1007400010F010F0141414FC001414F700FF000053
:10075000FF00FF1414F404FC141417101F10101FD2
:10076000101F1414141F00101010F0000000001FC0
:10077000101010101F10101010F010000000FF10CB
:100780001010101010101010FF10000000FF1400C7
:1007900000FF00FF00001F10170000FC04F41414F9
:1007A0001710171414F404F40000FF00F7141414C5
:1007B00014141414F700F7141414171410101F1045
:1007C0001F141414F4141010F010F000001F101F68
:1007D0000000001F14000000FC140000F010F010D6
:1007E00010FF10FF141414FF141010101F0000004D
:1007F00000F010FFFFFFFFFFF0F0F0F0F0FFFFFF51
:100800000000000000FFFF0F0F0F0F0F38444438A7
:1008100044FC4A4A4A347E02020606027E027E02F6
:1008200063554941633844443C04407E201E200601
:10083000027E020299A5E7A5991C2A492A1C4C723E
:1008400001724C304A4D4D303048784830BC625AC5
:10085000463D3E494949007E0101017E2A2A2A2A55
:100860002A44445F444440514A444040444A514031
:100870000000FF0103E080FF000008086B6B0836F2
:1008800012362436060F090F060000181800000063
:100890001010003040FF0101001F01011E00191D52
:1008A0001712003C3C3C3C00000000000D0AFFFF1A
:1008B000050E08090D0C06070F0400130393050E1F
:1008C00008090D0C06070F04FFFFC585848687C441
:1008D000FFFF001303931A9217FFFFFF6FF07F03D0
:1008E0000370037813F0800FFBD070474008FE437D
:1008F00040A004404408FE4344A004400018FE43C6
:1009000000C004403000FE43309004403400FE43F9
:10091000349004401C18FE431CC004401018FE43D1
:1009200010C004400818FE4308C004400C18FE43E1
:100930000CC004400C10FE430CB004401010FE43E9
:1009400010B004401810FE4318B004401C10FE43C1
:100950001CB004401410FE4314B004400418FE43BD
:1009600004C004400010FE4300B004400008FE43F1
:1009700000A004400408FE4304A004400C08FE4309
:100980000CA004400808FE4308A004401418FE43CD
:1009900014C004401818FE4318C004400410FE435D
:1009A00004B004400810FE4308B004401400FE43A5
:1009B000149004404C08FE434CA004400420FE4325
:1009C00004D004402410FE4324B004402010FE4311
:1009D00020B004402810FE4328B004402C10FE43F1
:1009E0002CB004400020FE4300D004404808FE43E1
:1009F00048A004401000FE4310900440090AFFFF85
:100A0000FFFFFFFFFFFFFFFFFFFFFF0D00060807CF
:100A1000FFFF0E0FFF0CFFFFFFFFFFFF0B05FFFFA8
:100A20001519151900010000D491FF1F12000000D4
:100A3000000200000092FF1F73000000002201006E
:100A40007492FF1F21000000002101005C92FF1F33
:100A500009000000000300009892FF1F0000000042
:100A600001030904E891FF1F0000000002030904CC
:100A7000E48FFF1F00000000030309049C92FF1F86
:100A80000000000000000000000000000000000066
:100A900065787000FFFFFFFF000000000000E03FEE
:100AA000000000000000E0BF763C7935EF39EA3DF8
:100AB000763C7935EF39EABD0000E0FE422EE63F94
:100AC0000000E0FE422EE6BFB892FF1FF8B500BF5F
:100AD000F8BC08BC9E46704749EA00003504000097
:0C0AE000B9360000B5520000217600007D
:040AEC00F8B500BF9A
:100AF00038B5084B1C681C6054B1074D94FAA4F338
:100B0000B3FA83F355F823309847631E1C40F5D1A0
:100B100038BD00BFA0D00440C491FF1F38B5084BBA
:100B20001C681C6054B1074D94FAA4F3B3FA83F324
:100B300055F823309847631E1C40F5D138BD00BFDF
:100B4000A0C00440A491FF1F38B5084B1C681C606E
:100B500054B1074D94FAA4F3B3FA83F355F8233054
:100B60009847631E1C40F5D138BD00BFA0B00440BB
:100B70007491FF1F38B5084B1C681C6054B1074DB9
:100B800094FAA4F3B3FA83F355F823309847631E1D
:100B90001C40F5D138BD00BFA0A004402491FF1F28
:100BA00038B5084B1C681C6054B1074D94FAA4F387
:100BB000B3FA83F355F823309847631E1C40F5D1F0
:100BC00038BD00BFA0900440EC90FF1F0000000063
:100BD000000102070B0102070B4A1400002000006D
:100BE0003200000001000000002000000020000092
:100BF00000100000AB0A00000008000066060000BC
:100C00005505000092040000000400008E0300005F
:100C100033030000E8020000AB02000024000000E3
:100C20000020000002000200FBFFFFFF00000000A8
:100C300000000000000000000000000000000000B4
:100C40000000000000000000000000000C00000098
:100C5000140500000C0000000000F0410200FFFF3E
:100C6000FFFF000064F00000F4F000000CF1000051
:100C7000DCF000007CF000000000000040F9000003
:100C800040F90000809DFF1F0000010001000000EE
:100C90000000000000000000000000000000000054
:100CA0002CFB00002CFB0000C09CFF1F0300040075
:100CB0000000000000000000000000000000000034
:100CC000000000004CF900004CF90000EA9BFF1FF7
:100CD0000000020001000000000000000000000011
:100CE000000000000000000074F9000060F900003E
:100CF0009C89FF1F01001E00000000000000000092
:100D000000000000000000000100000000000000E2
:100D1000A8F90000A8F90000F69CFF1F00000200DF
:100D200001000000000000000000000000000000C2
:100D30000000000028FA000028FA0000909CFF1F25
:100D4000000004000100000000000000000000009E
:100D50000000000000000000D8F90000E4F90000E5
:100D6000BC9CFF1F00000400010000000000000008
:100D7000000000000000000000000000B4F90000C6
:100D8000B4F900000A9CFF1F00007F000100000072
:100D90000000000000000000000000000000000053
:100DA00068F9000060F900007689FF1F010011005A
:100DB0000000000000000000000000000000000033
:100DC0000000000070FA000070FA0000E49CFF1FB1
:100DD0000000010001000000000000000000000011
:100DE00000000000108AFF1F6CF70000688FFF1FD3
:100DF000C889FF1F788BFF1F348AFF1FEC8AFF1FF3
:100E0000688EFF1F0000000094FA000094FA0000B2
:100E1000EC9BFF1F00000A00010000000000000022
:100E200000000000000000000000000080F9000049
:100E300060F900007489FF1F01000C000000000031
:100E400000000000000000000000000000000000A2
:100E500050FB000050FB0000809CFF1F00000100C1
:100E60000100000000000000000000000000000081
:100E70000000000050FA000050FA0000E89CFF1F3C
:100E800000001E0001000000000000000000000043
:100E900000000000000000007CFA00007CFA000066
:100EA000FA9BFF1F01000A00010000000000000083
:100EB0000000000000000000000000000CFB00002B
:100EC0000CFB0000769DFF1F0000010000000000E9
:100ED0000000000000000000000000000000000012
:100EE00020FB000020FB0000289DFF1F00000100E8
:100EF00000000000000000000000000000000000F2
:100F0000000000001CFA00001CFA0000F89CFF1F03
:100F100000000C00000000000000000000000000C5
:100F2000000000000000000038FB000038FB00005B
:100F3000209DFF1F000001000100000000000000D4
:100F4000000000000000000000000000F8FA0000AF
:100F5000F8FA0000BC8FFF1F0400500000000000E2
:100F60000000000000000000000000000000000081
:100F700000FB000000FB0000089EFF1F00000300B4
:100F80000000000000000000000000000000000061
:100F90000000000070FB000070FB00003A9DFF1F86
:100FA0000000180000000000000000000000000029
:100FB000000000000000000044FA000044FA0000B5
:100FC000E89BFF1F00000900010000000000000076
:100FD000000000000000000048F70000C0F600001C
:100FE000FCFB000018F6000014F700005CF600009F
:100FF000908DFF1F9C8BFF1F448EFF1F748CFF1F63
:10100000EC89FF1F2C8CFF1FC08FFF1FFC8DFF1F63
:10101000088CFF1FBC8CFF1F988CFF1F0000000076
:10102000ECF90000F8F900006E9DFF1F00000600BB
:1010300001000000000000000000000000000000AF
:10104000000000005CFB00005CFB0000269DFF1F11
:10105000000001000100000000000000000000008E
:101060000000000000000000C0F90000C0F900000E
:101070005C9CFF1F00001E0000000000000000003C
:1010800000000000000000000000000010FA000056
:1010900010FA0000249DFF1F000004000100000062
:1010A0000000000000000000000000000000000040
:1010B000ECFA0000ECFA0000689DFF1F000002003F
:1010C000010000000000000000000000000000001F
:1010D0000000000068FB000068FB0000849CFF1F0C
:1010E00000000600000000000000000000000000FA
:1010F000000000000000000044FB000044FB000072
:10110000B49CFF1F0000010001000000000000006F
:1011100000000000000000000000000054F9000082
:1011200060F90000A489FF1F01001E0000000000FC
:10113000000000000000000000000000548BFF1FB2
:10114000AC8EFF1FE48BFF1F108BFF1F188FFF1F3C
:101150002CFC0000C08BFF1F048DFF1F000000004F
:1011600088FA000088FA0000F29CFF1F00007F0050
:10117000010000000000000000000000000000006E
:1011800000000000CCF90000CCF90000829DFF1F98
:101190000000460000000000000000000000000009
:1011A00000000000E08CFF1F208EFF1FF0F6000003
:1011B000B4F60000ECFB000020FC000080F600000C
:1011C0009CF6000050FC00000000000064FA0000E3
:1011D00064FA00007E9DFF1F00007F0001000000F8
:1011E000000000000000000000000000808AFF1FD7
:1011F000D88DFF1F988FFF1F6C8DFF1FA48AFF1FC4
:10120000E0F10000D08EFF1FB48DFF1FC88AFF1FC2
:101210005C8AFF1F508CFF1F000000008CF900004B
:1012200060F90000AC89FF1F00000400000000000E
:1012300000000000000000000000000000000000AE
:1012400001000000000000000000000004FA00009F
:1012500004FA0000DC9BFF1F00007F00010000007B
:10126000000000000000000000000000040000007A
:101270000000000018FB000018FB0000CA9CFF1FC4
:10128000000001000000000000000000000000005D
:101290000000000016034E0075004500560049008E
:1012A00020004D00490044004900000008FE0000F5
:1012B00000000000E803000000000000006006409D
:1012C000C0FD000000000000000000000000000061
:1012D000000000000000000000000000000000000E
:1012E00000000000000000000000000000000000FE
:1012F00000000000000000000000000000000000EE
:1013000000000000000000000000000000000000DD
:10131000000000000000000008FE000000000000C7
:10132000E80300000000000000700640E0FD00003F
:1013300000000000000000000000000000000000AD
:10134000000000000000000000000000000000009D
:10135000000000000000000000000000000000008D
:10136000000000000000000000000000000000007D
:10137000000000000000000000000000000000006D
:1013800000000000B59C0000B59C0000B59C00006A
:10139000B59C00000A040000C0A2FF1FF1A50000D8
:1013A000F1A50000F1A50000F1A50000F1A50000E5
:1013B000F1A50000F1A50000F1A50000F1A50000D5
:1013C000F1A50000F1A50000F1A50000F1A50000C5
:1013D000F1A50000F1A50000F1A50000F1A50000B5
:1013E000F1A50000F1A50000F1A50000F1A50000A5
:1013F000F1A50000F1A50000F1A50000F1A5000095
:10140000F1A50000F1A50000F1A50000F1A5000084
:10141000F1A50000F1A50000F1A50000F1A5000074
:10142000F1A50000F1A50000F1A50000F1A5000064
:10143000F1A50000F1A50000F1A50000F1A5000054
:10144000F1A50000F1A50000F1A50000F1A5000044
:10145000F1A50000F1A50000F1A50000F1A5000034
:10146000F1A50000F1A50000F1A50000F1A5000024
:10147000F1A50000F1A50000F1A5000008000000A2
:10148000FFFFFFFF1201100100000040C01685049D
:101490007502010203010000180354006500650095
:1014A0006E00730079006400750069006E006F00C3
:1014B00009027300020100C03209040000020103A6
:1014C0000000072401000125000624020101000696
:1014D000240202020009240301030102010009247D
:1014E000030204010101000905040240000000009C
:1014F00005250101010905830240000000000525C2
:101500000101030904010002030000000921110187
:1015100000012221000705810340000107050203A5
:101520002000020006C9FF0904A15C750815002609
:10153000FF00954009758102952009769102950476
:101540000976B102C0000000040309040C03000086
:10155000000000000000000000000000000000008B
:10156000000001000000000000000000A495FF1F23
:101570000C96FF1F7496FF1F000000000000000083
:10158000000000000000000000000000000000005B
:10159000000000000000000000000000000000004B
:1015A000000000000000000000000000000000003B
:1015B000000000000000000000000000000000002B
:1015C000000000000000000000000000000000001B
:1015D000000000000000000000000000000000000B
:1015E00000000000000000000000000000000000FB
:1015F00000000000000000000000000000000000EB
:1016000000000000000000000000000000000000DA
:1016100001000000000000000E33CDAB34126DE677
:10162000ECDE05000B0000000000000000000000E0
:1016300000000000000000000000000000000000AA
:10164000000000000000000000000000000000009A
:10165000000000000000000000000000000000008A
:10166000000000000000000000000000000000007A
:10199000B892FF1F0000000000000000E496FF1F47
:1019A000E496FF1FEC96FF1FEC96FF1FF496FF1FB7
:1019B000F496FF1FFC96FF1FFC96FF1F0497FF1F66
:1019C0000497FF1F0C97FF1F0C97FF1F1497FF1F13
:1019D0001497FF1F1C97FF1F1C97FF1F2497FF1FC3
:1019E0002497FF1F2C97FF1F2C97FF1F3497FF1F73
:1019F0003497FF1F3C97FF1F3C97FF1F4497FF1F23
:101A00004497FF1F4C97FF1F4C97FF1F5497FF1FD2
:101A10005497FF1F5C97FF1F5C97FF1F6497FF1F82
:101A20006497FF1F6C97FF1F6C97FF1F7497FF1F32
:101A30007497FF1F7C97FF1F7C97FF1F8497FF1FE2
:101A40008497FF1F8C97FF1F8C97FF1F9497FF1F92
:101A50009497FF1F9C97FF1F9C97FF1FA497FF1F42
:101A6000A497FF1FAC97FF1FAC97FF1FB497FF1FF2
:101A7000B497FF1FBC97FF1FBC97FF1FC497FF1FA2
:101A8000C497FF1FCC97FF1FCC97FF1FD497FF1F52
:101A9000D497FF1FDC97FF1FDC97FF1FE497FF1F02
:101AA000E497FF1FEC97FF1FEC97FF1FF497FF1FB2
:101AB000F497FF1FFC97FF1FFC97FF1F0498FF1F61
:101AC0000498FF1F0C98FF1F0C98FF1F1498FF1F0E
:101AD0001498FF1F1C98FF1F1C98FF1F2498FF1FBE
:101AE0002498FF1F2C98FF1F2C98FF1F3498FF1F6E
:101AF0003498FF1F3C98FF1F3C98FF1F4498FF1F1E
:101B00004498FF1F4C98FF1F4C98FF1F5498FF1FCD
:101B10005498FF1F5C98FF1F5C98FF1F6498FF1F7D
:101B20006498FF1F6C98FF1F6C98FF1F7498FF1F2D
:101B30007498FF1F7C98FF1F7C98FF1F8498FF1FDD
:101B40008498FF1F8C98FF1F8C98FF1F9498FF1F8D
:101B50009498FF1F9C98FF1F9C98FF1FA498FF1F3D
:101B6000A498FF1FAC98FF1FAC98FF1FB498FF1FED
:101B7000B498FF1FBC98FF1FBC98FF1FC498FF1F9D
:101B8000C498FF1FCC98FF1FCC98FF1FD498FF1F4D
:101B9000D498FF1FDC98FF1FDC98FF1FE498FF1FFD
:101BA000E498FF1FEC98FF1FEC98FF1FF498FF1FAD
:101BB000F498FF1FFC98FF1FFC98FF1F0499FF1F5C
:101BC0000499FF1F0C99FF1F0C99FF1F1499FF1F09
:101BD0001499FF1F1C99FF1F1C99FF1F2499FF1FB9
:101BE0002499FF1F2C99FF1F2C99FF1F3499FF1F69
:101BF0003499FF1F3C99FF1F3C99FF1F4499FF1F19
:101C00004499FF1F4C99FF1F4C99FF1F5499FF1FC8
:101C10005499FF1F5C99FF1F5C99FF1F6499FF1F78
:101C20006499FF1F6C99FF1F6C99FF1F7499FF1F28
:101C30007499FF1F7C99FF1F7C99FF1F8499FF1FD8
:101C40008499FF1F8C99FF1F8C99FF1F9499FF1F88
:101C50009499FF1F9C99FF1F9C99FF1FA499FF1F38
:101C6000A499FF1FAC99FF1FAC99FF1FB499FF1FE8
:101C7000B499FF1FBC99FF1FBC99FF1FC499FF1F98
:101C8000C499FF1FCC99FF1FCC99FF1FD499FF1F48
:101C9000D499FF1FDC99FF1FDC99FF1FE499FF1FF8
:101CA000E499FF1FEC99FF1FEC99FF1FF499FF1FA8
:101CB000F499FF1FFC99FF1FFC99FF1F049AFF1F57
:101CC000049AFF1F0C9AFF1F0C9AFF1F149AFF1F04
:101CD000149AFF1F1C9AFF1F1C9AFF1F249AFF1FB4
:101CE000249AFF1F2C9AFF1F2C9AFF1F349AFF1F64
:101CF000349AFF1F3C9AFF1F3C9AFF1F449AFF1F14
:101D0000449AFF1F4C9AFF1F4C9AFF1F549AFF1FC3
:101D1000549AFF1F5C9AFF1F5C9AFF1F649AFF1F73
:101D2000649AFF1F6C9AFF1F6C9AFF1F749AFF1F23
:101D3000749AFF1F7C9AFF1F7C9AFF1F849AFF1FD3
:101D4000849AFF1F8C9AFF1F8C9AFF1F949AFF1F83
:101D5000949AFF1F9C9AFF1F9C9AFF1FA49AFF1F33
:101D6000A49AFF1FAC9AFF1FAC9AFF1FB49AFF1FE3
:101D7000B49AFF1FBC9AFF1FBC9AFF1FC49AFF1F93
:101D8000C49AFF1FCC9AFF1FCC9AFF1FD49AFF1F43
:101D9000D49AFF1FDC9AFF1FDC9AFF1F000002008D
:041DA000FFFFFFFF43
:00000001FF
